:020000042A00D0
:10000000D1DC4B843410D7730D000000FFFFFFFFDD
:10001000FFFFFFFF500000005000002AE010010029
:10002000E0F7000030F8002A0001000030F9002A53
:10003000001800000100000001000000FFFFFFFFAA
:10004000FFFFFFFFFFFFFFFFFFFFFFFFFFFFFFFFC0
:100050003A3500EA98D3002A98D3002A98D3002A88
:1000600098D3002A98D3002A98D3002A98D3002A3C
:1000700098D3002A7847C046640051E32033000A31
:100080000000B0E31EFF2FE130B48E4A08290FD3E1
:100090008D4C0578130A12026B405B00E35A534003
:1000A0001A04120C08390904090C401C0829F0D262
:1000B000002917D000780302491E08048349000C68
:1000C00014005C40240403D55204120C4A4001E0A1
:1000D0005204120C5B041B0C0400401E0004000CB4
:1000E000002CEDD1D04330BC0004000C704710B49C
:1000F000744A08290DD3764B047854402406E40D45
:100100001C5B120A624008390904090C401C0829CA
:10011000F2D2002914D000780302491E08046D4968
:10012000000C14005C40E40702D052084A4000E092
:1001300052085B080400401E0004000C002CF0D1A3
:10014000D04310BC0004000C704730B4624A082948
:100150000ED3624B0578940D6C402406A40D1C59F7
:100160001202624008390904090C401C0829F1D226
:10017000002914D000788305491E08045849000C52
:1001800014005C40A40002D552004A4000E0520036
:100190005B000400401E0004000C002CF0D1D04392
:1001A00030BC80008008704730B44B4B8343082A32
:1001B0000ED34A480D789C0D6C402406A40D0459BA
:1001C0001B026340083A1204120C491C082AF1D29F
:1001D000002A14D008788105521E1004404A000CF1
:1001E0001C004C40A40002D55B00534000E05B00C3
:1001F00049000400401E0004000C002CF0D1D8433C
:1002000030BC80008008704730B4C0430004000C4C
:10021000002A0FD02C4C0D78030A00026B405B00C3
:10022000E35A43401804000C521E1204120C491CDD
:10023000002AF0D1C04330BC0004000C704710B459
:10024000C0430004000C002A0BD0214B0C78444022
:100250002406E40D1C5B000A6040521E491C002A63
:10026000F4D1C04310BC0004000C7047030030B44C
:10027000100008290DD31B4A1D78040E6C40A40001
:1002800014590002604008390904090C5B1C082954
:10029000F2D2002913D01A781206491E124B090413
:1002A000090C0400544002D54000584000E04000D2
:1002B00052000C00491E0904090C002CF1D130BC7D
:1002C00070470000FFFF0000B0E1002A211000008D
:1002D000B0E3002A08840000FFFFFF3FB0DD002AE2
:1002E000C7B93060B0E5002AB71DC1040021016024
:1002F0004160704710B5254C20680DF0DBF90128EE
:100300000DD160680DF0D6F9002806D100F0C6F8CE
:1003100060680DF0CFF90028F8D01D48046110BCCA
:1003200008BC1847FFF7E6FF00F0F7F81948184C2B
:1003300020606060A060E0601748FFF7D7FF1748B3
:1003400061680DF0B8F91648A1680DF0B4F91548C8
:10035000E1680DF0B0F901F06EFC134C200000F0E4
:10036000A4F8FBE7002070470020704710B5642117
:10037000484300F09AF810BC08BC184770470020AA
:100380000A49401C8842FCDB70470000F8EF002A55
:10039000C4EF002AED02002A4038012A4838012A19
:1003A0005038012A5838012A10270000E8030000BD
:1003B00010B53148006802F09FF910BC08BC18471E
:1003C00010B501F067FD10BC08BC184710B501F06E
:1003D000ACFD002807D0284C206802F08DF901F010
:1003E000A4FD0028F8D110BC08BC184701207047B4
:1003F00010B504006068022806D1E169606900F068
:100400008BF9200001F0D1FD10BC08BC184738B5AD
:10041000002001F094FC01200023009017491848A7
:100420001A0001F09CFC144D286000281FD0C06801
:10043000002102F02DFE1349441828680021C068ED
:1004400002F026FE201A002811DD286802F054F977
:100450002868C169002903D038BC08BC01201847AE
:10046000C068002102F014FE201A0028EDDC38BC20
:1004700008BC002018470000D8EF002ADCEF002A53
:10048000F103002A20A10700FEE77047114901206F
:100490008863114908631149086070470D490120BC
:1004A000C8630D4900200863704770B5094C0025EA
:1004B000A5600121E1600DF027FA094A094B0DF012
:1004C0002BFA0DF0BBF9A1688142FCD3E56070BC4A
:1004D00008BC184700A000020000401A40A000021B
:1004E0008DEDB5A0F7C6A03F70B50400200004E074
:1004F000521E0B78491C0370401C002A05D0CB0704
:10050000DB0FC507ED0F2B43F2D1002A01D00CF011
:1005100071FC200070BC08BC184710B4FF4B0022CF
:100520001A609A800120411E8C0109190901CC181A
:100530008101411809015C50C9188A80401C1E289D
:10054000F1DBF749F74801624262C26202708262DF
:100550000121417010BC704710B4F24AF24CD06ACD
:1005600000238188C91EA14202D3838010BC70473A
:10057000916A002905D00860D06A9062D36210BCED
:10058000704790625062D36210BC7047F8B5E74F75
:100590003868C0680DF08EF8386801697E200DF06B
:1005A0008AF801250024DF48016B002918D9E043AF
:1005B000C00603D13868C0680DF07CF8DC48065DE1
:1005C0007E2E26D07D2E24D0396830060969000E93
:1005D0000DF071F86D1C641CD248006B8442E6D3A8
:1005E0003868C0680DF066F8386801697E200DF043
:1005F00062F86D1CA80609D1386801697E200DF0EB
:100600005AF8386801697E200DF055F8F8BC08BC2E
:100610001847386801697D200DF04DF820203968B1
:10062000464030060969000E0DF045F8AD1CD2E7D2
:1006300010B5BC4C206BC004010CBD48FFF757FD42
:10064000BB4A216B5054000A52185070891C216318
:1006500010BC08BC184700210278401C002A04D0B6
:10066000491C0278401C002AFAD10800704770B576
:1006700003001800FFF7EFFF0400AD4D0E202870B7
:1006800022001900681CFFF72FFFA649641C601C9C
:100690000A2208632A55FFF7CBFFFFF777FF70BCEC
:1006A00008BC184770B59F4C2169491C2161E16A5B
:1006B0000025002907D1216A00291CD0E1620A68BF
:1006C00022628D800D607D2821D07E2819D0E16ABC
:1006D000984B8A889A4207D22378002B02D0202395
:1006E00058402570891D5054E06A8188491C8180DA
:1006F00070BC08BC184790A0FFF7B9FF70BC08BCDD
:100700001847FFF729FF257070BC08BC1847012067
:10071000207070BC08BC1847F3B5050081B0814952
:1007200002980A6910180861C86A002808D1086A86
:10073000002853D0C86202680A62002282800260E8
:100740007848C66AB488B61D0298042831DD286846
:100750000090010E7D2948D00202130E7D2B44D05B
:100760000204120E7D2A40D00006000E7D283CD0E7
:100770007E293AD07E2B38D07E2A36D07E2834D0BF
:10078000301904226946FFF7AFFE664A1078002848
:1007900005D0305D20214840305500201070241DC8
:1007A0002404240C2D1D0298001F02900298042896
:1007B000CDDC029F7F1E14D328787D284AD07E2866
:1007C0003DD05C498C424AD256490A78002A45D02D
:1007D0002022504030550020087040E056A0FFF71E
:1007E00046FF03B0F0BC08BC1847032728787D28D3
:1007F00019D07E280CD04F498C4219D2494A117821
:10080000002914D0202148403055002010700FE0FE
:10081000002C04D04348C06A8480FFF79DFE414904
:100820000020087007E03F490120087003E03055C0
:10083000641C2404240C6D1C7F1ED7D2B3E7002C4B
:1008400004D03848C06A8480FFF786FE354900200E
:10085000087007E033490120087003E03055641C3C
:100860002404240C6D1C7F1EA6D203B0F0BC08BC6F
:100870001847F8B51C252B4F7869FFF7ECFE0400EC
:10088000354879692200FFF72FFE2200324E0832E8
:10089000944219DA31493B69402C0BDBB869FFF708
:1008A000DAFE05002C48B9692A00FFF71DFE00207A
:1008B000705509E01800E8400007000F085C30554B
:1008C0002D1F641C9442E7DB002030552248FFF7BF
:1008D000CEFEF8BC08BC184770B504000D00280017
:1008E000FFF7B9FE06002800FFF7C1FE10480D21F2
:1008F00001704470210A8170210CC170210E0171B8
:1009000032002900401DFFF7EFFD0648761D066303
:10091000FFF78EFEFFF73AFE70BC21E06038012A37
:1009200030AE012A0CF0002A05040000D4EF002AA2
:1009300044B6012A070400004552523A2057696E16
:10094000646F77206F76657272756E20646574656A
:10095000637465642E2E2E0044C6012AB0E9002A75
:1009600008BC184710B50520F6A1FFF7B5FF10BC6D
:1009700008BC00201847F8B50400F6492022E01D05
:100980000CF0FCF9002807D00520F3A1FFF7A4FF25
:10099000F8BC08BC0020184726002036307A022810
:1009A00007D20520F2A1FFF797FFF8BC08BC002092
:1009B0001847A088242807D20320F4A1FFF78CFF52
:1009C000F8BC08BC00201847FA4800254570FA48D2
:1009D00002270770F9492022401CFFF785FDF84CDB
:1009E0006770A770E570042020716571A571E571CD
:1009F00025726572A57203F0ADFD0300002B20D0B7
:100A00001800FFF728FE0206120EE272ED481900E8
:100A1000FFF76AFDE47A2C34E74F1E20611C38553D
:100A20004C1C7D54381903F097FD0119727A192076
:100A30000240481C7A54E449D2060AD501220A70C1
:100A400008E00820E1A1FFF747FFF8BC08BC002040
:100A500018470D70D74908630121C902884204D99B
:100A60000720E1A1FFF738FFFEE7FFF7E1FDFFF701
:100A70008DFD0024E64DE00040194068002801D0BB
:100A80000CF018FE641C042CF5DBF8BC08BC00203C
:100A9000184710B50520DFA1FFF71EFF10BC08BCEA
:100AA00000201847F0B583B005210291841D80888D
:100AB000262808D00320DDA1FFF70EFF03B0F0BC0D
:100AC00008BC00201847657820002030C17886785F
:100AD00009020E430779407900020743FF211931CB
:100AE000601CFFF704FBD7498E4208D00298D6A1BC
:100AF000FFF7F2FE03B0F0BC08BC002018478742A5
:100B000008D00298DCA1FFF7E7FE03B0F0BC08BCF8
:100B100000201847012D04D0022D07D0032D15D039
:100B200065E00520BBA1FFF7D7FE60E003F03AFFC8
:100B3000002807D0DAA1FFF7CFFE03B0F0BC08BC55
:100B400000201847DFA0FFF792FD50E0E078A6787C
:100B50006179000206432079000409060843064330
:100B6000201DC178A47909020C4301794079090458
:100B7000000601430C43E44833008021DBA20094CB
:100B80000CF068F8E048FFF772FD0125AD02DE4881
:100B90002B008021DDA20CF05DF8DB48FFF767FD3C
:100BA000E248019029006002A84200D201000198A9
:100BB0000CF0CAF9002C17D002273D00022C00D2FD
:100BC0002500019A2900300003F020FF002807D0FB
:100BD000D7A1FFF781FE03B0F0BC08BC0020184786
:100BE0007619641B002CE8D1D6A0FFF740FD7248AF
:100BF000242101706F4A01211163D849401C03F080
:100C000042FF002807D0D6A1FFF766FE03B0F0BC74
:100C100008BC00201847FFF70BFDFFF7B7FC03B037
:100C2000F0BC08BC0020184710B56248C1780279B2
:100C3000114307D00F20D0A1FFF74EFE10BC08BC17
:100C4000002018475C4A0C21117001210163FFF755
:100C5000EFFCFFF79BFCCF48006880680CF02AFD92
:100C6000FFF714FCFFF710FC10BC08BC002018476D
:100C700010B50520C8A1FFF72FFE10BC08BC00204E
:100C8000184770B50300981D9988491F0A04120C73
:100C900081784478037909020C43C17809041B0662
:100CA00019430C43401D210001431143C9070BD0D8
:100CB00015009E4B01001800FFF716FC9B482A0008
:100CC000210003F086FD02E0210003F082FD0028F0
:100CD00006D0B8A1FFF700FE70BC08BC0020184782
:100CE0003548082101704470210A8170210CC170BF
:100CF000210E01712F4905200863FFF799FCFFF7CA
:100D000045FC70BC08BC0020184710B5294CE078A1
:100D1000217908430DD001212748C90203F0D6FDEF
:100D200000280ED0A8A1FFF7D7FD10BC08BC0020FA
:100D300018470F20A8A1FFF7CFFD10BC08BC00206A
:100D400018475DE1496E76616C696420436F6D6D93
:100D5000616E6400C1E9002A496E76616C696420A5
:100D60006D61676963206E756D62657200000000D9
:100D7000496E76616C69642070726F746F636F6C1A
:100D80002076657273696F6E0000000050617261B9
:100D90006D6574657220526571756573742050615C
:100DA000636B6574204C656E677468204572726F62
:100DB000720000000CF0002A44B6012AE2E9002A81
:100DC00064B6012A70B6012ABDF2002A556E72651A
:100DD000636F676E697A656420666C61736820640E
:100DE0006576696365000000496E7465726E616CBA
:100DF000206572726F72202D207265706C795F624F
:100E00007566666572206F76657272756E00000099
:100E10004038012A46656174757265206E6F7420D2
:100E2000636F6D70696C656420696E00496E7661F0
:100E30006C6964207061636B6574206C656E6774A7
:100E400068000000ADDE00004750502F496E666F0D
:100E500020636F6D6D616E64206661696C65642EE0
:100E600020496E76616C6964204D61676963204E2C
:100E7000756D6265720000004750502F496E666FB5
:100E800020636F6D6D616E64206661696C65642EB0
:100E900020496E76616C6964204352430000000073
:100EA0005365742061637469766520626F6F742086
:100EB000706172746974696F6E206661696C6564D3
:100EC00000000000536574206163746976652062D8
:100ED0006F6F7420706172746974696F6E207375BE
:100EE000636365737366756C6C7900007A65726F05
:100EF0006F75742073746172742025642C206C6586
:100F00006E2025640000000084C6012A7A65726F95
:100F1000696E67206F75742025642062797465732B
:100F200020617420612074696D65000040B2012A5F
:100F30005A65726F696E67206F7574206661696C9F
:100F4000656400005A65726F6564206F7574207364
:100F500075636365737366756C6C79003CF0002A89
:100F6000506172746974696F6E20696E666F206675
:100F700061696C656400000043616E6E6F7420727D
:100F800065736574206265666F726520636C6F734C
:100F900065000000D4EF002A53696D706C652077FE
:100FA00072697465206E6F7420616C6C6F77656414
:100FB00000000000577269746520756E7375636375
:100FC00065737366756C00004572617365206661B8
:100FD000696C65640000000043616E6E6F7420658B
:100FE00072617365207768656E206E6F7420707211
:100FF0006576696F75736C79206F70656E656400D6
:10100000F9491E20087001202063FFF711FBFFF74C
:10101000BDFA10BC08BC0020184710B5811D80889F
:10102000401E0404240CF0480A2202702200491CCD
:10103000401CFFF759FAED48641C0463FFF7F8FA07
:10104000FFF7A4FA10BC08BC0020184710B5E64909
:1010500012200870E549012008631520E4A1FFF77C
:101060003BFC10BC08BC0020184770B5C479DF4DAC
:101070002879002810D0A04207D00F20E2A1FFF766
:101080002BFC70BC08BC00201847E8A0FFF7EFFA63
:1010900070BC08BC00201847200003F08FFA00281D
:1010A00007D00720ECA1FFF717FC70BC08BC00209C
:1010B00018472C71CC491420087001202863FFF7D1
:1010C000B7FAFFF763FA70BC08BC0020184710B5E8
:1010D000C64CE078217908430AD003F076FB00285B
:1010E0000ED0E0A1FFF7F8FB10BC08BC00201847A9
:1010F0000F20E0A1FFF7F0FB10BC08BC0020184750
:101100000020E0702071B84916200870012020638B
:10111000FFF78EFAFFF73AFA10BC08BC0020184718
:1011200010B5C07903F046FA002806D0DBA1FFF71E
:10113000D3FB10BC08BC00201847AC4901208860D4
:10114000A94B18221A700863FFF772FAFFF71EFA0C
:1011500010BC08BC0020184770B503000833818814
:10116000891E0A04120CC179A04CA068012807D07E
:101170000F20D1A1FFF7B0FB70BC08BC00201847BE
:1011800001204002824207D90320D8A1FFF7A4FB27
:1011900070BC08BC00201847180003F00DFA924AF2
:1011A00000211A230225002817D0607904280BD0CB
:1011B000E160137050702563FFF73AFAFFF7E6F924
:1011C00070BC08BC00201847E1600720CFA1FFF7E2
:1011D00083FB70BC08BC002018470120E06013703E
:1011E00051702563FFF724FAFFF7D0F970BC08BCF3
:1011F0000020184770B503000833C5798088801E29
:101200000204120C794CA068012807D00F20C9A154
:10121000FFF762FB70BC08BC00201847E06801289B
:1012200007D00F20CEA1FFF757FB70BC08BC0020F1
:1012300018472900180003F026FA6B4902221C23E4
:1012400000281CD0A07904280DD0012813D0022832
:1012500011D003280FD00720CDA1FFF73DFB70BCB4
:1012600008BC002018470720C9A1FFF735FB70BC58
:1012700008BC002018470B704870226304E0E5703A
:101280000B70002048702263FFF7D2F9FFF77EF958
:1012900070BC08BC0020184770B5831D80880728E3
:1012A00007D0C4490320FFF717FB70BC08BC00201F
:1012B0001847987859781A7900020143D8780004C1
:1012C00012061043014398795C790002044301201F
:1012D0008002844207D90320B7A1FFF7FDFA70BC52
:1012E00008BC00201847404D202228002A705A7858
:1012F00042709A788270DA78C2701A790271C01DD1
:10130000220003F004FC0004000C06D0AFA1FFF79C
:10131000E3FA70BC08BC002018476C71200AA87161
:101320003248E41D0463FFF783F9FFF72FF970BC1F
:1013300008BC00201847F7B5A94B07000C009D44D6
:101340000126F6026D4632003A21280003F09BF98F
:10135000002809D09DA1FFF7BFFA0020C043A14B90
:101360009D44F0BC08BC184732000021280003F05F
:10137000CEFB0004000C002805D09BA1FFF7ACFABF
:101380000120C043EBE7A24B28196B449A68203038
:1013900039000BF02FFD32000021280003F019FA6C
:1013A000002805D09BA1FFF797FA0320C043D6E79A
:1013B0000020D4E770B58A4B9D4404000126F60254
:1013C0006D4632003A21280003F05DF900280AD06A
:1013D0007EA1FFF781FA0020C0430123DB029D4478
:1013E00070BC08BC184729E144B6012A0CF0002A59
:1013F000506F776572206F6666206E6F742073750C
:1014000070706F7274656400416C726561647920FC
:101410006F70656E656420696E20646966666572CA
:10142000656E74206D6F646500000000416C72652C
:10143000616479206F70656E65642C2069676E6FDA
:1014400072696E67206F70656E20696E2073616DC2
:1014500065206D6F646500004F70656E2066616980
:101460006C656400436C6F7365206661696C6564CC
:101470000000000043616E6E6F7420636C6F7365D3
:10148000207768656E206E6F742070726576696F64
:1014900075736C79206F70656E6564005365742098
:1014A0007365637572697479206D6F646520666118
:1014B000696C65642E0000004E6F20736563757261
:1014C000697479206D6F64652072656365697665FE
:1014D00064206265666F72652070617274697469F8
:1014E0006F6E207461626C65000000005061727460
:1014F0006974696F6E207461626C65206C656E67DB
:10150000746820657863656564656400556E6B6E0C
:101510006F776E206572726F72206163636570749D
:10152000696E6720706172746974696F6E2074618E
:10153000626C65004E6F2073656375726974792003
:101540006D6F6465207265636569766564206265A8
:10155000666F7265206F70656E206D756C746900C2
:101560004E6F20706172746974696F6E207461626D
:101570006C65207265636569766564206265666F77
:101580007265206F70656E206D756C746900000067
:101590004F70656E206D756C7469206661696C654D
:1015A000642C20756E6B6E6F776E206572726F7231
:1015B000000000002C0E002A5061636B65742074DB
:1015C0006F6F206C61726765000000005265616496
:1015D00020756E7375636365737366756C000000C8
:1015E00000F8FFFF0C0800007265616420656E74EE
:1015F0006972652074726163656162696C6974798E
:101600002064617461206661696C6564000000009B
:101610000008000077726974652020656E74697235
:10162000652074726163656162696C6974792064B4
:10163000617461206661696C65640000320000219C
:10164000280003F064FA0004000C00280AD0FF49C7
:10165000FFF742F90120C0430123DB029D4470BC27
:1016600008BC18473F225201200008A90BF0C2FB1A
:101670000020F1E770B5801D817844780279090275
:101680000C43C1780904120611430C438179457952
:1016900009020D430121C9028D4207D90320ECA1A3
:1016A000FFF71AF970BC08BC03201847C01D2A00B8
:1016B0002100FFF740FE002809D0FF240934200054
:1016C000EFA1FFF709F9200070BC08BC1847F448E7
:1016D0002A2101704470210A8170210CC170210EF1
:1016E00001714571290A8171EE4907200863FEF7EF
:1016F0009FFFFEF74BFF70BC08BC00201847F0B5F9
:10170000E94B9D440027027AC179837A1202114382
:10171000427A12041B061A431143E44A6A44916058
:10172000C57A007B000205430024E148854209D9BF
:101730000320E0A1FFF7D0F80320EA4B9D44F0BC62
:1017400008BC184702A8FFF735FE0004000C00286B
:1017500004D0E5A1FFF7C0F80120EEE7A80AA9052B
:1017600000D0401C0190019800284CD9CF4A601C41
:101770006A440121D06089028002A84201D3A002FC
:10178000291A0E04360CC64A2C20791C0904090CAF
:10179000D055C648A3026844806818184B1C1B0427
:1017A0001B0C5054040A591C0904090CD454030C92
:1017B0004C1C2404240C5354010E631C1B041B0CEE
:1017C0001155591C0904090CD654340A4B1C1B042E
:1017D0001B0C545402A94118581C04049818240CDA
:1017E00032000BF007FBAF48A1190163FEF720FFA1
:1017F000FEF7CCFE0027AD486844C0680404240C02
:1018000001988442B2D3002097E710B5801D41783B
:10181000272902D18078282807D03620BAA1FFF7DF
:101820005BF810BC08BC0120184703F0A1F99D49E2
:1018300001228A609A4A272313705070022008639D
:10184000FEF7F6FEFEF7A2FE10BC08BC002018470B
:1018500008B5801D00210091002211006B4603F0A5
:1018600098F98F4A3221117000995170090A9170CC
:10187000D070AA2010718B4905200863FEF7D8FEAE
:10188000FEF784FE01B008BC00201847F0B583B015
:10189000821D8088072808D0A4490320FFF71CF880
:1018A00003B0F0BC08BC0020184790785578117937
:1018B00000020543D07800040906084305439079E7
:1018C00056790002064376483621017051794170FD
:1018D000917981700021C17001710624300A0127BD
:1018E000411C002927D9401C02906D48FF22001995
:1018F0000132290001AB03F05DF900280ED0072862
:1019000007D08BA1FEF7E8FF03B0F0BC08BC0020B5
:101910001847FF3401342404240C0CE0FF35013552
:10192000FF3401342404240C38007F1C02993F0446
:101930003F0C8842D9D35A49019848715949A01996
:101940000863FEF775FEFEF721FE03B0F0BC08BC8D
:1019500000201847F8B50100881D8988491F0A042E
:10196000120C81784478037909020C43C178090488
:101970001B0619430C43461D170A0125781C002835
:101980001AD97F1CFF220132210030006B4603F080
:1019900009F9002806D06BA1FEF79EFFF8BC08BC31
:1019A00000201847FF340134FF36013628006D1C33
:1019B0002D042D0CB842E5D3394834210170447010
:1019C000210A8170210CC170210E017100994171B1
:1019D000344906200863FEF72BFEFEF7D7FDF8BC5E
:1019E00008BC00201847F0B587B000265E4C206880
:1019F000C0680BF05FFE2B48406A002823D02949BD
:101A0000012088704C6A20684862002800D18862F2
:101A1000002020602348C069002815D000200690CF
:101A20000025A088002810DD4F480068C0680BF032
:101A300041FEA088471B802F00DD80276119891D8A
:101A400006983A0092E0E8E0A4E097E0E815002A62
:101A50005772697465207472616365205061636BAD
:101A6000657420746F6F206C617267652C6F76658A
:101A70007220323034382062797465732E00000091
:101A80005772697465207472616365205061636B7D
:101A9000657420756E7375636365737366756C002A
:101AA00044B6012A0CF0002AECF7FFFF0008000002
:101AB000FF7F00005265616420747261636520508D
:101AC00061636B657420746F6F206C617267652C45
:101AD0006F766572203078374646462062797465A5
:101AE000732E00001408000044554D50207472619C
:101AF00063656162696C69747920646174612066F0
:101B000061696C65640000006E6F7420612068611B
:101B10006E646C655F77726974655F70726F74650F
:101B2000637420636F6D6D616E6421002C0E002A5A
:101B30005265616420756E73756363657373667552
:101B40006C6C000052706D62206175746820646175
:101B500074612077726974652020756E7375636394
:101B600065737366756C0000D4EF002AFEF767FB9F
:101B70000690ED19A088A84200DD55E73449069883
:101B8000884203D033A0FEF772FD3EE0A088801E9D
:101B9000A08002E0A088801EA080A779362F26DDD5
:101BA000A01D0290A08803902F48049001A80590E2
:101BB0000025002001902D48E9004158002905D05A
:101BC00002A80BF078FD012800D10126019A002A15
:101BD0000AD025492648FEF787FC2648019901636B
:101BE000FEF726FDFEF7D2FC6D1C042DE1DB002E76
:101BF0000BD1781E352805D81E494978002913D005
:101C0000012F11D02000FEF7ADFE1A48016A2160B5
:101C10000462406A002800D0F1E61649002088706E
:101C200007B0F0BC08BC1847810013484158200099
:101C30000BF041FDE9E7114CFEF730FC2068C0686D
:101C40000BF038FDFEF72AFCFFF7CDFEF4E70000AD
:101C5000470F00004552523A2043524320696E76A6
:101C6000616C69640000000044BE012A4038012A0A
:101C700044B6012A0CF0002A40F0002AD4EF002AD2
:101C800070B50500CB48416801290CD0816B012952
:101C900009D0002134224A431418E269002A05D0F1
:101CA000491C0229F6DB70BC08BC1847200000F074
:101CB000A0FA0028F7D02035BF4800F01DFD687A53
:101CC0000028F0D0200000F094FA0028F4D170BC75
:101CD00008BC184710B501290FD003290AD1B74C09
:101CE0002178012901D1FFF7CBFFE068002801D05E
:101CF0000BF0E0FC10BC08BC18470021C0690C28A0
:101D000003D0FF38E13803D101E0402100E0AC49C5
:101D1000AC4A0B0A50680171437190690171090A5C
:101D2000417110BC08BC184700218161A349496872
:101D3000002900D008477047A049896808479E4994
:101D4000C860704710B50400A068FFF799FF9B4971
:101D5000200089680BF0AFFC10BC08BC1847FFB529
:101D600083B00C9D14001E00002794480570924A11
:101D7000002901D09068C16193499248416093491C
:101D80008161934893494860934B94484360944BD6
:101D9000894A1360C160012001F028FA864800F0EA
:101DA00083FC864803998160002C00D04460002E9B
:101DB00000D0C660804E01AAF06802A900F08CFE37
:101DC000884886607F494A6892780274864A4261F0
:101DD00000238361012220242254844A4262002D80
:101DE0003CD000208249342402006243714C141913
:101DF000A660744A92699278227402035218626152
:101E00007C4AA261202213557B4A6262E361401C36
:101E10000006000E0228E6D3002F2FD0664800F0FF
:101E200084FB764801210172F068002201F08FF8EE
:101E30000122F068110001F08AF8F0680022022106
:101E400001F085F8F0680122022101F080F85A487B
:101E5000012100F045F9012D0DD00FE0684CA6607E
:101E60008869807820746361A361202003556548E8
:101E70006062E361D0E7A068FFF702FF07B0F0BC43
:101E800008BC4D48184710B54B4800F03EFC10BC4C
:101E900008BC184770B50500524C6068012805D190
:101EA000454800F029FC60680128F9D0A069411C70
:101EB000A16161690D547E2D02D1A069012804D869
:101EC000A06901218903884202D3200000F091F922
:101ED00070BC08BC184770B505000E00414C606826
:101EE000012805D1344800F007FC60680128F9D0CA
:101EF000002D07D1002E05D06069320029000AF0BC
:101F000079FF00E06561A661200000F072F9606869
:101F1000012805D1284800F0EFFB60680128F9D0BE
:101F20003148606170BC08BC18472E4840680128E1
:101F300005D02148806B012801D000207047012086
:101F40007047F8B506000F002D4C25006868012881
:101F500005D1194800F0D0FB68680128F9D0002E9F
:101F600003D1002F01D0666100E06661A761200007
:101F700000F03FF9F8BC08BC002018470021C161FF
:101F80007047174A002800D01081002900D05181E5
:101F90007047002A08D1124A002801D01389038013
:101FA000002901D05089088070470021C1618068F4
:101FB00066E600006C07022AACF1002A18F1002A3C
:101FC000000200005CF1002A4CF1002A53F1002AC3
:101FD00043F1002A84F1002A3AF1002A9CF1002AF8
:101FE00028F1002A0407022A04C7012A291D002A11
:101FF000D407022A00100000451D002ACCF1002A57
:102000003807022A391D002A406803E00068491E8B
:102010000904090C002801D00029F7D17047406855
:10202000002806D0426852798A4202D0006800280F
:10203000F8D17047C06AC0687047C06AC068C0689D
:10204000002806D0426892788A4203D000680028AF
:10205000F8D1002070478068002808D003898B429F
:1020600002D1837A934203D000680028F6D1002081
:1020700070470269002A00D01047704701620421AE
:10208000F7E7F0B5060083B0F06843689C788C42AF
:1020900020D1D97891421DD1C468002C15D00025DB
:1020A00061688878C2094B790F791B023B436F4600
:1020B00028C7C9788B070107B0689B0FC068090F54
:1020C00000F02EFD2468002CEAD103B0F0BC08BC5F
:1020D0000020184703B0F0BC08BC0020C0431847DC
:1020E000F8B504000E000025200020300090407A52
:1020F000002807D0002E05D0B04203D0681EF8BCDF
:1021000008BC1847B0425FD0002E25D03100200017
:10211000FFF785FF0700002F0DD0F8680022406808
:1021200081783800FFF7ADFF002809DAF8BC08BC59
:102130000020C0431847F8BC08BC0020C043184723
:1021400000984672E762002060627868007A410079
:102150002000FFF793FF21E0009900204872E06221
:1021600000212000FFF78AFF0126E06800223100ED
:1021700000F09CFEE0680022310000F042FDE068C3
:102180000122310000F092FEE0680122310000F0EF
:1021900038FD761C3606360E032EE6D303212000CA
:1021A000FFF767FFE06800F08FFF002805D00128E7
:1021B00005D0022804D1FF4D02E0402500E00825AB
:1021C000280000F08AFF10E0E06800F07DFF0028A2
:1021D00005D0012805D0022804D1F64D02E04025A3
:1021E00000E00825280000F078FFF8BC08BC0020BB
:1021F000184710B5F049016000214160C161816854
:10220000002908D0CA68C2602031497A002908D163
:10221000017C090705D00321416010BC08BC081FE0
:10222000184700F0FAFD10BC08BC184770B506004E
:102230001D00E24C30003430002900D134304168B8
:10224000012904D042618561FFF7D3FF0400201EFD
:1022500000DB280070BC08BC184702000B003032BD
:102260000121E3E7F8B507000E00B01C0025D34CB0
:102270004178012904D0022905D003291BD10EE0A1
:102280003D682C7817E001783800FFF7BDFE002884
:1022900011D04568E878A97804020C430BE0027875
:1022A00070793379010219433800FFF7D4FE002812
:1022B00001D045682C78002D0FD0F079B17900025B
:1022C0000843A04200DA040023002A00012138005C
:1022D000FFF7ACFFF8BC08BC18472000F8BC08BCEE
:1022E000184710B54A780A2A4AD213007B441B7952
:1022F000DB189F44044D454D4512264D2B3ACA79B3
:102300008B7911021943022942D30021018602214F
:10231000FFF7A3FF10BC08BC1847CA7889781302DE
:102320000B43010020310A00497A002930D11906F7
:10233000090E1172C06800F08EFB10BC08BC0020B2
:102340001847FFF78FFF10BC08BC1847CA798B7974
:10235000110219431CD0010020314A7A0A7401216C
:10236000FFF77BFF10BC08BC1847CA788B781102B6
:1023700019430906090EFFF7B3FE10BC08BC184745
:102380004269002A04D00BF097F910BC08BC18472A
:1023900010BC08BC0020C043184770B505000C00F5
:1023A00060792279010211432800FFF743FE61782A
:1023B00003294AD004DC002911D0012904D144E0CA
:1023C0000A291DD00B292CD000283ED00269002AF2
:1023D0003BD021000BF070F970BC08BC18470028F6
:1023E00033D0E079A1790002084302282DD30020E0
:1023F000288602212800FFF730FF70BC08BC184770
:10240000002822D0E179A279090211431DD0017D73
:102410003020415501212800FFF71FFF70BC08BC88
:102420001847E86A002810D0E178A27823790902D9
:1024300011430A066179120E090219430906090EB1
:10244000FFF71FFE70BC08BC184770BC08BC00201A
:10245000C043184710B54B689B781C07240FDB0955
:102460000A61002A05D0C0681A00210000F000FBB4
:1024700004E0C0681A00210000F012FB10BC08BC88
:102480000020184770B505000C0060792279010220
:1024900011432800FFF7D1FD0023DB43002811D0B2
:1024A0006178002912D0012921D003292CD00C29D0
:1024B0002FD0C268002A2CD021000BF0FDF870BC90
:1024C00008BC184770BC180008BC1847E179A2790D
:1024D0000902114302291CD30069C007C00F2886D6
:1024E00002212800FFF7B9FE70BC08BC1847E1784C
:1024F000A278090211430CD1010000222800FFF745
:10250000A9FF70BC08BC1847E178A2780902114302
:1025100003D070BC180008BC184701000122280035
:10252000FFF798FF70BC08BC184770B50400E0685E
:1025300002F050FB0600A0690025B04222D0E56100
:10254000002E16D0656264212000FFF797FDE06839
:1025500002F050FB002804D019492000FFF78EFD3F
:102560000BE000212000FFF789FDE06802F047FB47
:1025700003E000212000FFF781FDA661002120007B
:10258000FFF777FDE06800F09FFD002824D00128C8
:1025900024D0022824D00020E169814205D0656260
:1025A000E06101212000FFF764FDE06800F098FD84
:1025B000050007E00002000051555242FFFFFFFFF7
:1025C000DC050000606AA8421FD0002D0AD000215F
:1025D0002000FFF753FD13E00C20DDE70120DBE7CF
:1025E0005F48D9E7E06A002806D04068007A4100D9
:1025F0002000FFF743FD03E000212000FFF73EFD30
:10260000656205212000FFF734FD70BC08BC184747
:1026100010B504002000FFF788FF00212000FFF71D
:102620005FFD002128200155E06800F014FA032026
:10263000E066A06310BC08BC184710B50400494B05
:102640000878C006C00E04D0012807D002280ED199
:1026500009E02000FFF745FE030008E02000FFF737
:102660009CFE030003E02000FFF70CFF0300002B9B
:1026700009DD22000423303200212000FFF7D6FDBF
:1026800010BC08BC1847002B07D00022E0681100DE
:1026900000F0EEF910BC08BC184700212000FFF73D
:1026A000DCFD10BC08BC184770B504000025A5610E
:1026B000E561200020300572E562457200212000AE
:1026C000FFF7DCFCE463802144200155A56503206D
:1026D000A063246778210D558C210D51E066224AB4
:1026E000E068210000F084F8E0680122002100F099
:1026F0008FFC70BC08BC184710B5002802D0C06819
:1027000000F07FF910BC08BC184770B50500002424
:10271000164E03E02800FFF7EFFF641CA86B0128AA
:1027200002D130688442F5D300212800FFF7D8FC9D
:10273000E86800F045FC0020A861E86120352872B7
:1027400070BC08BC184710B504002000FFF7D4FF88
:102750002034607A002800D0012010BC08BC184743
:10276000E0010000FFFFFFFF7CF2002A78F2002A60
:10277000FB4840787047F8B5FF21FA4881310AF0EC
:1027800005FCC321F84889010AF000FC002501225C
:102790000021F44BE801C718A801F34B2818800169
:1027A000C61888010818400133188801381883605A
:1027B000002044011A51401C4028FADB491C022920
:1027C000EFDB6D1C032DE3DBE849E64801600164A3
:1027D0000168E74A11430160FF21813102F059FA93
:1027E000C321E148890102F054FAF8BC08BC18473B
:1027F000F8B506000027DA4882600C207043DD4AF5
:1028000080188160300002F006FA032002F09EFC7E
:10281000300002F00DFAD84DB4002859FF30813055
:10282000816A89088900891C81623000FFF7A3FF53
:102830002859CC49FF304130816128590021FF30AF
:10284000413081602859FF308130836A0822134368
:1028500083622859FF308130C162285980308261FB
:10286000FFF786FF012806D12859FF304130016863
:102870000122114301603800F8BC08BC1847F8B5C4
:102880000700BD4DBC0028590121FF308130C162D5
:102890002959FF318131C86AC007C00F0028FAD119
:1028A000B6480126760300902859FF304130016870
:1028B000314301600098082102F0E5F9A949A848D0
:1028C000283106C9143006C02859FF30413000684D
:1028D00030400028E8D02859FF3041300168B1432A
:1028E00001600C204743A348381880689C498968D8
:1028F0004A68A3490AF0E0FEF8BC08BC1847F0B5E6
:1029000085B081009C484058FF308130C16B0091F8
:102910000099C16300200190002601989149C001EF
:10292000401804900198810140188F498001401897
:102930000390019831010918012088400099014253
:102940002FD00498B1014018402102F09CF9B10148
:10295000039871184901441802940025002720218A
:10296000200002F090F96068000CC719002D02D118
:10297000606805062D0E2068012801D0246800E05B
:102980000024002CEBD10298C469A069C11BE1614D
:10299000606902F078F9002D14D0802D1BD003203F
:1029A0006060761C3606360E012EC2D90198401C96
:1029B0000006000E019001980328ADD305B0F0BCCD
:1029C00008BC184702206060616A0029E9D0200035
:1029D0000AF071FEE5E701206060E2E70C21484360
:1029E0006449401880685E49896889680847F5E746
:1029F0000C2148435F494018806859498968096833
:102A0000084770B505005C48A90041580800FF312F
:102A100041314C680A00FF308130C66A546060065C
:102A200002D52800FFF7E4FFE00502D52800FFF7F4
:102A3000DEFF600702D52800FFF7D0FFE00702D0D5
:102A40002800FFF75CFFF00702D02800FFF717FF10
:102A500070BC08BC184701234A061B06D218464B17
:102A600080001858FF30413042613D480170704786
:102A700010B403000020002903D0002A03D0414AEB
:102A800002E0414A00E001229C003B4B89001B59B7
:102A9000FF31C1315C58944314435C5010BC704703
:102AA00030B4040000200023002904D0002A04D000
:102AB000364A2E4B03E0344A01E041224023A50070
:102AC0002D4C89006459FF31C1316558134095433D
:102AD0001D43655030BC704710B40023204CA478CF
:102AE000002C01D02A4805E083002348C0588030DC
:102AF000036880680B60106010BC704700B582B03E
:102B00000021019100916A4601A9FFF7E5FF204AE3
:102B100000990120914200D0002002B008BC184763
:102B2000F8B505000C0016001F0000200090002CD6
:102B300009D0032C03D2022E01D2022D07D3F8BCF8
:102B400008BC03201847F8BC08BC00201847012E19
:102B500020D02800FFF7D2FF00282BD000202AE049
:102B600088F2002A0028022A8029022A0000400058
:102B700000800000745E022A70F3002A2828022ACE
:102B80009CF2002A00000100010001000000410049
:102B9000EFCDAB002800FFF7B1FF002801D00020E7
:102BA00001E001208005B90440180121C905411840
:102BB000F94804E04020B90041188031F748069AEE
:102BC000E3011704F64A9B18B2019F50079E0127A4
:102BD0007F07012E11D09E583E439E50F14AAB0014
:102BE000D358A200FF32C1329C58014084430C43A9
:102BF0009C500098F8BC08BC18479E58BE439E5095
:102C0000ECE770B40024032903D2022A01D202287F
:102C100001D3032413E0E24ECD010023AD19960148
:102C2000AB5100290BD0012A0CD080228300DD4853
:102C3000C3588800FF30C130195891431950200003
:102C400070BC7047D84AF1E7D848C0687047F0B503
:102C500083B08C460193D64D8401D7490019800179
:102C6000401861468C010919D24F4901461802905B
:102C70006D1C01208003834200D218006901741882
:102C800000212160A160E16021616161A161E161D8
:102C9000010480316160002D03DD691E4901711856
:102CA0000C60A260A168090B0903E160E168C91921
:102CB000E160E168C91921612169C919616161692E
:102CC000C919A1611B1A1218002B01D03F2DCFDBAF
:102CD000089800282CD06046012829D1FFF7B4FFBE
:102CE000010001980AF02EFB002921D1019800284B
:102CF0001ED0681C1CD06D1C02994120400109188F
:102D000068010C1800202060A060E0602061606114
:102D1000A061E06180206060002D03DD6D1E680110
:102D200008180460A548A060E06020616061A061AF
:102D30000120206060680121C9030843606003B07E
:102D4000F0BC08BC1847FFB5050083B00D980C0017
:102D5000160006998C46924AE1018918B2018F1833
:102D600031010A190121914002918E4BAD00002CD6
:102D70000CD15959FF318131C96AC907C90F0029DE
:102D800004D007B0F0BC08BC052018470C990122FC
:102D90001205914204D907B0F0BC08BC03201847C3
:102DA00080494959FF318131896B029A11400029CC
:102DB00004D007B0F0BC08BC0720184700900C9B5B
:102DC000310020006246FFF742FFA0012018810178
:102DD00079480818B101711849014618BE600020F1
:102DE000F8600C99069801F054FF00246001301837
:102DF000202101F04EFF641C412CF7D34021380004
:102E000001F047FF674902984959FF318131086352
:102E100007B0F0BC08BC00201847F0B583B0040030
:102E2000E768207C05072D0FC60960698446A26902
:102E30002020035D032D04D303B0F0BC08BC0320A5
:102E400018475849B8000958A800FF30C130095840
:102E50000120C005012E00D0802001420FD068461D
:102E60000CC03200290038006346FFF76CFF0028D1
:102E70000AD00321616003B0F0BC08BC184703B05E
:102E8000F0BC08BC07201847012161600021E16106
:102E9000A901494A691889018918B201B218520179
:102EA0008918CC6103B0F0BC08BC1847F7B50F0017
:102EB00082B0049901240901C9198C40860039485F
:102EC0008059FF308130806B2040019001980028AC
:102ED00038D03349F801411804988001081840217E
:102EE00001F0D1FE0025B80133493818800141189E
:102EF00004988201801840010F18680138182021B9
:102F000001F0C1FE6D1C412DF7D3F869019900292C
:102F10000FD0244B9959FF3181314C639959FF31BE
:102F200081314A6B2240002AFBD1896B2140002964
:102F3000F0D1002806D003214160416A002901D068
:102F40000AF0B9FB05B0F0BC08BC0020184710B46B
:102F50001201521801219140124C8300E058FF30B9
:102F60008130806B084000280ED0E058FF3081305F
:102F70004163E058FF308130426B0A40002AFBD1A8
:102F8000806B08400028F0D1E058FF308130C16BE1
:102F9000C16310BC002070470000FFFFFFFF00006E
:102FA0000028022A70F3002A0000800088F2002A1C
:102FB000FFFFFFFF001000008029022A98F2002A7C
:102FC00070B5050000260024220031002800FFF71C
:102FD0006DFF641C2406240E022CF5D3761C3606E5
:102FE000360E032EEFD300260024220031002800E5
:102FF000FFF707FE641C2406240E022CF5D3761C72
:103000003606360E032EEFD370BC08BC00201847DE
:10301000F0B40025022901D2022802D3F0BC03201B
:103020007047814C635C002B02D0F0BC06207047D7
:103030007E4B002A00D07E4B7E4E7F4A80000029C6
:103040000AD017588037BE6010588030C360012006
:1030500060542800F0BC7047175880373E60105805
:1030600080304360F3E7022901D2022801D3032014
:1030700070478200704B0020002905D09A5880329A
:10308000D060694A505470479A5880325060F8E7CF
:103090000022022901D2022801D303207047664B87
:1030A0008000002902D0012906D00AE0185880309B
:1030B00040680202120A04E018588030C068020218
:1030C000120A5C48801A70475B4980000858FF303C
:1030D000813040680001800F70475849C8607047D0
:1030E000554980000858FF308130406880210840F1
:1030F000002800D001200006000E70474E498000D5
:103100000858FF30813040680005800F704781000B
:1031100049484058FF3041300168012211430160A5
:103120007047F8B500250024454E09048919870029
:103130004148C259FF324132116309E03E49C95941
:10314000FF3141310D6B2E000640012001F0FEFFE2
:1031500001208007864205D12100FF22641CF53240
:103160009142EBD32804F8BC08BC000E1847FFB509
:1031700017001E0081B00024314DFF2E09D001A898
:1031800003C8FFF7CEFF0006000EB0433E400643E3
:1031900000E03E000298032100048019490740180E
:1031A00001998E0024498A59FF32413210632F0061
:1031B00008E021488059FF304130056B3D40012037
:1031C00001F0C4FFBD4205D12000FF21641CF53190
:1031D0008842EED305B0F0BC08BC184710B501F02A
:1031E0005FFE10BC08BC0006000E1847134948706B
:1031F000704770B506000C00150000213000FFF785
:1032000032FF01213000FFF72EFF0B4AB0001158AA
:1032100080310C6010588030856070BC08BC184745
:1032200006498870704700008BF2002A000000C039
:10323000000000C1FFFFFF0070F3002A88F2002A9F
:103240000000004070B56424FF4DA869C00303D599
:1032500070BC08BC01201847012002F05FFE641E0C
:10326000F3D270BC08BC00201847F7480021016069
:1032700001610168F54A91430122D2038918016076
:1032800001683F22120211430160F14941608168E7
:10329000C90CC904891C8160C168C90CC904093101
:1032A000C160EC494161EC4901610168EB4A11439D
:1032B0000160EB48026AFF2101310A430262E948DA
:1032C00002680A430260BDE770B5E748816A0024DE
:1032D000C9070125002905D0016A0462816AA94352
:1032E000816204E0416A4462816A294381624B2021
:1032F000000202F0FBFDDD48816AC90706D0016AC1
:103300000462816A49084900816204E0416A4462BA
:10331000816A29438162D648816AC90708D0016A57
:10332000C909C9010162816A49084900816206E050
:10333000416AC909C9014162816A29438162CD4854
:10334000C16889088900491CC1608168C90706D025
:1033500001680460816849084900816004E04168AF
:103360004460816829438160C348816AC9070AD0E3
:10337000016AC909C9010162816A4908490081627B
:1033800070BC08BC1847416AC909C9014162816A19
:103390002943816270BC08BC184770B5B248816A85
:1033A0002B25C9070124002905D0016A0562816A1D
:1033B000A143816204E0416A4562816A21438162DE
:1033C0007D20400202F092FDA848816AC90706D01C
:1033D000016A0562816A49084900816204E0416A24
:1033E0004562816A21438162A148816AC90709D087
:1033F000016AC909C90113310162816A490849009A
:10340000816207E0416AC909C90113314162816AD9
:103410002143816297488168CA071321002A06D098
:1034200002680160816849084900816004E04268DF
:1034300041608168214381608F48816AC9070BD050
:10344000016AC909C9012B310162816A4908490031
:10345000816270BC08BC1847416AC909C9012B3197
:103460004162816A2143816270BC08BC184783486D
:10347000834A106050609060D0601061506190612C
:10348000D06180498861106250620860486088603D
:10349000C86008614861C8610862486288627A4809
:1034A00042687A490A40521D426082680A40121DF1
:1034B0008260C2680A40121DC26002690A40121D81
:1034C000026142690A40521D426182690A40121D2E
:1034D0008261C2690A40D21DC261026A0A40121D9D
:1034E0000262426A0A40121D4262826A0A40921DCA
:1034F0008262C26A0A40521DC26270475F486449D4
:10350000086048608860C8606249086048608860F8
:10351000C860614842685D490A40921D4260826805
:103520000A40921D8260C2680A40D21DC2600269D0
:103530000A40D21D02615948016AC90AC9023431E0
:103540000162704756480F2101605649564A116082
:1035500051609160554A116051609160D16042683C
:103560004A490A40121D426082680A40121D826068
:10357000C2680A40121DC26002690A40121D02613F
:10358000704710B54A48016A494A40200143116218
:1035900048490968474A0143116047490968464A52
:1035A0000143116044498968014391604249C968F7
:1035B0000143D16040490969014311613F49096AEA
:1035C0003E4A014311623D49496A014351623C4907
:1035D00009683B4A014311603A49096A394A014383
:1035E000116239490968384A01431160374A116A42
:1035F00001431162516A0143516235490B6803432B
:103600000B604B6803434B60324B1B68314C0343E8
:103610002360304B9B680343A3602E4BDB6803435E
:10362000E3602C4B1B69034323612A4B1B6A034352
:103630002362284B5B6A03436362264B9B6A034306
:10364000A362244BDB6A47E04031900000C00F00CA
:103650000E1003000000C000001000000000100069
:1036600080349000C0349000402790008024900067
:10367000C02D900040269000C022900000820000E3
:10368000003630010038300180383001F0FF000092
:103690000036400100384001803840014000F00011
:1036A00080385001F481000000365001003850018C
:1036B00000249000C0209000002190008020900005
:1036C000002E9000C023900000259000C0219000A3
:1036D00040259000402190000343E362C94B1B6BDF
:1036E00003432363C74B5B6B03436363C54B9B6B14
:1036F0000343A363C44B1C6804431C60C34B1C6896
:1037000004431C605C6804435C60C14B1C6A044356
:103710001C621C6804431C60BE4B1C6804431C6094
:103720001C6A04431C62BC4B1C6804431C60BB4BFA
:10373000DC6A0443DC62BA4B1C6804431C60946A74
:1037400004439462B74A146A04431462B64A146983
:1037500004431461546904435461946904439461BB
:103760000A6A02430A624A6A02434A62AF490A6825
:1037700002430A60AE4AD46A50210C43D4621A6AEA
:103780000A431A62AB490A6A02430A62FFF76FFEF4
:10379000FFF7B4FEFFF7D6FEA749F020886110BC02
:1037A00008BC1847F8B54B20000202F09FFBA34964
:1037B00040208861A24802F0B1FBA248016A0125BD
:1037C00029430162016A0226B14301629E489F4F6C
:1037D00038619F4802F08AFB9E480168102421430B
:1037E000016001680422114301609B480068C00722
:1037F00004D0FFF769FD984900200860FFF735FD08
:1038000000287ED03868204338607868204378608C
:10381000FFF7C3FD9149086820430860904802689B
:1038200022430260826822438260C2682243C260EF
:103830000269224302618B4A12688A4B22431A6052
:10384000026A224302626F48026822430260826871
:1038500022438260C2682243C2600269224302613D
:10386000026A22430262426A22434262826A22431D
:103870008262C26A2243C262026B22430263426BCB
:1038800022434263826B224382637748006A764A0E
:10389000204310627548006A744A204310625A48F7
:1038A0000068594A204310605B4800685A4A204328
:1038B000106057480068564A204310605548006819
:1038C000544A204310605248006A514A2043106213
:1038D0005048006A4F4A20431062534804614461D3
:1038E0008461634A502010605060614884604B4896
:1038F000C4624B4A1068204310604A480462446224
:1039000000E074E05B48806A5A4B304398625A4842
:1039100000685A4B1843584B18608C62CC62584868
:1039200004605848006A40210843564908625648D6
:10393000564908625648016A21430162416A21439F
:1039400041625448416B29434163534841682943CC
:1039500041604C48006A0121090308434949086253
:103960004848006A4D490843464908624C494D4859
:1039700081604D4941614D4B0021D9624C498161C3
:103980004C4901624C4901634C484D4908604D481F
:103990004D4948604D495120C8604D48016A214356
:1039A0000162416A214341624A48016A214301623E
:1039B0001E480168214301604748016A21430162B2
:1039C000416A21434162816A214381621848C16A88
:1039D0002143C162106A20431062404800780028E9
:1039E00001D0FFF7CEFDF8BC08BC01201847F8BC99
:1039F00008BC00201847D5E610B5FFF765FC10BCE1
:103A000008BC184740219000002C900040209000F6
:103A100080269000C02690008022900040279000D1
:103A200080279000802B9000402690000029900075
:103A30008024900080259000C003301800002000F2
:103A400088130000802E900011080000C02790000D
:103A500078690000C02E90004031900080209000D6
:103A600000219000C0209000C0239000002490000E
:103A700040299000C02290004030900000100000CB
:103A8000002E9000C02F900010010000802D9000AB
:103A90000027900080000028C000002800080000D7
:103AA0004B800091000000040080000080010004B1
:103AB0000100EC1700042035C70300000500FF805B
:103AC00080000004FF1400004002000480219000E8
:103AD00040259000C02A9000C0219000A4F2002A46
:103AE00010B5002801D10F2903D310BC08BC002059
:103AF00018474C4801604C48425C4C48415C4C487B
:103B0000006802F098FA10BC08BC0120184770B594
:103B100000280DD1464C00252068290002F010FA3B
:103B2000206802F039FA3F4801682800FFF7D8FF03
:103B300070BC08BC1847012070470120704707B5CA
:103B400082B0002803D0002005B008BC18473948CF
:103B50000168374803290BD00068012304AA03A990
:103B600002F0A0FB0128EFD005B008BC00201847E8
:103B70006A46918901910068012304AA01A902F013
:103B800059FBEFE707B582B0002803D0002005B04D
:103B900008BC184727480168254803290AD000684F
:103BA000012303A902F09AFB0128F0D005B008BC5C
:103BB000002018476B46998901910068012301A9EB
:103BC00002F054FBF0E770B51400002801D1012980
:103BD00003D970BC08BC00201847164800290ED035
:103BE00004210160124D0168286802F057FA286824
:103BF000210002F063FA70BC08BC012018470321C1
:103C00000160EFE710B5002803D010BC08BC00200D
:103C100018470748006802F045FC10BC08BC0120AA
:103C200018470000405A022AB3EA002AA4EA002AF0
:103C300098EA002AA8F2002A10B5002402210020E8
:103C4000FFF74EFF002800D101240020FFF75FFF9F
:103C5000200010BC08BC184710B50124002802D071
:103C60000024FCF78CFB200010BC08BC184730B5C2
:103C700083B005001A240020029001900221280040
:103C800002AAFFF77FFF012833D16946087A0009AD
:103C900000010190F0282CD1E821280001AAFFF7AB
:103CA00071FF012825D168460079012810D002282B
:103CB00010D0032810D0062810D0082810D00928CA
:103CC00010D00A2810D00B2810D00C2810D010E0EB
:103CD0000E240EE010240CE00F240AE0122408E069
:103CE000132406E0172404E0182402E0162400E060
:103CF0001924200003B030BC08BC184730B583B08D
:103D0000040000250020029001900A220121FFF703
:103D10005AFF002800D101250221002002AAFFF746
:103D200031FF002800D16D1C6846007A0007000FA3
:103D3000092802D90920207000E02070E821002025
:103D400001AAFFF71FFF002800D16D1C684600790B
:103D500006210A2802D00C2813D10EE02078012871
:103D600005D0022806D003280BD3217009E00320D8
:103D7000207006E00520207003E02078002800D0A5
:103D80002170280003B030BC08BC184738B50400C7
:103D9000002500200090E8216A46FFF7F3FE002886
:103DA00000D10125684600780A2809D00C280AD0DD
:103DB00003202070002D09D038BC08BC0120184712
:103DC00002202070F6E701202070F3E738BC08BC21
:103DD00000201847FD49087000207047FB4900206B
:103DE00008707047F8B50500002400200090F74ED9
:103DF0003078322804D02870F8BC08BC002018475E
:103E0000022100206A46FFF7BDFE002800D12124D0
:103E1000FFF7E4FF002800D021243078287020002C
:103E2000F8BC08BC184738B5002400200090FF25D6
:103E3000E63570222900FFF782FE002800D1012418
:103E4000290000206A46FFF79DFE002800D1641C6F
:103E50006846007880070FD552224F210020FFF7D7
:103E60006EFE002800D1641C002155220800FFF7D7
:103E700066FE002800D1641C002C03D038BC08BCAE
:103E80000120184738BC08BC0020184738B500246A
:103E900000200090002201211000FFF7B3FEE8216E
:103EA00000206A46FFF76EFE694608780A280AD0A5
:103EB0000C280AD0C64D852229000020FFF73FFEBE
:103EC000002804D004E0C34DF5E7C34DF3E7012417
:103ED000B02229000020FFF732FE002800D1641C28
:103EE000C02229000020FFF72AFE002800D1641C10
:103EF000902229000020FFF722FE002800D1641C38
:103F0000002C0AD15A224F210020FFF718FE00286A
:103F100000D10124B148B249C8600122110000203B
:103F2000FFF770FE002C03D038BC08BC01201847F6
:103F300038BC08BC0020184708B5002000900121BB
:103F40006A46FFF71FFE00280ED068460078C007BB
:103F500006D0A449A4220020FFF7F1FD002807D0D5
:103F600001B008BC0020184701B008BC0120184768
:103F700001B008BC01201847F0B589B009200890AD
:103F800032200790002506950195FFF755FE0400A5
:103F900000210A220800FFF716FE00190406240E6D
:103FA0000321002005AAFFF7EDFD6946087D5A2888
:103FB00004D152224F210020FFF7C1FD0A22012126
:103FC0000020FFF700FE041908A8FFF797FE041968
:103FD000FFF729FF041900210A220800FFF7F3FD6B
:103FE00000190406240E0321002005AAFFF7CAFDCC
:103FF0006846007D5A2804D152224F210020FFF745
:104000009EFD0A2201210020FFF7DDFD0419FFF7C4
:104010003DFF00190406240E734841693B22090143
:10402000090C520191420FD34069D11C0001000CD0
:10403000884209D8FF2100227231012002F0D1FA12
:1040400000190406240E07E001210022080002F0F6
:10405000C8FA00190406240E07A8FFF7C3FE0419C6
:1040600006A8FFF793FE04196846007E02F09EFA48
:104070000419FFF761FF0419FFF75EFF0019070637
:104080003F0E1821002001AAFFF77CFD002807D071
:1040900069460879C009C0010190002805D08DE06B
:1040A00009B0F0BC08BC012018474F21002004AA29
:1040B000FFF768FD00281DD06846027C06200243F9
:1040C00004924F210020FFF73AFD002817D04749FE
:1040D000002003AAFFF756FD002815D06846007B94
:1040E00081064C0F4607760F0020FFF7C0FD192808
:1040F0000FD025E009B0F0BC08BC0120184709B07A
:10410000F0BC08BC0120184709B0F0BC08BC012075
:10411000184700956846007B4006C50F34490020CB
:104120006A46FFF72FFD002864D0684600784208F1
:1041300052002A432E490020FFF701FD00285ED0DF
:104140004F21002004AAFFF71DFD00285CD068461F
:10415000027CFB20024004924F210020FFF7EFFC7D
:10416000002856D0FF250B352900002002AAFFF7B2
:1041700009FD002852D06846007A7101C006C00EC1
:1041800008430206120E29000020FFF7D8FC002881
:1041900049D09C21002002AAFFF7F4FC002847D058
:1041A0006846007A6101C006C00E08430206120E7E
:1041B0009C210020FFF7C3FC00283ED0002F41D0F7
:1041C00009B0F0BC08BC0120184713E04C5A022A81
:1041D00053010000760100006201000009080000A0
:1041E00000289000090200004020800055030000D4
:1041F000B502000009B0F0BC08BC0120184709B0A6
:10420000F0BC08BC0120184709B0F0BC08BC012074
:10421000184709B0F0BC08BC0120184709B0F0BC31
:1042200008BC0120184709B0F0BC08BC01201847A1
:1042300009B0F0BC08BC0120184709B0F0BC08BCAC
:104240000120184709B0F0BC08BC0020184738B559
:10425000002500950024652100206A46FFF792FCA6
:1042600000282CD0684602781020024365210020E7
:10427000FFF765FC002826D00095642100206A46DF
:10428000FFF780FC002822D0684600784206520ED4
:10429000803264210020FFF752FC00281BD00095DB
:1042A0004025652100206A46FFF76CFC002816D0E7
:1042B000684600782840800915D0012416E038BCF3
:1042C00008BC0120184738BC08BC0120184738BC7E
:1042D00008BC0120184738BC08BC0120184738BC6E
:1042E00008BC012018476420FCF749F8002CD8D0FE
:1042F00038BC08BC0020184738B5002500950024BC
:10430000642100206A46FFF73DFC002820D0684663
:1043100000784206520E64210020FFF710FC0028AE
:104320001AD000954025652100206A46FFF72AFC37
:10433000002815D0684600782840800914D06420F1
:10434000FCF71DF8002CEED038BC08BC0020184744
:1043500038BC08BC0120184738BC08BC01201847ED
:1043600038BC08BC012018470124EBE7F8B504006D
:10437000002500200090012C05D0002C03D0F8BCB3
:1043800008BC09201847FF260B36310000206A467A
:10439000FFF7F8FB002812D0012C14D069460878EA
:1043A000FB21084000906846027831000020FFF7AA
:1043B000C6FB00280DD02800F8BC08BC1847F8BC84
:1043C00008BC01201847694608780421084300907A
:1043D000E9E7F8BC08BC0120184738B504000025FF
:1043E0000020009007216A46FFF7CCFB002812D07E
:1043F000012C14D069460878802108430090684653
:10440000027807210020FFF79AFB00280DD0280032
:1044100038BC08BC184738BC08BC0120184769469E
:1044200008784006400E0090E9E738BC08BC01203F
:1044300018470000044C05498C4204D2002020603B
:10444000241D8C42FBD3704730F8002A9066022A64
:10445000F0B5FFB082B005000024012300216A46B8
:10446000FF4F786800F0FCFF002805D000207FB0E7
:1044700002B0F0BC08BC184770AB9878DA7999792B
:10448000120211431A7A5B7A12041B061A43114373
:10449000A84201D10800EAE770AB987CDA7D997DEB
:1044A000120211431A7E5B7E12041B061A4311434B
:1044B000A84201D10800DAE778AB9878DA799979DF
:1044C000120211431A7A5B7A12041B061A43114333
:1044D000A84201D10800CAE778AB997CDA7D987DC3
:1044E000120210431A7E5B7E12041B061A4310430D
:1044F000A942BCD00600052901D00020B7E77868A2
:10450000A11901236A4600F0ABFF002801D000206A
:10451000ADE770AB9978DA799879120210431A7A7C
:104520005B7A12041B061A43104332191018A94271
:104530009DD070AA907CD17D947D09020C43117EA0
:10454000527E0904120611430C430528D7D00020DF
:104550008DE77047C3A07047F0B50022C3494023E0
:104560000C0049105B00C829FBDC6343551C8154D7
:104570000A126C1C42550022002917DD1D042D0E65
:10458000AE461D021E062D0E360E1F0EAC46230033
:10459000641CC6547546631C055565465C1CC554B1
:1045A0002300641CC754521C8A42F0DB2000F0BC7C
:1045B00008BC1847002070470020704710B5040061
:1045C000FBF76CFF042C03D010BC08BC0720184775
:1045D00010BC08BC0020184770B50025A04C6068CE
:1045E000002803D070BC08BC00201847FBF756FF1A
:1045F0000021280000F0E3FD606000280CD0FBF7EC
:104600004DFF606801F0EEF8162809D000280CD0A4
:1046100070BC08BC0720184770BC08BC07201847AE
:104620000020A06070BC08BC1847FBF737FF0121D1
:10463000280000F0C4FDA060FBF730FF0221280035
:1046400000F0BDFDE060FBF729FF0421280000F029
:10465000B6FD2061FBF722FF0521280000F0AFFD29
:104660006061FBF71BFF0621280000F0A8FDA06198
:10467000FBF714FF0721280000F0A1FDE06170BCEA
:1046800008BC0020184770B50C001500FFF7A4FF08
:10469000072801D0002004E070BC08BC07201847A0
:1046A000401CA842FCD36E4D002007210122102C93
:1046B00052D00EDCA41E0E2C27D223007B441B7983
:1046C000DB189F4426282A4C512222534F555B5712
:1046D000592D232C5ED00CDC132C53D004DC112C70
:1046E00020D0122C11D14BE0212C4DD0222C0CD1FA
:1046F0004DE0272C5AD004DC252C4FD0262C04D199
:1047000050E0282C56D03A2C58D070BC08BC07205A
:104710001847297055E0297053E02A70286250E04C
:1047200029704EE028700B20FFF792FE002801D080
:10473000286246E00C20FFF78BFE002801D028629B
:104740003FE00E20FFF784FE002801D0286238E009
:1047500070BC08BC072018472A70286231E0287016
:1047600028622EE029702CE029702AE0297028E0C8
:10477000297026E0297024E0297022E0297020E0C9
:1047800029701EE029701CE02870286219E02A7048
:10479000286216E002212970286212E003212970A4
:1047A00028620EE00421297028620AE005212970A0
:1047B000286206E006212970286202E028702C4851
:1047C000286270BC08BC00201847002070470020F9
:1047D0007047F8B505000E00170021480278010067
:1047E0008968072A08D213007B441B79DB189F4491
:1047F0001307090B0D0F1100F8BC08BC0020184767
:104800000C000AE0C46808E0046906E0446904E0BA
:10481000846902E0C46900E04468002C02D0012AE7
:1048200004D032E0F8BC08BC07201847002E2CD179
:10483000FF20BF30405D012280280ED02800FF30CD
:10484000C130837B802B08D0807F802805D0FF205B
:10485000EF30405D802800D00022002A15D009E00A
:10486000BCF2002A654D4D43000000000008000026
:1048700000180400002908D0080000F0B3FF002849
:1048800003D0F8BC08BC07201847D148417801295B
:1048900000D0760A006A3618FBF700FE790AF805A0
:1048A00001D0012000E000200B182A003100200078
:1048B00000F046FE002803D0F8BC08BC07201847CB
:1048C000F8BC08BC002018470720704770B50600E8
:1048D00090B0BF4D2878072808D2010079440979A3
:1048E00049188F4414080A0C0E10120010B070BC46
:1048F00008BC00201847AC680AE0EC6808E02C69A6
:1049000006E06C6904E0AC6902E0EC6900E06C6808
:10491000002C0CD0FBF7C2FD2000694600F0E2FC41
:10492000002809D010B070BC08BC0720184710B090
:1049300070BC08BC072018472878002811D0012136
:104940004902300008F000FB012332000021200062
:1049500000F0F6FD00280BD010B070BC08BC07209A
:104960001847019A0021521E200000F0B2FE0DE00F
:1049700001990123491E3200200000F0E1FD0028CA
:1049800004D010B070BC08BC07201847002804D021
:1049900010B070BC08BC0720184710B070BC08BC31
:1049A0000020184710B58A480178072908D20A0064
:1049B0007A441279921897441307090B0D0F1100CE
:1049C00010BC08BC0720184784680AE0C46808E0E7
:1049D000046906E0446904E0846902E0C46900E017
:1049E0004468002C0AD0FBF759FD200000F0FAFEC5
:1049F000002807D010BC08BC0720184710BC08BC12
:104A00000720184710BC08BC00201847F8B506005E
:104A10000D0017006E480178072908D20A007A4471
:104A20001279921897441307090B0D0F1100F8BC67
:104A300008BC0720184784680AE0C46808E00469D5
:104A400006E0446904E0846902E0C46900E0446867
:104A5000002C0ED0FBF722FD2B041B0C3A0031007A
:104A6000200000F06DFD002807D0F8BC08BC07202E
:104A70001847F8BC08BC07201847F8BC08BC002041
:104A800018470720704770B590B006000D005048D9
:104A90000178072908D20A007A44127992189744BB
:104AA00014080A0C0E10120010B070BC08BC0020D4
:104AB000184784680AE0C46808E0046906E04469AD
:104AC00004E0846902E0C46900E04468002C0CD072
:104AD000FBF7E4FC2000694600F004FC002809D044
:104AE00010B070BC08BC0720184710B070BC08BCE0
:104AF00007201847402230006946FBF7F5FC28687C
:104B00004030286010B070BC08BC00201847F8B5D1
:104B1000060015002E4A1078002807D0012803D07F
:104B2000F8BC08BC00201847946800E05468002CCA
:104B300009D0480A116A4718FBF7B0FC690AE80572
:104B400005D0012004E0F8BC08BC0720184700206D
:104B50000B1832003900200000F082FC002803D03E
:104B6000F8BC08BC07201847F8BC08BC0020184750
:104B700010B51748806800F054FE0006000E0028AB
:104B800003D010BC08BC0720184710BC08BC00208C
:104B9000184710B5180001F059F910BC08BC000402
:104BA000000C184710B501F00DF910BC08BC00044A
:104BB000000C184708B5009313000A0001000020FC
:104BC00000F0AEFE01B008BC0004000C1847000065
:104BD000BCF2002AFB4980000858FF308130406851
:104BE000C007C00F002800D00120F7490006000EC2
:104BF0004870704700207047F34800787047F24AC9
:104C0000012111708200EF488058FF304130026866
:104C10000A4302607047EC4A002111708100101DA8
:104C20004058FF3041300168490849000160704731
:104C300010B50400E54902200871B22000F056FAD0
:104C4000B32000F053FAB32000F059FA012000F02D
:104C50007DFAB32000F066FA012000F077FAD94916
:104C6000A00009580122D207FF3181314A60702328
:104C7000602281212000FEF77AFAB22000F03EFA8D
:104C800010BC08BC184710B500F076FA10BC08BC80
:104C9000184710B500F06FFA10BC08BC184710B5E3
:104CA0000400FF23002284212000FEF760FAFF2386
:104CB000002287212000FEF75AFA642000F055FAFE
:104CC00010BC08BC184710B50400FF230022912136
:104CD0002000FEF74CFAFF23002293212000FEF76C
:104CE00046FA642000F041FA10BC08BC184710B521
:104CF000002909D0012904D1182308220421FEF734
:104D000036FA10BC08BC1847182300220421FEF70D
:104D10002EFA10BC08BC184770478100A9484058BB
:104D2000FF308130416A2022914341627047810007
:104D3000A4484058FF308130416A202291434162AB
:104D4000704710B504002000FFF7A9FF2000FFF70F
:104D5000BAFF022300220A212000FEF708FA0423EA
:104D600000220A212000FEF702FA10231A008421F3
:104D70002000FEF7FCF920231A0084212000FEF712
:104D8000F6F90A2000F0E2F910BC08BC184710B58B
:104D900004001023002284212000FEF7E8F92023DC
:104DA000002284212000FEF7E2F90A2000F0CEF96B
:104DB00010BC08BC184710B504002000FFF76FFFB7
:104DC0002000FFF780FF02231A0084212000FEF755
:104DD000CEF901231A0084212000FEF7C8F9202310
:104DE0001A0084212000FEF7C2F9322000F0AEF94B
:104DF00010BC08BC184710B504002000FFF74FFF97
:104E00002000FFF760FF0223002284212000FEF72C
:104E1000AEF90123002284212000FEF7A8F93220F8
:104E200000F094F910BC08BC184710B5040020002D
:104E3000FFF735FF2000FFF746FF08231A00842103
:104E40002000FEF794F902231A0084212000FEF7C7
:104E50008EF901231A0084212000FEF788F9322000
:104E600000F074F910BC08BC184710B58721FEF794
:104E700058F98007C00F10BC08BC184710B587212F
:104E8000FEF74FF9C007C00F10BC08BC184710B59B
:104E90008721FEF746F9C006400F10BC08BC184732
:104EA000F1B582B000250020009001240826F3E02F
:104EB000132C7ED220007844007900188744EA0938
:104EC00015EAEA406898A9C0C3C6C9CCCFD2D5D8E4
:104ED000EC0002980121FFF70AFF0298FFF727FF75
:104EE0000298FFF72EFF0224D6E000270298FFF772
:104EF000BCFF0006000E01900298FFF7C8FF0500F6
:104F00000198012801D0002D0BD00A2000F01EF9D5
:104F10000198012803D0002D03D0082409E00524BE
:104F200007E0962000F012F97F1C3F063F0E062F87
:104F3000DCD1022C00D106240298FFF728FFABE059
:104F40000298FFF738FF0298FFF798FF0406240E37
:104F50000298FFF79CFF05000298FFF74CFF0298AC
:104F6000FEF7CCF82100294302D0012C06D007E03F
:104F7000002801D007248FE009248DE0002D03D004
:104F8000002D03D0082487E0072485E0102483E067
:104F90000298FFF710FF0298FFF770FF0406240E37
:104FA0000298FFF774FF05000298FFF724FF0298AC
:104FB00000E06FE0FEF7A2F82100294308D0012CA1
:104FC0000CD00DE070F3002A6CF3002A745E022A04
:104FD000002801D007245FE009245DE0002D03D004
:104FE000002D03D0082457E0072455E0102453E097
:104FF0000298FFF71AFF0298FFF740FF0006000E25
:10500000002802D0012847D101E00A2444E00B2403
:1050100042E00298FFF732FF0006000E022D05D095
:10502000032D09D0042D09D0102435E0012801D02A
:105030000D2431E00C242FE00E242DE00F242BE072
:105040000026112428E00126112425E0022611243F
:1050500022E0032611241FE0042611241CE005266B
:10506000112419E00626112416E00726112413E066
:105070000298FFF714FE0298FFF725FE0298002120
:10508000FFF735FE0298FFF748FE0298FEF73FF85B
:10509000122401E007261124122C06D00098009952
:1050A000401C6429009000D202E7009864280DD3C8
:1050B00007260298FFF7F3FD0298FFF704FE029817
:1050C0000021FFF714FE0298FFF727FE300003B01F
:1050D000F0BC08BC1847024802490860704700004D
:1050E00004010000C016800001207047B22801D0E2
:1050F000B328704721482249C86070477047012291
:10510000B12806D0B32803D11D49086910430861AE
:1051100070471C48016880231943016001681143EE
:1051200001607047B12807D0B32804D11448016941
:105130004908490001617047124801688022914383
:1051400001600168490849000160704770B50500B9
:105150000024002D06D90C4E300000F0DFFE641C48
:10516000AC42F9D370BC08BC184710B500F0D6FEAD
:1051700010BC08BC1847704770470000000A0000C8
:105180000029900040025012E803000010B501F021
:10519000E9FE10BC08BC184731B50024009900296D
:1051A00009D00868002806D0684603F067F9200097
:1051B00038BC08BC184738BC08BC14201847F3B5E5
:1051C000060081B000250095042E04DB03B0F0BC7E
:1051D00008BC00201847300001F0B7FE002807D0B7
:1051E000029801F065FE009003B0F0BC08BC1847BF
:1051F000300002F08BF800282DD0300001F0D0FEF6
:1052000007003C000C340299300003F010F9010053
:105210000090002924D0207A04282AD0012857D0D1
:10522000052855D0022853D0062851D0080001F097
:10523000EFF920722076207A00281ED0042821D091
:10524000200001F0AEFA002820D020610098FFF77E
:10525000A3FF00953CE003B0F0BC08BC0020184759
:10526000200003F027F9002832D1200002F0ECF8EA
:105270002EE0684603F002F92AE00098FFF78CFF61
:10528000009525E0684603F0F9F821E0F848B10000
:10529000405841680122120311434160200002F08E
:1052A000CBF9002805D020610098FFF775FF009525
:1052B0000EE00121200001F07CFE200001F0D4FA74
:1052C00000280AD0206125720098FFF765FF00953D
:1052D000009803B0F0BC08BC184702206072803709
:1052E0003D77F5E7F0B585B006000C00002003908F
:1052F000002101910091002E0AD03568002D07D0C1
:105300002868042809D305B0F0BC08BC142018474D
:1053100005B0F0BC08BC14201847002C05D00020B4
:1053200020607068411C05D005E005B0F0BC08BCE9
:105330001420184700200290287A00280BD02070F3
:10534000686AE0603068006803F055FDC00705D06A
:105350000120207604E01520039031E00020207623
:10536000287A27002037022833D0062831D0029827
:10537000002842D016200390002060606020405D2D
:10538000207400206061387100982062686BE061D1
:10539000E88FE084280040300490008820852900B0
:1053A0002000072242312A3007F024FD0498407A79
:1053B0007874E86C60630498103003C8E163A063FC
:1053C0002100300002F0C4F9039805B0F0BC08BC1D
:1053D000184730006A4601A902F039FE039001988F
:1053E00060606020405D2074E86A6061300002F017
:1053F000D2FE3871286AA060C6E7E8696060BDE740
:1054000010B5002809D00468002C06D020680428B4
:1054100007D310BC08BC0020184710BC08BC0020F3
:1054200018478C2000598030007F00280BD1207A4B
:10543000002808D0200001F0A5FE092807D010BCE4
:1054400008BC0120184710BC08BC002018470020E9
:10545000207210BC08BC184700207047002070471D
:10546000FFB505000E001F008FB0002D0AD02C687C
:10547000002C07D02068042809D313B0F0BC08BC66
:105480001420184713B0F0BC08BC142018478C2017
:1054900000598030007F002804D013B0F0BC08BC55
:1054A0001B201847207A00280CD001280FD005288F
:1054B0000DD002280BD0062809D0102013B0F0BC64
:1054C00008BC1847152013B0F0BC08BC18472800CA
:1054D00001F040FB0028F6D101231800012F00D174
:1054E000002012221100002800D11121069108A8E5
:1054F000037000200D90217A052908D0062906D0D6
:10550000616A714307916968032902D00DE007962B
:10551000F9E7069202900390049005902868012113
:1055200002AAFFF733FE0028CDD1119B02222000F2
:1055300006A9009701F049FB13B0F0BC08BC18475E
:10554000FFB505000E001F008BB0002D0AD02C689F
:10555000002C07D02068042809D30FB0F0BC08BC89
:10556000142018470FB0F0BC08BC142018478C203A
:1055700000598030007F002804D00FB0F0BC08BC78
:105580001B201847207A00280CD001280FD00528AE
:105590000DD002280BD0062809D010200FB0F0BC87
:1055A00008BC184715200FB0F0BC08BC18472800ED
:1055B00001F0D0FA0028F6D101231800012F00D104
:1055C000002019221100002800D1182102916846FC
:1055D000037400200990207A052808D0062806D0F8
:1055E000606A704303906868032802D002E0039663
:1055F000F9E702920D9B0022200002A9009701F01A
:10560000E4FA0FB0F0BC08BC18470120704700282E
:1056100007D004210180174941808021416000208A
:1056200070471420704770B50D000024042803DB78
:1056300070BC08BC0020184703F0DDFBC10702D096
:10564000012D00D10124800700D50124200070BC69
:1056500008BC184701207047F0B50E0089B0082734
:10566000042809DB142009B0F0BC08BC184700006E
:10567000F065022A0002000001F092FC05000C35E2
:105680000124002001900290039004900590069060
:10569000079008900D2000900120694608726889E3
:1056A00000040190280001F0F4FD0398C004000FED
:1056B0000399C905C90F864201D1012907D02000ED
:1056C0000F21641C09038842DBD33800CBE7002795
:1056D000FBE7F0B589B003000C001600002B0AD0E0
:1056E0001D68002D07D02868042809D309B0F0BC34
:1056F00008BC1420184709B0F0BC08BC1420184797
:10570000287A062806D0022804D0162009B0F0BC5A
:1057100008BC1847180001F01DFA0028F6D1012036
:1057200069460872002707970194232000902800FB
:1057300001F0AFFD0028E9D1287A062818D0761E9E
:10574000700200190190242000902800694601F0A1
:10575000A0FD0028DAD101200790019726200090B3
:105760002800694601F095FDFE49002804D007E0B5
:10577000A019401E0190E6E7039A0A4200D00F20CC
:105780000728C3D10398084204D009B0F0BC08BC74
:105790000F201847280001F00FFD0728FAD009B0A4
:1057A000F0BC08BC184710B5002809D000680028D4
:1057B00006D00168042907D310BC08BC1420184780
:1057C00010BC08BC14201847017A062903D010BC6D
:1057D00008BC16201847E44902F027F910BC08BCA1
:1057E0000028184710B5002809D00168002906D004
:1057F0000A68042A07D310BC08BC1420184710BC40
:1058000008BC14201847097A022905D0062903D0BC
:1058100010BC08BC1620184702F0D7FC10BC08BC0E
:10582000184710B500280BD00168002908D00A6875
:1058300012041214042A07DB10BC08BC14201847F9
:1058400010BC08BC142018470A7A022A01D0062A84
:1058500003D14031897F012903D010BC08BC162038
:10586000184702F045FC10BC08BC184716207047CA
:1058700000280CD08178022901D0062907D1002206
:10588000825EBA490A6082780A718088C88070474F
:105890001620704710B5002807D00268002A04D0EF
:1058A00002F0C8FC10BC08BC184710BC08BC14208F
:1058B0001847F8B50D0016001F00AD4CA16800296F
:1058C00005D10121FFF77BFCA060002809D0A0686A
:1058D0003B002A003100FFF7C3FDF8BC08BC0028DC
:1058E0001847F8BC08BC16201847F8B50D0016007C
:1058F0001F009F4C2168002904D1FFF760FC206045
:10590000002809D020683B002A003100FFF7A8FDDD
:10591000F8BC08BC00281847F8BC08BC162018477B
:10592000FFB5FFB006001500FFB01C0091B004A841
:10593000859086AF8E484068002802D00068002815
:1059400007D103213000FFF73AFC8949486000285D
:1059500052D0200A0126411C002978D93A00803211
:10596000FFA98A6364324A639C320A634032CA6286
:10597000859A401CFF32E1328A62486285983C0079
:10598000E430FF34E1340862280A2906090C084390
:10599000FFAAD061C421380007F0F8FAFFAA906B83
:1059A000002141648164C164016541658165C1650F
:1059B0000166FF21506B013107F0E8FAFFAA106B76
:1059C000002141668166C1660167D16A0020486393
:1059D000D069208300206083A0836648E083644808
:1059E000406801F0B7F8002808D011207FB07FB0E0
:1059F00015B0F0BC08BC18471620F7E75C48012139
:105A000040686A460068FFF7C1FB002801D0AA2061
:105A1000ECE75748FFA9C969406801233A00FFF73E
:105A20008FFD002804D052484068FFF7B5FBDDE742
:105A30004F48FFA9859AC96940680123FFF710FD07
:105A4000002805D04A484068FFF7A6FBCEE734E0BF
:105A5000FFA8806A808B010A0006000C0143FFA8A2
:105A6000406E0160002907D041484068FFF794FB71
:105A7000FFA8406E0068B9E7FFABFF22196A586CB7
:105A8000013207F0B7F901214902380007F07EFA28
:105A900001218598490207F057FA6D1C2D042D0C41
:105AA000FFAB586CFF30013058643000761C596AE7
:105AB0003604360C884200D266E72D484068FFF76E
:105AC0006BFB002892E730B5C9B0040002ADFF229D
:105AD00021000132E431280007F0F8F92000FF30FE
:105AE0008130010064310EC9006F449342AB06C39C
:105AF00045902148005946902000FF30E130018B4D
:105B000040AA9183418BD183818B1184C08B5084B7
:105B10002020C434FF2301901D332A00132117A035
:105B2000009402F02EFE49B030BC08BC012018479A
:105B3000F7B5174B05009D44164A04A86A44106245
:105B400051620B4F7E68002E2FD0306800282CD079
:105B500010480C04240C3DAA6844082D826277D2B8
:105B60001AE000000080FFFD0001A20388F3002A74
:105B700078F3002A00040000F40100004A52443A7D
:105B8000313233343536373839303A54455354008E
:105B9000D0F7FFFF000800002800784400790018C3
:105BA0008744092E5779D4D4D4A05520C54B9D44A1
:105BB000F0BC08BC1847C44AC4216A44106A07F004
:105BC000E5F9C24836AA031D076818CBC1683597A6
:105BD00018C2389100693990BB4AFF2401346A44E5
:105BE000906A210007F0D2F900207D907E907F908E
:105BF0008090819080AA108150819081D48192E020
:105C0000B148C4216844006A07F0C0F9AE48FF21DA
:105C10006844806A013107F0B9F9AB486844046907
:105C20004369C26981697E937FAB7D9406C300217D
:105C3000359136913791389139913A913B913C9118
:105C4000819180A8018141818181A149C1816AE05E
:105C50007CE09D4BC4216B44186A07F097F99A4B7E
:105C6000FF226B44996B986A013207F0C3F8002059
:105C70007D907E907F908090F968819180AB1C81AF
:105C80009449598198819448D8818F4B6B44186A04
:105C9000FFF719FF47E08C4AC4216A44106A07F0F5
:105CA00075F90020359036903790389039903A90B9
:105CB0003B903C90844AFF216A44906A013107F08E
:105CC00065F9814A6A44100010308BC880977DAF17
:105CD0000BC70020819080AA1481508190817F4859
:105CE000D08120E07848C4216844006A07F04EF96A
:105CF0000024359436943794389439943A943B94EC
:105D00003C947148FF216844806A013107F03EF9F4
:105D10007D947E947F948094819480A804814481B2
:105D200084816F49C181300000F014FF002800D049
:105D30003CE7022D6A4617D0002D15D030680121AE
:105D4000FFF724FA002814D022202FE75E4C01230D
:105D50006C44A26B616A3000FFF782FB002801D01F
:105D6000552023E7002021E75E493068FFF70EFA4F
:105D7000E8E7554C01236C44226A616A3000FFF762
:105D8000DFFB0028D4D111E730B5FFB00D0082B0A1
:105D90006C46220029000120FFF7CAFE002807D127
:105DA000220029000620FFF7C3FE002805D022208C
:105DB0007FB002B030BC08BC18474B497D98C86022
:105DC0000020F5E7FFB50700FFB01D0082B06E466A
:105DD000454C6068002802D00068002806D10321E5
:105DE0000020FFF7ECF96060002813D000221100BA
:105DF0001000FFF7C9FF002807D182993A0002205E
:105E0000FFF796FE002807D013207FB006B0F0BC45
:105E100008BC18471120F8E782993A000720FFF7DD
:105E200087FE002801D01420EFE782993200052078
:105E3000FFF77EFE002801D01520E6E770A8808FCE
:105E400028606068FFF7A8F90020DEE770B5FFB0B2
:105E500081B005006E46244C6068002802D00068BE
:105E6000002806D103210020FFF7A9F9606000286F
:105E700013D0002211001000FFF75AFE002807D1AE
:105E8000002211000720FFF753FE002807D0222030
:105E90007FB001B070BC08BC18475520F8E732004D
:105EA00000210420FFF744FE002800D00120002834
:105EB000EED170A8808F28606068FFF76DF9002030
:105EC000E6E700003C080000000800007C5B002AB8
:105ED00000020000000100000003000000040000B8
:105EE000000500000100008078F3002A10B5094980
:105EF000401807F0E5FB0848016010BC08BC1847D3
:105F000010B50449401807F0DBFB0348416010BCA2
:105F100008BC1847E7030000B4F3002A10B5044991
:105F20000968484307F074FB10BC08BC1847000020
:105F3000B4F3002A002802D0FE49006808607047C8
:105F4000F8B50C000F2824D20022FB4F8300FE5826
:105F50000DE06968182555434959814206D1182139
:105F60004A43F64840688018F85006E0521C002E5C
:105F700003D1F24D29689142EBD8FD58002D08D08D
:105F8000EF481918280002F0D9FF002C01D0A868AA
:105F90002060F8BC08BC18470F280CD28100E648E6
:105FA0004058002807D0E64A5158002903D0096814
:105FB000002900D0084770470F280CD28100DE4826
:105FC0004058002807D0DE4A5158002903D04968BC
:105FD000002900D0084770470F280ED28100D6480C
:105FE0004058002809D0D64A5258002A05D0926855
:105FF000002A02D0D34BC918104770470F280ED281
:106000008100CD484058002809D0CD4A5258002A76
:1060100005D0D268002A02D0CA4BC9181047704771
:106020000F2806D28100C4484058002801D040689B
:1060300070470020704730B40F280DD28300BE484F
:10604000C058002808D0BE4CE358002B04D01B6970
:10605000002B01D030BC184730BC70470F280CD241
:106060008200B5488058002807D0B54B9A58002ABE
:1060700003D05269002A00D0104770470F280CD275
:106080008200AD488058002807D0AD4B9A58002AAE
:1060900003D09269002A00D0104770470F280CD215
:1060A0008200A5488058002807D0A54B9A58002A9E
:1060B00003D0D269002A00D0104770470F280CD2B5
:1060C00082009D488058002807D09D4B9A58002A8E
:1060D00003D0126A002A00D0104770470F280CD254
:1060E000810095484058002807D0954A515800290A
:1060F00003D0496A002902D00847002070470020D9
:1061000070470F280CD281008B484058002807D0D8
:106110008B4A5158002903D0896A002902D00847C8
:1061200000207047002070470F280CD28100824861
:106130004058002807D0824A5158002903D0C96A24
:10614000002902D0084701207047012070470F281E
:106150000CD2810078484058002807D0784A51581E
:10616000002903D0096B002902D00847002070479E
:106170000020704770B50C0073490F2816D28300B9
:106180006D48C058002811D06D4DEB58002B0DD034
:106190005D6B002D1AD04369002B0FD01E68002EB6
:1061A0000CD01E68A64205D1596807E070BC08BC37
:1061B0000020184708331E68002EF2D1002905DBA5
:1061C00007F07BFA70BC08BC0120184770BC08BC03
:1061D0000020184770B50C005B490F2816D28300C9
:1061E0005548C058002811D0554DEB58002B0DD004
:1061F0009D6B002D1AD04369002B0FD01E68002E16
:106200000CD01E68A64205D1596807E070BC08BCD6
:106210000020184708331E68002EF2D1002905DB44
:1062200007F04BFA70BC08BC0120184770BC08BCD2
:106230000020184730B40F2812D284003E4800597D
:1062400000280DD03E4D2C59002C09D0E46B002CB9
:1062500009D0002907D0002A05D0A44630BC6047E9
:1062600030BC0020704730BC0020704730B40F288D
:1062700012D284003048005900280DD0304D2C59DE
:10628000002C09D0246C002C09D0002907D0002A4A
:1062900005D0A44630BC604730BC0020704730BCFD
:1062A0000020704730B40F2812D2840022480059D1
:1062B00000280DD0224D2C59002C09D0646C002CE4
:1062C00009D0002907D0002A05D0A44630BC604779
:1062D00030BC0020704730BC0020704730B40F281D
:1062E00012D284001448005900280DD0144D2C59A6
:1062F000002C09D0A46C002C09D0002907D0002A5A
:1063000005D0A44630BC604730BC0020704730BC8C
:10631000002070470F2819D28200074880580028B3
:1063200014D0074B9A58002A10D0D26C002A0DD0F6
:1063300010470000BCF3002AFC5E022AA4EB002AEE
:10634000385F022A745F022AFFFFFFFF704730B4F4
:106350000F280DD283005D48C058002808D05C4C3F
:10636000E358002B04D01B6D002B01D030BC184724
:1063700030BC704730B40F280DD283005348C0584A
:10638000002808D0524CE358002B04D05B6D002B42
:1063900001D030BC184730BC7047F0B40D004D49F7
:1063A0000F281FD284004948005900281AD0484EAF
:1063B0003459002C16D0A66D002E13D04469002C41
:1063C0000BD02768002F08D02768AF4201D1616841
:1063D00003E008342768002FF6D1002902DBB44619
:1063E000F0BC6047F0BC7047F0B40D0039490F288D
:1063F00021D284003548005900281CD0344E34592D
:10640000002C18D0E66D002E15D0002B13D0446957
:10641000002C0BD02768002F08D02768AF4201D18D
:10642000616803E008342768002FF6D1002902DBF9
:10643000B446F0BC6047F0BC70470F280CD2820015
:1064400022488058002807D0214B9A58002A03D0B0
:10645000126E002A00D0104770470F280CD282001D
:106460001A488058002807D0194B9A58002A03D0A0
:10647000526E002A00D0104770470F280ED28200BB
:1064800012488058002809D0114B9A58002A05D08C
:10649000926E002A04D0002902D0104700207047D5
:1064A0000020704730B40F280DD283000748C05831
:1064B000002808D0064CE358002B04D0DB6E002BDC
:1064C00001D030BC184730BC70470000FC5E022A87
:1064D000385F022AFFFFFFFF10B50022F121B5202F
:1064E00000F07FF800280022E821B52000F079F8BC
:1064F00000280022E921B52000F073F800280022CE
:10650000BF21B52000F06DF800280022C521B5207C
:1065100000F067F800280022EF21B52000F061F8B4
:1065200000280022F021B52000F05BF800280022AE
:106530000221B52000F055F810BC08BC002818470F
:1065400010B50022F121B52000F04BF80028002200
:10655000E821B52000F045F80028FF2100220B318A
:10656000B52000F03EF800280022BF21B52000F041
:1065700038F800280022C521B52000F032F80028A4
:10658000FF2100220D31B52000F02BF80028002259
:10659000F021B52000F025F8002800220221B520C6
:1065A00000F01FF810BC08BC0028184710B5040004
:1065B0000020FDF75CFB172807D019280BD01828FE
:1065C00009D010BC08BC322018472000FFF7B8FFE4
:1065D00010BC08BC18472000FFF77EFF10BC08BCA9
:1065E000184710B50006000E05F06AF810BC08BC8C
:1065F000184700000120704700680121FB4AC905C7
:1066000080001258506B08400028FBD000207047D3
:10661000F8B5050028680168042903D30020F8BCF8
:1066200008BC1847F14E8C00305901680122114313
:10663000016030594168120211434160305941688C
:106640005700B94341607D20C00002F07BFA305909
:106650004168394341607D20C00002F073FAE44A8A
:1066600030594168E34B9943114341602868002148
:1066700000F09FFC280005F047F80028CFD1280043
:1066800001F0EFFAF8BC08BC1847F0B40124036825
:106690001D042D14067A7D27D74B3F01022E0AD008
:1066A000062E08D0002900D03B008421095800297B
:1066B00005D04B4305E00029F7D03B00F5E7CF4973
:1066C0004B43A900C94D6E587362836D012B02D1F3
:1066D000406A0404240C1000604369588862F0BCCE
:1066E000704710B58AB0020003200190012069466E
:1066F000087300210891107A02280DD006280BD0CB
:106700000291100001A900F0C4FD0498040C2000BF
:106710000AB010BC08BC18470224B9480290100007
:1067200001A900F0B6FDF2E7F8B507000825B54E5F
:106730000124380000F026FD04280AD0642002F06D
:1067400001FA2000641CB042F3D32800F8BC08BC56
:1067500018470025F9E770B401680820A34B01220F
:10676000050489005B58A84C596B1A260E40002E70
:1067700002D00E2070BC70472A260E40002E02D098
:106780000D2070BC70472140002904D09F489863B9
:10679000002070BC70471100521CA942E4D370BCA9
:1067A000704730B589B004000220009000200190AD
:1067B00004216A46117207902000694600F069FDC5
:1067C0000500002D04D0280009B030BC08BC1847D3
:1067D000227A03A8022A07D0062A05D0210005F054
:1067E000BAF9002813D004E0210001F0D8FB0028FA
:1067F00008D02000FFF775FF6081280009B030BC89
:1068000008BC184709B030BC08BC1420184709B0B0
:1068100030BC08BC1420184730B589B004007C4D4A
:106820001020009001950120694608720020079011
:10683000200000F02EFD0100002902D10398800005
:10684000002800290BD165622068820067488058C3
:10685000C26A704B1A4001235B031A43C26209B03B
:1068600030BC08BC08001847F0B583B004002768A6
:106870000121200000F048FF00281DD10220607295
:106880000126A6652000FFF7C7FF0500207A022831
:1068900006D0062804D0012816D0052814D03DE0E3
:1068A00000215D20005D04280AD3200001F0B0FA29
:1068B0000500002D32D0280003B0F0BC08BC1847FA
:1068C000380001F003FA29E066630020019002908D
:1068D000200001A904F095FF0028EDD16846007A58
:1068E00005280ED00021380002F0FFFA200005F044
:1068F000DAF80500002D0AD0280003B0F0BC08BC6F
:106900001847200005F0E5F80028F6D1EEE76846C4
:106910004079002802D0200005F025F8200000F082
:1069200031FC042800D00925280003B0F0BC08BCC5
:10693000184700B5030089B00020002A13D00C20AE
:10694000009001206A46107201290AD000200790A9
:10695000002001901800694600F09BFC09B008BCBB
:1069600018470120F3E70129F8D11800FFF7DCFEF2
:1069700009B008BC1847F7B50C00150084B000201A
:10698000029004980768002001900126A00700D01B
:106990000026002C0ED0002D51DDB80003901348C6
:1069A00003994158486B2A220240002A07D00D2043
:1069B000029044E007B0F0BC08BC0D201847002D41
:1069C0003BD0154A0240002A37D0094A104000281F
:1069D00024D0002E22D001952100380001AA05F014
:1069E000ABFE0198291A0C19050026E0F065022A71
:1069F0000080000000C000008813000050C30000A9
:106A0000000002000000080000010000FF078001F4
:106A1000000200000F00FEFF000020008031086827
:106A2000002E02D02060241D06E000212070000A04
:106A3000641C491C0429F9D32D1F002DAFDC0298DA
:106A40000D2802D1049800F01FFDF948BA00F7495B
:106A500080588163029807B0F0BC08BC1847F0B5B5
:106A60000C00150085B000210491006803900020FF
:106A700002900120A20700D000200190002C11D02C
:106A80000398EA4A8600EA4880598263002D42DD75
:106A9000E7488759796B1A200840002807D00E2054
:106AA000049038E005B0F0BC08BC0E201847002D5B
:106AB0002FD0E048084000282BD1DF4808400028AC
:106AC00012D0019800280FD0202D0DDB02950398DD
:106AD000210002AA05F046FE0298291A0C190500A9
:106AE000D3488059416B14E00198002805D02068F4
:106AF00080373860241D2D1F0BE0002200202378F2
:106B000083401A43641C08302028F8D380373A6049
:106B10002D1F002DBCDC0498002812D1C74B0800A3
:106B2000184000280DD1C24882591A20014000297E
:106B300002D00E20049004E0516B08001840002899
:106B4000F3D0BB49B94889598863049805B0F0BCB3
:106B500008BC184710B5002804D001684268531CCF
:106B600004D004E010BC08BC1420184700224B6875
:106B7000934203D110BC08BC00201847097A0229AF
:106B800005D0062903D010BC08BC1620184701F018
:106B90003EFA10BC08BC184730B589B004000D009F
:106BA0003722009262891004019001206946087220
:106BB00000200790200000F06CFB2900200000F06E
:106BC00068FB09B030BC08BC1847FFB587B0109E01
:106BD000040015000020049000278C20005900902C
:106BE00020680021820092488058C162A807C1171E
:106BF0000691491C32002000FFF747FD03900398DF
:106C0000002824D0002001900290A06D002800D020
:106C1000666A69468E8001204872A80701D5012066
:106C20000872009E8036306A002802D00120694632
:106C30008871A80703D5206801A905F0FBFCE807C7
:106C40000BD008992000FFF7A7FF05900AE0142059
:106C500020610BB0F0BC08BC18470899200000F078
:106C600018FB0590059800283AD1306A002816D004
:106C70000123A80700D40223B76A039A0A9900984F
:106C800006F01CFD0700002F09D1A80703D42068D7
:106C900001A905F0CFFC2000FFF75DFD0490306AEC
:106CA000002801D0002F1BD0A80706D5039A0A9907
:106CB0000098FFF760FE04900CE0002069468871A0
:106CC000206801A905F0B6FC039A0A990098FFF71D
:106CD000C6FE049020680021820055488058C16299
:106CE0006068032803D00022E8070DD013E0206875
:106CF0000421FEF7B1FC0490049800281FD00BB0CB
:106D0000F0BC08BC2920184708980068122801D058
:106D1000192800D1012206992000491CFFF709FE1D
:106D20000590306A00280AD0002F08D10121A80759
:106D300000D40221F26A009806F0BEFC0490049987
:106D40000598002900D0049820610BB0F0BC08BC65
:106D5000184730B589B004000A200090608900040B
:106D6000019004206946087200200790200000F07E
:106D700090FA0500002D04D0280009B030BC08BCF2
:106D80001847227A022A06D0062A04D009B030BC5D
:106D900008BC14201847210003A801F000F90028BE
:106DA00004D0280009B030BC08BC184709B030BC7A
:106DB00008BC14201847F8B50400206806043614EF
:106DC00000271F490025200000F02FFE00282AD1AF
:106DD0003900300000F07AFF0021200000F094FC20
:106DE000002820D1200000F027FC00281BD1200023
:106DF000FFF7AFFF002816D10D48B1004058416899
:106E000001221203114341600121200000F0D1F85A
:106E10002000FFF729FD002805D10221617280348E
:106E2000E16880310D77F8BC08BC1847FF07800186
:106E3000F065022A0000010000400000000100008F
:106E40000000B703F8B506000024300000F0A8F8F1
:106E50000500002D01D02C000C34607A012823D0CD
:106E6000022821D09021200006F090F820008030E8
:106E70000700C56026602E600120287100221100E5
:106E8000300001F07CFE02F01BF8266001206072E9
:106E9000A065F868002180300162280000F026FA21
:106EA000F8BC08BC01201847F8BC08BC01201847F2
:106EB000F1B5394E37680025380000F071F804004C
:106EC0000C34042F38D23800FFF7BCFF002833D031
:106ED0000099380001F0ABFA0500002D1CD0207A93
:106EE000012829D0052827D0022825D0062823D01C
:106EF00030792072F0886081207A2076207A00280C
:106F000013D02000FFF757FF002813D0206128007E
:106F1000FEF742F900250FE0200001F0CBFA00282F
:106F20000AD1200000F090FA06E02800FEF734F9BC
:106F3000002501E019486060002D02D1002030607A
:106F400070602800F8BC08BC184713490A688242E0
:106F500004D10879022803D0062801D00020704708
:106F60000120704730B5140089B0172200920191BA
:106F700001216A46117200210791694600F089F9E2
:106F8000002802D103998900002903A92EC92EC423
:106F900009B030BC08BC184788F3002AFFFFFFFF88
:106FA000042801D300207047B0214843FF4940180E
:106FB0007047F8B505000E002F682C7A380001F0F4
:106FC00059FF02002900FA484031052E30D2330023
:106FD0007B441B79DB189F44021414140600F54807
:106FE0000223CB7724E0022C06D0062C04D0012CFF
:106FF00005D0052C03D004E00423CB7701E0012366
:10700000CB77022C06D0062C04D0012C0CD0052CFA
:107010000AD00DE0C97F042902D0032902D007E07D
:10702000E54805E0E54803E0C87F01280FD0E448C3
:10703000904200D31000009002223800694601F00F
:107040009EFD009880356860F8BC08BC1847DD4894
:10705000EEE7F8B500681927DB4D01247F018600B3
:10706000A859406B80210840002806D10A2001F071
:1070700069FD2000641CB842F2D3BC4214D28020C7
:10708000AA5929009063651CBC420DD20C00A0597E
:10709000406B8021084000280AD00A2001F052FDF0
:1070A00028006D1CB842F2D3F8BC08BC0620184773
:1070B000F8BC08BC00201847F0B400270A7A002A60
:1070C00021D0042A17D001240B000C330022002CFD
:1070D0000BD90568AE00BC4DAD5996001436AD59BC
:1070E0001D601B1D521CA242F3D30868342804D033
:1070F000352802D007E00424E6E7C868CF2109025A
:10710000084200D00B273800F0BC7047F0B40200F2
:1071100001201268AC4C0123C70495006459626BCE
:1071200040261640002E0DD04020A74BA063002023
:10713000A64C16002640002E21D05B599C630023EC
:10714000CB611CE004261640002E03D00420A0636F
:10715000022014E0D607F60F002E0CD0086829286C
:1071600007D0012805D0052803D004200123A363FC
:1071700005E00020FAE71E005B1CBE42CFD30A6286
:10718000F0BC704710B58AB009240D21019101218E
:107190006A4611730021089141890904029101A9ED
:1071A00000F077F8002802D10498C004040F2000F2
:1071B0000AB010BC08BC1847F1B507250098006854
:1071C000824F0124860080488059406B3840002857
:1071D00004D07D4880598763002508E00A2001F02B
:1071E000B1FC21000120641CC0048142EBD3002DBE
:1071F00005D00098FFF7C6FF042800D1002528001D
:10720000F8BC08BC1847F0B585B00068002200271C
:10721000009701970297039704976B4E6C4C83007D
:107220007D25ED00AA4202D3F258D76207E0F55857
:10723000AC63521CF5586D6B2540002DF0D10A68E7
:107240006C46A2810123A3800A7A002A06D06A46EE
:1072500053810A7A042A01D16A461381CA69002A35
:1072600001D06A4653800A68352A07D0112A05D012
:10727000122A03D0182A01D0192A01D16A46138094
:1072800049680491694605F0AFF905B0F0BC08BC47
:10729000184770B506000C00002521003000FFF7EC
:1072A000B2FF2068002813D0207A00280AD02100DD
:1072B0003000FFF72BFF00280DD121003000FFF731
:1072C000FBFE0500E06900280CD0002D06D009E087
:1072D0003000FFF7BEFE70BC08BC18473000FFF757
:1072E0006BFF0500280070BC08BC184710B500688B
:1072F000012101F08CFD10BC08BC184710B50068D6
:10730000002101F084FD10BC08BC1847F8B504004A
:10731000042C03D3F8BC08BC002018472000FFF75A
:107320003FFE060035000C352F008037FE60687A7E
:10733000012808D0022806D00021A02081513079F0
:10734000002804D01FE0F8BC08BC01201847902199
:10735000280005F01BFEFE602C60346001203071B7
:107360001C49002008551C4908551C480078002875
:1073700009D101F0D1FD0100012210008840174918
:10738000401E48600A703000FFF7B0FF0022110075
:10739000200001F0F4FB05212800FFF70AFE7D2004
:1073A000C00001F0CFFB01F08BFD19E0B05F022AB5
:1073B000204E00009001000020CB000090650000EE
:1073C000A861000050C30000F065022A00008000A0
:1073D000FF078001C8F3002ACCF3002AC0F3002A7B
:1073E000D7490022A0000B58DA600B58DA62D54A60
:1073F0000B589A630B585A689C46D34B9A43634682
:107400005A60D24A0B589A6308580022C26320007F
:1074100001F0FBFC2C600120687201F027FDB860D0
:107420000120A8653000FFF7E5F8002808D0012208
:107430000021200001F0A3FBF8BC08BC0120184784
:10744000F8BC08BC00201847F8B5040020008030C4
:10745000C56806002868617A002911D029790027BB
:1074600000290AD08100B6484058016849084900FF
:1074700001602800FFF742FF2F7127726772776063
:10748000F8BC08BC00201847F0B583B006000C36E5
:10749000076805213000FFF78CFDA94DBC00285975
:1074A0004168009101680191C06B029001220021A6
:1074B000380001F064FB2959009848602959019867
:1074C000086029590298C863707A022808D0002100
:1074D0003000FFF76EFD03B0F0BC08BC0120184778
:1074E00001213000FFF765FDF5E730B4002A31D007
:1074F0000B68047A022C01D0062C02D19C00240FC8
:1075000054701C0C94701C0AD4701371091D0B6804
:107510001C03240F14729C05A40D091D0B68A40004
:107520009D0F2C4314619C03640F1476007A02288B
:1075300001D006280BD15078032808D35804C00E78
:1075400050769805C00E9076D806C00ED076486862
:10755000C00F107730BC704700290FD002680E238F
:107560008B700023CB700A71426809230B7292065C
:10757000920E80681204000C02430A61704770B5D5
:1075800005000B001400002C26D01868800F207016
:10759000297A012923D0052921D0220019002800A9
:1075A000FFF7A3FF6178280040304177217F002951
:1075B00026D06178032923D301218177E07E617E83
:1075C000401C4002491C4843A17E491C4843C11746
:1075D000C90D08184012286270BC08BC1847012861
:1075E00007D0220019002800FFF77FFF70BC08BCFD
:1075F000184721001800FFF7AFFF70BC08BC184700
:107600000021817770BC08BC184730B40124921C5B
:10761000250095405B1C5D438C404462610A6943D0
:10762000C16130BC704701238B4043629902490A13
:10763000521C5143C1617047F0B595B0060030004F
:10764000FFF7A0FD032804D0092015B0F0BC08BC4A
:10765000184709200A90042008A9087400241194EE
:10766000708900040B9030000AA9FFF712FE1390F6
:107670001398002825D10094019402940394049453
:107680000594069407940894099430006A460DA95D
:10769000FFF775FF307A35004035012816D00528F0
:1076A00014D003240227062824D06846027E017ADB
:1076B000049B3000FFF7A9FF68460079322821D0EB
:1076C000EF77139815B0F0BC08BC184768460078EF
:1076D000012808D06846027E017A049B3000FFF73B
:1076E00094FFEC77EDE76846017A049A3000FFF7E3
:1076F0009AFFF6E768460079322801D0EF77E0E795
:10770000EC77DEE7EC77DCE710B50C008AB0002CF4
:1077100002D041890A0400E000220292072101916F
:1077200001216A4611730021089101A9FFF7B1FDFB
:10773000002C00D100200AB010BC08BC1847000083
:10774000F065022AFF078001000C000000004000E5
:107750004068401C0878012805D0022803D005287D
:1077600001D0062813D1012812D0052810D00228F4
:1077700001D006280BD1087C322808D017DC0F284E
:1077800005D00EDC002802D0082800D00A28704757
:10779000087C0028FBD00128F9D00228F7D0032864
:1077A00070471428FCD01E28FAD028287047642877
:1077B000FCD005DC3C28F9D04628F7D0502870478B
:1077C0007828FCD08C28FAD0A0287047F0B5FFB0FC
:1077D000FFB085B00600042E06D300207FB07FB036
:1077E00005B0F0BC08BC18473000FFF7D9FB070014
:1077F0003C000C348C20075106212172012200210B
:10780000300001F0BCF93800FFF770FD00221100D4
:10781000300001F0B4F904212000FFF7CAFB01F0A9
:107820004FFB694D0023B4002859C3602859C36237
:1078300066482959886328594168654A91434160DF
:107840006448295988632859C3632859016801226B
:107850001143016028594168120211434160300010
:1078600001F0D3FA3800FEF7C5FE002826D001212A
:10787000300001F03AFB295928004A6801231B0314
:107880001A434A600021544D02AA5154491CA9428E
:10789000FADB0022009201926B461D800121597192
:1078A0001A71005985623000694604F0C3FE2A004F
:1078B000380002A9FFF7D3F801208FE700208DE7F9
:1078C000F3B5060083B0002501950295042E04D37C
:1078D000002005B0F0BC08BC18473000FFF760FB83
:1078E00007003C000C348C20075106202072012236
:1078F0000021300001F043F93800FFF7F7FC0022C7
:107900001100300001F03BF904212000FFF751FB8A
:1079100001F0D6FA2C4D0023B4002859C360285931
:10792000C3622A482959886328594168284A9143E3
:1079300041602848295988632859C3632859016838
:10794000012211430160285941681202114341602C
:10795000300001F05AFA3800FEF74CFE00282ED015
:107960000121300001F0C1FA2859290042680123A1
:107970001B031A43426019480A59506240206A4664
:10798000908001255572157209598862300001A94D
:1079900004F050FE049940223800FEF7ECFF04008A
:1079A00000206A465072300001A904F043FE28000E
:1079B000002C8ED005B0F0BC08BC0020184705B0E4
:1079C000F0BC08BC00201847F065022AFF078001C0
:1079D000000C00000000400000040000FFFFFFFF5B
:1079E00000B589B00D21009141890904019101215F
:1079F0006A461172002107916946FFF74AFC002888
:107A000005D10398C004000F042803D0082009B052
:107A100008BC18470398000603D509B008BC13201A
:107A2000184709B008BC0020184710B504008AB0F8
:107A300006200190029101206946087308902000F9
:107A400001A9FFF726FC002803D12000FFF7C8FF9B
:107A500000280AB010BC08BC18478006400FC21EA0
:107A6000042A01D3072801D9142070470870002088
:107A7000704770B505000C0028004030017F0029D8
:107A80000FD0607B002813D0207C002810D0FF4945
:107A90002800FFF7CAFF00280ED070BC08BC0020E9
:107AA000184700212962817770BC08BC0020184764
:107AB00070BC08BC00201847607B217C80024843D2
:107AC000286270BC08BC0020184700B589B00D21A1
:107AD000009141890904019101216A461172002136
:107AE00007916946FFF7D5FB002803D103980028CA
:107AF00003DA1C2009B008BC184709B008BC0020F4
:107B0000184710B58AB0082201920024029401227D
:107B10006B461A7308940B000092022201A9FFF72A
:107B200054F80AB010BC08BC1847F0B50E00170096
:107B300089B00024002F15D005680121D4484902DE
:107B400005F002FAD2492800FFF7DBFF002805D133
:107B5000D048C07AC108C90709D01C2009B0F0BCC0
:107B600008BC184709B0F0BC08BC142018478008AE
:107B7000C00704D01C2009B0F0BC08BC1847C64997
:107B80002800FFF752FF0028F5D1296A002906D006
:107B9000380005F0D7FB002906D0471C05E01C2063
:107BA00009B0F0BC08BC184707001C200090012059
:107BB000694608720790002F24D9287A052815D025
:107BC000062813D0286A696A6043801948430190E7
:107BD00028006946FFF75DFB0028E1D103980028E3
:107BE00008DA1C2009B0F0BC08BC1847286A6043BA
:107BF0008019ECE72800FFF768FF0028F2D1641C29
:107C0000BC42DAD309B0F0BC08BC0020184710B55C
:107C1000046801219E48490205F096F99C4920001C
:107C2000FFF76FFF002805D19A48407B8109C907FB
:107C300003D01C2010BC08BC18478108C90703D01A
:107C400010BC08BC1C201847C00703D010BC08BCDF
:107C50000020184791492000FFF7E7FE10BC08BC40
:107C60001847F0B58BB000210A91006809900024F4
:107C70008B4F0026012500950197684605720796EF
:107C800009986946FFF705FB00281AD103980028D8
:107C900011DA0398800FC00703D00398400FC00784
:107CA00004D00BB0F0BC08BC022018470BB0F0BCED
:107CB00008BC062018477B4800F044FF641C142CC5
:107CC000D9D30A980BB0F0BC08BC184770B50500B2
:107CD0000024002904D0012908D0022916D10BE084
:107CE0000021280001F001F901240FE00121280002
:107CF00001F0FBF8012409E0280001F00BF9040071
:107D0000012C03D10221280001F0EFF8002C03D050
:107D100070BC08BC0120184770BC08BC0020184784
:107D200030B4002971D003008033DC7B1A7C12024E
:107D300022435C7C24041443CC639C7CDA7C1202D6
:107D400022431C7D240414430C645C7D9A7D120242
:107D50002243DC7D240414434C641C7E5A7E1202B0
:107D600022439C7E240414438C64DA7E0C0020346D
:107D700062760500A0352A78E2746A7BA273AA7B3A
:107D8000E273EA7B6273EA7CE2726A7FA271EA7F45
:107D900062710200C032137823719378E370137913
:107DA000A370137A6370537A2370937ACB77D37A64
:107DB0008B77537B4B77937B0B77D37BCB76137C83
:107DC0008B76537C4B76937C0B76137D4B61547D85
:107DD000240223434B61947D240423434B61D47DCF
:107DE000240623434B61537F0B74927FCA730200B6
:107DF000E03213784B739278CA72FF30E130007E24
:107E0000087030BC01207047FFE730BC002070478D
:107E1000F0B59BB004002068189000200190582114
:107E200002A805F0B3F81A492000FFF76AFE0028FF
:107E30004CD1174802A9FFF773FF207A062802D118
:107E40000798002841D0079800280AD0E069002848
:107E500003D001218905884203D90798400A4002CE
:107E6000E0616846C07D002800D0E06208A8C07CC0
:107E700001A9FFF7F2FD002828D168460079250006
:107E80006035287608A8807A80070DE00001AF03EE
:107E90007062022A1063022A0001AB030001AD03E5
:107EA0000080FF4050C3000026004036002813D059
:107EB000F8492000FFF7B9FD002807D108A8807A0B
:107EC000800707D50420F07706E001201BB0F0BC46
:107ED00008BC18470320F07701212000FFF769F85C
:107EE000189800F088FF800604D5022708A80078BB
:107EF000287003E0012708A880782870E649380236
:107F000041182000FFF791FD19901998002804D01E
:107F100019981BB0F0BC08BC184718983900FFF737
:107F2000D5FEB07F012804D1200002A9FFF7A1FDF2
:107F300019900120E0676946C97C002929D0687042
:107F4000032060636846C07CC00160660720E0676C
:107F50000020102502AB8100CA18D66B002E0CD071
:107F6000666B761C66632E00E76F86403743E767D3
:107F7000D26B266A724309198A66401C0428EADB20
:107F800010A840788034207019981BB0F0BC08BC51
:107F90001847002169706063DAE70120704730B547
:107FA000002830D000292ED00268120ECA8702683D
:107FB0000C009203920F4034227702681204120ED2
:107FC00022800268A270436804228D184035AB708D
:107FD0001B0A521E002AF8DC8268120EE27100228F
:107FE00022728268120C62728268C36812041B0CCF
:107FF0001A43CA64C0680004000EFFF7CEFF30BC0D
:1080000008BC0120184730BC08BC0020184770B5D8
:1080100005684468611C00D1002400686030002CB1
:1080200002D0417800290ED0007EC000204301021A
:108030009A4801432800FFF7F8FC002800D16C6043
:1080400070BC08BC184770BC08BC1620184770B438
:1080500003684068441C00D10020002803D061243C
:10806000E45C002C16D001252C00DE6F84403442E5
:1080700013D0002814D0012817D002281BD00428C0
:1080800020D0052823D0062826D0072829D070BC68
:108090001420704770BC1620704770BC14207047C5
:1080A000D8690860002010601FE0586E8002400A06
:1080B0000860156019E0586E8002400A08600220CE
:1080C000106012E0986E0860042010600DE0D86E19
:1080D00008600520106008E0186F08600620106036
:1080E00003E0586F08600720106070BC00207047E4
:1080F00010B50468FFF78BFF002810D101216848F4
:10810000490204F021FF66492000FFF7FAFC00282D
:1081100005D16448407B8109C90703D01C2010BCED
:1081200008BC18478008C00703D010BC08BC1C203E
:1081300018475D492000FFF778FC10BC08BC1847C1
:10814000F8B504000D00160027682000FFF75FFF58
:1081500000280FD17B68002B0FD0042B0DD0052BEE
:108160000BD0062B09D0072B07D0012B0DD0022BEB
:108170000BD01620F8BC08BC18473200290020009C
:10818000FFF7D3FCF8BC08BC18472000FFF73FFD01
:10819000F8BC08BC184701684068421C00D10020A8
:1081A0006031097E012907D0022908D0072908D1AA
:1081B000002806D101207047012802D1704702280B
:1081C00001D00020704701207047F8B50468456869
:1081D000691C00D10025616BA94203D81420F8BCAA
:1081E00008BC1847FFF7D7FF01281FD060682B4F46
:1081F000002808D07820005DC10239432000FFF735
:1082000014FC0028EBD10726002D00D02E00616859
:10821000F0000843010239432000FFF706FC002864
:10822000DDD160342676F8BC08BC1847F8BC08BC21
:1082300000201847F0B50E0083B000250024006828
:1082400002900298006A01900298603040780028FD
:108250000CD00198002809D0029880300078C0071F
:1082600009D003B0F0BC08BC16201847162003B094
:10827000F0BC08BC18470027052F24D238007844EA
:108280000079001887440214171A1D00074C35683E
:1082900019E000000001B9030000B7030000B303B8
:1082A0007062022A1063022A0004AD0300008F03EB
:1082B000364C756807E0364CB56804E0354CF56817
:1082C00001E0354C3569002D2AD001982D186D1E1E
:1082D0000199280005F036F8009000980006010C7E
:1082E00002982143FFF7A1FB0028C0D100980004A9
:1082F000000E010201200004201801430298FFF73C
:1083000094FB0028B3D100980002000E0102012066
:108310004004201801430298FFF787FB0028A6D1EC
:108320007F1C052FA8DB306900281CD01B4C029A4B
:108330001B4D127E71690120022A00D100204143A9
:10834000002900D1012500272806010C02982143AD
:10835000FFF76BFB00288AD12D0A012000042418A6
:108360007F1C042FF0DB307EE721890400024118D6
:108370000298FFF75AFB0028B7D10A490298FFF785
:1083800054FB03B0F0BC08BC00281847000092035F
:10839000000095030000980300008C030000880390
:1083A0000002000000019B034D484E4A904206D84F
:1083B00000210160416081600C309042F9D9704722
:1083C000704747484749884205D80268002A03D0C9
:1083D0000C308842F9D900207047002101604160CB
:1083E000816041484168491C41607047F8B506000A
:1083F0003B4C3C4DAC420FD83B4F2068002805D089
:108400000068B04202D12000FFF7E7FF786820281B
:1084100002D00C34AC42F0D9F8BC08BC1847324842
:108420000178002902D101210170BDE77047F8B53C
:1084300006000F000120FFF7C3FF2B4D68680128DD
:1084400006DA0020FFF7BCFFF8BC08BC0020184784
:10845000FFF7B7FF0400002C09D030040014FEF72A
:108460009FFD0C30206067606868401E68600020D7
:10847000FFF7A6FF2000F8BC08BC184710B50400A1
:10848000206800280FD00120FFF79AFF21680868B4
:10849000027A002A0AD00800FFF79FFF0020FFF7AA
:1084A0008FFF0020206010BC08BC18470068FFF751
:1084B0009DFFF3E70A490C4A5268202A09D0094B6C
:1084C00099420BD80A68002A05D0824203D10120C4
:1084D0007047002070470C319942F3D90020704753
:1084E0007064022AE465022AD0F3002AF0B589B04C
:1084F000040008001100402906D008D901AE1C254F
:10850000320004F056F804E00600402513E00600AF
:108510000D004020401B0890152067194001089964
:108520003818362204F006FD172040010899381843
:108530005C2204F0FFFC0020002D11D95C27325C86
:10854000362115234A4021185B01CB181A70325C82
:1085500017235B017A40C9180A70401CA842EED369
:10856000200004F016F815204001211840222000B8
:1085700003F0D3FF2000A830050004F00AF817200C
:10858000400121184022280003F0C7FF2000FF30DF
:10859000A8222100513004F099FC2000FF30A822CD
:1085A0002900F93004F092FC09B0F0BC08BC18476F
:1085B00010B504002100FF31A8225131200004F041
:1085C00085FC2100A822FF31F931A01804F07EFCBF
:1085D00010BC08BC184710B503F09FFF10BC08BCC6
:1085E000184770B58EB004000D001600200007A9D2
:1085F00003F051FF2000A8301C22040007A903F05B
:108600008CFF2000694603F046FF320028006946CF
:1086100004F0F0FB0EB070BC08BC1847F0B5FFB01A
:10862000CAB0CEAC30CC16001F000A00010068466C
:10863000FFF75CFF3A0031006846FFF7CCFF2A00E5
:1086400021006846FFF7CDFF7FB04AB0F0BC08BC00
:108650001847F0B589B0040008001100402906D081
:1086600008D96E462025320003F0E3FB04E0060043
:10867000402513E006000D004020401B0890152007
:108680006719400108993818362204F053FC172066
:108690004001089938185C2204F04CFC0020002DA1
:1086A00011D95C27325C362115234A4021185B0121
:1086B000CB181A70325C17235B017A40C9180A7014
:1086C000401CA842EED3200003F0A3FB152040017C
:1086D00021184022200003F060FB2000A830050094
:1086E00003F097FB1720400121184022280003F0D7
:1086F00054FB2000FF30A8222100513004F0E6FB9B
:108700002000FF30A8222900F93004F0DFFB09B077
:10871000F0BC08BC184710B504002100FF31A822A6
:108720005131200004F0D2FB2100A822FF31F931A1
:10873000A01804F0CBFB10BC08BC184710B503F020
:108740002CFB10BC08BC184770B590B004000D009D
:108750001600200008A903F0DEFA2000A83020222D
:10876000040008A903F019FB2000694603F0D3FABE
:1087700032002800694604F03DFB10B070BC08BC14
:108780001847F0B5FFB0CAB0CEAC30CC16001F0011
:108790000A0001006846FFF75CFF3A0031006846B6
:1087A000FFF7CCFF2A0021006846FFF7CDFF7FB01E
:1087B0004AB0F0BC08BC1847F0B58DB00400080002
:1087C0001100802906D008D96E463025320003F00A
:1087D0004DFE04E00600802513E006000D00802019
:1087E000401B0C902920671940010C99381836223B
:1087F00004F0A0FB2D2040010C9938185C2204F0F5
:1088000099FB0020002D11D95C27325C36212923E9
:108810004A4021185B01CB181A70325C2D235B0192
:108820007A40C9180A70401CA842EED3200003F019
:1088300009FE2920400121188022200003F0C6FDF6
:108840002000FF304930060003F0FCFD2D204001E0
:1088500021188022300003F0B9FDFF25493568005A
:108860002A002100201804F031FB7B20C0002A00E0
:108870003100201804F02AFB0DB0F0BC08BC1847EA
:1088800070B50400FF254935680021182A00200032
:1088900004F01CFB7B20C00021182A00601904F0A2
:1088A00015FB70BC08BC184710B503F08FFD10BC59
:1088B00008BC184770B598B004000D0016002000E1
:1088C0000CA903F02CFD2000FF30493030220400B9
:1088D0000CA903F07BFD2000694603F020FD320067
:1088E0002800694604F086FA18B070BC08BC184726
:1088F000FFB56C4C6C4AA5446A44D56C946C1F005F
:108900000A0001006E463000FFF756FF66493A0044
:108910006944C96A3000FFF7C7FF2A002100300010
:10892000FFF7C8FF614CA544F0BC08BC1847F0B580
:1089300091B0040008001100802906D008D96E46C5
:108940004025320003F0D6FC04E00600802513E049
:1089500006000D008020401B10902920671940015F
:1089600010993818362204F0E5FA2D2040011099AC
:1089700038185C2204F0DEFA0020002D11D95C27A3
:10898000325C362129234A4021185B01CB181A702A
:10899000325C2D235B017A40C9180A70401CA84242
:1089A000EED3200003F092FC292040012118802200
:1089B000200003F04FFC2000FF304930060003F098
:1089C00085FC2D20400121188022300003F042FC5C
:1089D000FF25493568002A002100201804F076FAA6
:1089E0007B20C0002A003100201804F06FFA11B07B
:1089F000F0BC08BC184770B50400FF254935680075
:108A000021182A00200004F061FA7B20C000211800
:108A10002A00601904F05AFA70BC08BC184710B557
:108A200003F018FC10BC08BC184770B5A0B00400D7
:108A30000D001600200010A903F0B5FB2000FF3048
:108A400049304022040010A903F004FC20006946CC
:108A500003F0A9FB32002800694604F0CBF920B0EE
:108A600070BC08BC1847FFB50E4C0F4AA5446A44B9
:108A7000D56C946C1F000A0001006E463000FFF7B1
:108A800056FF09493A006944C96A3000FFF7C7FF39
:108A90002A0021003000FFF7C8FF044CA544F0BCB9
:108AA00008BC1847DCF9FFFF000600003406000090
:108AB000F149421A88421CD00ADC072819D09028B4
:108AC00013D0FF38913810D0EC4940180BD10EE08C
:108AD0007D20C000101A0CD0E94940180BD07D2130
:108AE0000901401A07D00120704700207047032079
:108AF00070470420704705207047DF49421A8842BA
:108B00001CD008DC902813D0FF38913812D0DB49F4
:108B100040180BD110E07D20C000101A0ED0D849AB
:108B200040180DD07D210901401A09D00620704758
:108B300000207047012070470620704707207047CB
:108B40000920704770B5CF4C0025A5620121E16274
:108B500004F0DAFECC4ACD4B04F0DEFECC4B002212
:108B600004F0DAFECB4B002204F0BCFD04F066FEFC
:108B7000A16A8142FCD3E56270BC08BC1847F8B515
:108B800006000F00140002253868FFF791FF03006C
:108B90003868FFF7B2FF18204343BF4818184169EF
:108BA000002900D100250B2212028023002E36D08E
:108BB000BA4F012E75D0022E71D0032E2CD1002C6D
:108BC0002AD0B74E012C6BD0F4689443F460F4685B
:108BD0001C43F460041D90CCFF003C4307693F0434
:108BE0006D012F43AF4D3C432C40F568AE4F3D40E7
:108BF0002C43F460C068B060F0689843F060F0689F
:108C0000090205235B021943904311400843F060B9
:108C10003068102108433060F8BC08BC1847002CAD
:108C2000FAD0A24E012C2AD0F46A9443F462F46A7A
:108C30001C43F462041D90CCFF003C4307693F04D1
:108C40006D012F43974D3C432C40F56A964F3D40B4
:108C50002C43F462C068B062F06A9843F062F06A34
:108C6000090205235B021943904311400843F06257
:108C7000306A102108433062F8BC08BC1847306BDA
:108C8000012108433063FF20F530FFF75BFF306BB5
:108C9000400840003063F8BC08BC184701E03AE0E7
:108CA0009CE0002CF7D0012C28D0FC689443FC6099
:108CB000FC681C43FC60041D50CCF600344306697C
:108CC00036046D012E43774D34432C40FD68764EBB
:108CD00035402C43FC60C068B860F8689843F86081
:108CE000F868090205235B021943904311400843C9
:108CF000F8603868102108433860CCE738690121F2
:108D000008433861FF20F530FFF71CFF3869400841
:108D100040003861BFE7002C2AD0012C51D0FC6AFA
:108D20009443FC62FC6A1C43FC62041D50CCF600B8
:108D30003443066936046D012E435A4D34432C40AA
:108D4000FD6A594E35402C43FC62C068B862F86A2F
:108D50009843F862F86A090205235B0219439043BD
:108D600011400843F862386A10210843386292E7DC
:108D7000FC6A9443FC62FC6A1C43FC62041D50CCF8
:108D8000F6003443066936046D012E43454D3443E5
:108D90002C40FD6A444E35402C43FC62C068B862EA
:108DA000F86A9843F862F86A090205235B021943DE
:108DB000904311400843F862386A10210843386232
:108DC00069E7386B012108433863FF20F530FFF76E
:108DD000B9FE386B4008400038635CE73069012118
:108DE00008433061FF20F530FFF7ACFE30694008E2
:108DF000400030614FE70021042802D22C49800056
:108E00000958080070470020704700207047042868
:108E100001D302207047264A81005158002906D00C
:108E20002449254A002804D0022809D00EE0022057
:108E30007047086A03235B0318408018086205E046
:108E4000486A07235B031840801848620020704777
:108E5000042805D0082805D0102805D00420704724
:108E6000012070470420704704207047202070477D
:108E70007047704711487047A861000070B3FFFF4A
:108E800040A2FFFF00A000028DEDB5A0F7C6A03FF5
:108E9000000064400000F03FC4EA002A402890002F
:108EA000802890007F00FF0080FF00FF00289000D6
:108EB000D8F3002A80208000DB1E0000A08601007D
:108EC000164B187801280FD0154A1648026016492B
:108ED0000A60164A42604A60154A82608A60154AF2
:108EE000C260CA60012018707047002203239B02F1
:108EF000002904D001290BD0022908D11A008100D1
:108F00000848405841681A409943114341607047EE
:108F1000094AF4E70120704719207047E8F3002A56
:108F200000004012F065022A0066022A00001412B6
:108F30000000181200001C120008000010B503F019
:108F400087FD10BC08BC1847FFB583B00CAC30CC13
:108F5000109A002601200290FF2C01D100270297D1
:108F6000002901D0012900D1059370272F40002A44
:108F700004D0012A53D0032A55D14CE0002902D055
:108F8000012951D11EE00298002812D005990398BA
:108F900001AAFAF7F7FD012810D168460079A0432D
:108FA0002A0022400243019205990398FAF7C7FD6F
:108FB00004E0059903982A00FAF7C1FD012833D08F
:108FC000012631E0E143090716D0059903983A00DC
:108FD000FAF7B5FD012810D10599039801AAFAF70F
:108FE000D1FD2107090F6A4612798A43F0231943FC
:108FF00029401143019100E00195012807D16846FD
:1090000002798020059902430398FAF798FD012818
:109010000AD0012608E01800FAF71EFE04E0002935
:1090200007D0012905D02126300007B0F0BC08BCCC
:109030001847012904D1059903983A00FAF77FFDF2
:10904000012805D10097059903986A46FAF79AFD19
:10905000012809D10299012903D16A4611782140DA
:109060000091694609788D42012801D00126DBE78D
:109070000026D9E7F0B587B00327A026FF250024F6
:10908000012806D0B5287ED0232007B0F0BC08BC4C
:109090001847012907D0FF390A3975D0222007B0B7
:1090A000F0BC08BC184706A8FAF728FEA42001A9BE
:1090B00011C10022FF4B012110000394009504947C
:1090C000FFF742FF0028EAD1012001A911C10022C7
:1090D0000090F94B1100100003940494FFF734FF43
:1090E0000028DCD1642001A911C10022FF231A331A
:1090F00011001000039400950494FFF725FF002849
:10910000CDD1802001A911C100220090B823110007
:10911000100003940494FFF717FF0028BFD1F82034
:1091200001A911C100221C23110010000394009515
:109130000494FFF709FF0028B1D100224323DB008C
:109140001100100002940394019600950494FFF717
:10915000FBFE0028A3D1A82001A911C10022DE2313
:1091600011001000039400950494FFF7EDFE002811
:1091700095D1022001A911C106204F230022110020
:109180000394049401E01AE105E100901000FFF758
:10919000DBFE002883D1442001A911C10022FF2356
:1091A0008F3311001000039400950494FFF7CCFE58
:1091B000002888D1952001A911C1002289239B0094
:1091C00011001000039400950494FFF7BDFE0028E1
:1091D00087D1C62001A911C10022C82311001000A7
:1091E000039400950494FFF7AFFE002888D103A9EB
:1091F0000194029490C100221923022110000094CE
:10920000FFF7A2FE002889D10022FF23A13311001D
:10921000100002940394019600950494FFF794FEC5
:10922000002889D10022FF23A233110010000294EC
:109230000394019600950494FFF786FE002889D1D7
:109240000022FF239333110010000294039401962F
:1092500000950494FFF778FE002889D10022FF23AF
:109260009433110010000294039401960095049425
:10927000FFF76AFE00288DD10022FF239A331100E8
:10928000100002940394019600950494FFF75CFE8D
:1092900000288ED10022FF239B331100100002947E
:1092A0000394019600950494FFF74EFE00288FD199
:1092B000102001A911C10022822311001000039483
:1092C00000950494FFF740FE00288FD10022FF2371
:1092D00081331100100002940394019600950494C8
:1092E000FFF732FE00288ED10022FF2382331100C7
:1092F000100002940394019600950494FFF724FE55
:1093000000288ED1002281231100100002940394C2
:10931000019600950494FFF717FE00288FD1A12035
:1093200001A911C1002280231100100003940095AF
:109330000494FFF709FE00288FD1072001A911C16D
:109340000022FF23043311001000039400950494BD
:10935000FFF7FAFD00288ED1222001A911C10022B9
:10936000FF230D3311001000039400950494FFF7C0
:10937000EBFD00288DD103A90194029490C1002235
:109380004E4B022110000094FFF7DEFD07B0F0BC49
:1093900008BC0028184706A8FAF7B0FCF02001A97D
:1093A00011C100221C2311001000039400950494A5
:1093B000FFF7CAFD07B0F0BC08BC00281847E92930
:1093C00077D009DC022900D1FEE3BF2978D0C52976
:1093D00077D0E82908D1BEE0EF2900D1F5E3F029E4
:1093E00000D1F3E3F12904D0222007B0F0BC08BC7F
:1093F000184706A8FAF782FCBB2001A911C1FF2675
:10940000D736002233000121100003940095049404
:10941000FFF79AFD0028E8D1F82001A911C1002228
:10942000330001211000039400950494FFF78CFD94
:109430000028DAD1B8266F460294039460C7FF2350
:109440000022DF33012110000494FFF77DFD002886
:10945000CBD1B92001A911C1FF27E73700223B007A
:1094600001211000039400950494FFF76DFD00287E
:10947000BBD1CF2001A911C100223B000121100066
:10948000039400950494FFF75FFD0028ADD1F3200D
:1094900001A911C100223B00012110000394009595
:1094A0000494FFF751FD00289FD1BC2001A911C1F0
:1094B00008E063E0090200001602000066030000F5
:1094C0007FE00EE3FF230022EF330121100003941D
:1094D00000950494FFF738FD002886D1BA2001A931
:1094E00011C1FF27F73700223B0001211000039430
:1094F00000950494FFF728FD00288CD1FB2001A9DA
:1095000011C100223B000121100003940095049436
:10951000FFF71AFD00288CD1CA2001A911C1002231
:109520003B0001211000039400950494FFF70CFD0B
:1095300000288DD16F460294039460C7FF23002258
:10954000FF33012110000494FFF7FEFC07B0F0BCCC
:1095500008BC0028184706A8FAF7D0FB6F4602940B
:109560000394002260C7DC23110010000494FFF76D
:10957000EBFC002807B0F0BC08BC184706A8FAF7B7
:10958000BDFBF22001A911C1FF230022E633012116
:109590001000039400950494FFF7D6FC0028E9D14D
:1095A0006F4602940394002260C7FF23E133110049
:1095B00010000494FFF7C8FC002807B0F0BC08BCFA
:1095C000184706A8FAF79AFB562001A911C10022F4
:1095D000272311001000039400950494FFF7B4FCB6
:1095E0000028EAD11C2001A911C100222823110062
:1095F0001000039400950494FFF7A6FC0028DCD12A
:10960000C02001A911C100222923110010000394D8
:1096100000950494FFF798FC0028CED11D2001A9E5
:1096200011C1002228231100100003940095049416
:10963000FFF78AFC0028C0D1002229231100100066
:1096400001940294039400950494FFF77DFC002894
:10965000B3D11E2001A911C100222823110010003E
:10966000039400950494FFF76FFC0028A5D109200E
:1096700001A911C1002229231100100003940095B3
:109680000494FFF761FC002897D11F2001A911C1A4
:109690000022282311001000039400950494FFF782
:1096A00053FC002889D100222923110010000194C5
:1096B0000294039400950494FFF746FC002890D18F
:1096C000202001A911C100222823110010000394B9
:1096D00000950494FFF738FC002890D19D2001A943
:1096E00011C1002229231100100003940095049455
:1096F000FFF72AFC002890D1212001A911C10022E6
:10970000282311001000039400950494FFF71CFC1B
:10971000002890D100222923110010000194029406
:10972000039400950494FFF70FFC002890D12420A7
:1097300001A911C1002228231100100003940095F3
:109740000494FFF701FC002890D100222923110086
:10975000100001940294039400950494FFF7F4FB25
:10976000002891D1252001A911C100222823110030
:109770001000039400950494FFF7E6FB002891D1B4
:10978000F82001A911C1002229231100100003941F
:1097900000950494FFF7D8FB002890D1262001A95A
:1097A00011C1002228231100100003940095049495
:1097B000FFF7CAFB002890D1402001A911C1002267
:1097C000292311001000039400950494FFF7BCFBBB
:1097D000002890D1272001A911C1002228231100BF
:1097E0001000039400950494FFF7AEFB002890D17D
:1097F000F02001A911C100222923110010000394B7
:1098000000950494FFF7A0FB00288FD15B2001A9ED
:1098100011C1002227231100100003940095049425
:10982000FFF792FB00288FD1832001A911C10022EC
:109830002E2301211000039400950494FFF784FB6C
:1098400000288ED1982001A911C100222E230121C8
:109850001000039400950494FFF776FB00288ED146
:1098600000222E23012110000294039401960095FA
:109870000494FFF769FB00288FD1B42001A911C11E
:1098800000222E2301211000039400950494FFF779
:109890005BFB00288FD1E82001A911C100222E23F3
:1098A00001211000039400950494FFF74DFB00285C
:1098B0008FD1982001A911C100222F23012110006E
:1098C000039400950494FFF73FFB00288FD192206A
:1098D00001A911C100223423012110000394009535
:1098E0000494FFF731FB00288FD10022342301219B
:1098F000100002940394019600950494FFF724FB52
:10990000002890D1BC2001A911C1002234230121DB
:109910001000039400950494FFF716FB002890D1E3
:10992000F62001A911C100222A230121100003946D
:1099300000950494FFF708FB002890D1002224260C
:1099400026231100100002940394019600950494BC
:10995000FFF7FAFA00288FD1E22001A911C10022F5
:109960002A2301211000039400950494FFF7ECFAD8
:1099700000288FD1DB2001A911C100222A23012157
:109980001000039400950494FFF7DEFA00288FD1AD
:109990008D2001A911C1002234230121100003945C
:1099A00000950494FFF7D0FA00288FD1A42001A9D4
:1099B00011C1002225231100100003940095049486
:1099C000FFF7C2FA00288FD10022252311001000D2
:1099D00002940394019600950494FFF7B5FA0028C9
:1099E0008FD1812001A911C100223423012110004F
:1099F000039400950494FFF7A7FA00288FD1D42090
:109A000001A911C100223523012110000394009502
:109A10000494FFF799FA00288FD1062600224F23DD
:109A20001100100002940394019600960494FFF72D
:109A30008BFA00288FD1082001A911C100220090C3
:109A4000FE4B1100100003940494FFF77DFA0028E8
:109A50008FD1022001A911C100224F231100100053
:109A6000039400960494FFF76FFA00288FD1002228
:109A7000CD26332311001000029403940196009523
:109A80000494FFF761FA00288FD100222E230121D0
:109A9000100002940394019600950494FFF754FA81
:109AA000002890D1A42001A911C100222523110072
:109AB0001000039400950494FFF746FA00288FD114
:109AC00003A90194029490C17D230022DB000221AE
:109AD00010000094FFF738FA002807B0F0BC08BC6B
:109AE000184706A8FAF70AF9562001A911C1002261
:109AF000382311001000039400950494FFF724FA12
:109B00000028EAD11C2001A911C10022392311002B
:109B10001000039400950494FFF716FA0028DCD196
:109B2000C02001A911C100223A23110010000394A2
:109B300000950494FFF708FA0028CED11D2001A952
:109B400011C10022392311001000039400950494E0
:109B5000FFF7FAF90028C0D100223A2311001000C3
:109B600001940294039400950494FFF7EDF9002802
:109B7000B3D11E2001A911C1002239231100100008
:109B8000039400950494FFF7DFF90028A5D109207C
:109B900001A911C100223A2311001000039400957D
:109BA0000494FFF7D1F9002897D11F2001A911C112
:109BB0000022392311001000039400950494FFF74C
:109BC000C3F9002889D102E07CE313E24CE30022D0
:109BD0003A23110010000194029403940095049418
:109BE000FFF7B2F900288CD1202001A911C1002271
:109BF000392311001000039400950494FFF7A4F991
:109C000000288CD19D2001A911C100223A23110006
:109C10001000039400950494FFF796F900288CD166
:109C2000212001A911C10022392311001000039441
:109C300000950494FFF788F900288CD100223A237C
:109C40001100100001940294039400950494FFF70E
:109C50007BF900288CD1242001A911C100223923CD
:109C600011001000039400950494FFF76DF900288B
:109C70008CD100223A231100100001940294039425
:109C800000950494FFF760F900288DD1252001A9E3
:109C900011C100223923110010000394009504948F
:109CA000FFF752F900288DD1F82001A911C1002237
:109CB0003A2311001000039400950494FFF744F92F
:109CC000002890D1262001A911C1002239231100BA
:109CD0001000039400950494FFF736F9002890D102
:109CE000402001A911C100223A2311001000039461
:109CF00000950494FFF728F9002890D1272001A9A6
:109D000011C100223923110010000394009504941E
:109D1000FFF71AF9002890D1F02001A911C1002203
:109D20003A2311001000039400950494FFF70CF9F6
:109D300000288FD15B2001A911C100223823110016
:109D40001000039400950494FFF7FEF800288FD1CB
:109D5000832001A911C100223F2301211000039497
:109D600000950494FFF7F0F800288ED1982001A9FF
:109D700011C100223F230121100003940095049497
:109D8000FFF7E2F800288ED100223F2301211000C6
:109D900002940394019600950494FFF7D5F80028E7
:109DA0008FD1B42001A911C100223F23012110004D
:109DB000039400950494FFF7C7F800288FD1E8209A
:109DC00001A911C100223F23012110000394009535
:109DD0000494FFF7B9F800288FD1982001A911C188
:109DE0000022402301211000039400950494FFF702
:109DF000ABF800288FD1922001A911C10022452380
:109E000001211000039400950494FFF79DF80028A9
:109E10008FD1002245230121100002940394019662
:109E200000950494FFF790F8002890D1BC2001A978
:109E300011C1452300220121039401E042030000E7
:109E4000100000950494FFF77FF800288DD1F620CC
:109E500001A911C100223B230121100003940095A8
:109E60000494FFF771F800288DD1002224263723AF
:109E70001100100002940394019600950494FFF7DA
:109E800063F800288CD1E22001A911C100223B23F4
:109E900001211000039400950494FFF755F8002861
:109EA0008CD1DB2001A911C100223B23012110002C
:109EB000039400950494FFF747F800288CD18D2077
:109EC00001A911C10022452301211000039400952E
:109ED0000494FFF739F800288CD1A42001A911C1FE
:109EE0000022362311001000039400950494FFF71C
:109EF0002BF800288CD10022362311001000029488
:109F00000394019600950494FFF71EF800288CD165
:109F1000812001A911C100224523012110000394D1
:109F200000950494FFF710F800288FD1D42001A9E0
:109F300011C10022462301211000039400950494CE
:109F4000FFF702F800288FD1062600224F231100C8
:109F5000100002940394019600960494FEF7F4FF17
:109F600000288FD1082001A911C100220090FF4BC9
:109F70001100100003940494FEF7E6FF00288FD12F
:109F8000022001A911C100224F23110010000394E7
:109F900000960494FEF7D8FF00288FD10022CD262A
:109FA0004423110010000294039401960095049438
:109FB000FEF7CAFF00288FD100223F2301211000A5
:109FC00002940394019600950494FEF7BDFF0028C7
:109FD00090D103A90194029490C17D230022DB005B
:109FE000022110000094FEF7AFFF002807B0F0BC7C
:109FF00008BC184706A8F9F781FE152001A911C170
:10A000000022132311001000039400950494FEF71E
:10A010009BFF0028EAD1022001A911C106200022DD
:10A0200000904F231100100003940494FEF78CFF5E
:10A030000028DBD1842001A911C1FF26FD360022B2
:10A04000330001211000039400950494FEF77CFF77
:10A050000028CBD11B2001A911C10022132311001C
:10A060001000039400950494FEF76EFF0028BDD104
:10A07000992001A911C1002233000121100003948D
:10A0800000950494FEF760FF0028AFD1A32001A93A
:10A0900011C10022330001211000039400950494A3
:10A0A000FEF752FF0028A1D1AC2001A911C1761CF6
:10A0B0000022330001211000039400950494FEF760
:10A0C00043FF002892D1D22001A911C10022330000
:10A0D00001211000039400950494FEF735FF002839
:10A0E00084D1C52001A911C1002233000121100033
:10A0F000039400950494FEF727FF00288AD1CF2609
:10A10000FF230022FD3301211000029403940196E5
:10A1100000950494FEF718FF00288AD1A72001A912
:10A1200011C1FF230022FF33012110000394009589
:10A130000494FEF709FF00288BD1D02001A911C19A
:10A14000FF230022FF3301211000039400950494A3
:10A15000FEF7FAFE00288AD1FC2001A911C1FF23D5
:10A160000022FE3301211000039400950494FEF7B1
:10A17000EBFE002889D1BD2001A911C1FF230022D7
:10A18000FE3301211000039400950494FEF7DCFED9
:10A19000002888D18A2001A911C1FF230022FE33A3
:10A1A00001211000039400950494FEF7CDFE0028D1
:10A1B00088D1CE2001A911C10022FF23F93311005B
:10A1C0001000039400950494FEF7BEFE002887D18A
:10A1D000EA2001A911C10022FF23FE331100100063
:10A1E000039400950494FEF7AFFE002886D1F42076
:10A1F00001A911C10022FF23FE33110010000394B6
:10A2000000950494FEF7A0FE002886D169460294CA
:10A21000039460C1FF260022FF36330011001000B6
:10A220000494FEF791FE002886D1F82001A911C1FF
:10A230000022330011001000039400950494FEF7EF
:10A2400083FE002887D103A90194029490C1FF23C3
:10A250000022F533022110000094FEF775FE00285D
:10A2600007B0F0BC08BC184706A8F9F747FD002264
:10A27000DB230121100002940394019600950494BD
:10A28000FEF762FE0028EBD1C62001A911C1002211
:10A29000DA2311001000039400950494FEF754FE95
:10A2A0000028DDD103A90194029490C10022C823A3
:10A2B000022110000094FEF747FE07B0F0BC08BC76
:10A2C0000028184706A8F9F719FDD82001A911C1DF
:10A2D0000022072311001000039400950494FEF758
:10A2E00033FE07B0F0BC08BC00281847F0B50200E8
:10A2F00087B00020F826FF250024012A06D0B52AC1
:10A300007ED0232007B0F0BC08BC184707270129DE
:10A310000BD0FF390A3974D06729F3D0682971D07E
:10A32000222007B0F0BC08BC184706A8F9F7E6FCE5
:10A33000A82001A911C10022D42311001000039408
:10A3400000950494FEF700FE0028EAD16846007EDE
:10A35000012811D9BB2001A911C100220823110035
:10A36000100003940095049402E0000045030000EF
:10A37000FEF7EAFD0028D4D16846007E01280DD101
:10A38000AC2001A911C10022FF4B01211000039450
:10A3900000950494FEF7D8FD0028C2D16846007EDF
:10A3A00001280DD9A42001A911C10022F64B0121D9
:10A3B0001000039400950494FEF7C6FD0028B0D168
:10A3C000B52001A911C10022F04B01211000039416
:10A3D00000950494FEF7B8FD0028A2D1AD2001A994
:10A3E00011C141230022DB000121100003940095DC
:10A3F0000494FEF7A9FD002893D1012001A902E0F1
:10A4000080E182E095E011C100220090E04B110054
:10A41000100003940494FEF797FD002881D1D22008
:10A4200001A911C10022D94B01211000039400950C
:10A430000494FEF789FD002887D1F92001A911C1F4
:10A4400041230022DB0001211000039400950494B5
:10A45000FEF77AFD00288ED1642001A911C10022E7
:10A46000FF231A3311001000039400950494FEF7A3
:10A470006BFD002891D100221C23110010000294D2
:10A480000394019600950494FEF75EFD002884D1A4
:10A49000F62001A911C10022FF23D93311001000B9
:10A4A000039400950494FEF74FFD002887D1952072
:10A4B00001A911C1002289239B00110010000394FF
:10A4C00000950494FEF740FD002886D1FF26002267
:10A4D0000436330011001000029403940197009594
:10A4E0000494FEF731FD002886D133006E460294B5
:10A4F00003940022A0C6110010000494FEF724FD6E
:10A5000007B0F0BC08BC0028184706A8F9F7F6FB0E
:10A51000F02001A911C100221C2311001000039496
:10A5200000950494FEF710FD002807B0F0BC08BCAD
:10A53000184706A8F9F7E2FBA82001A911C10022DB
:10A54000D42311001000039400950494FEF7FCFC42
:10A550000028EAD16846007E01280DD9BB2001A958
:10A5600011C10022082311001000039400950494E7
:10A57000FEF7EAFC0028D8D16846007E01280DD1FC
:10A58000AC2001A911C100227F4B012110000394CE
:10A5900000950494FEF7D8FC0028C6D16846007EDA
:10A5A00001280DD9A42001A911C10022764B012157
:10A5B0001000039400950494FEF7C6FC0028B4D163
:10A5C000B52001A911C10022704B01211000039494
:10A5D00000950494FEF7B8FC0028A6D1AD2001A98F
:10A5E00011C141230022DB000121100003940095DA
:10A5F0000494FEF7A9FC002897D1012001A911C1FC
:10A6000000220090624B1100100003940494FEF7A6
:10A610009BFC002889D1D22001A911C100225B4BEB
:10A6200001211000039400950494FEF78DFC00288E
:10A630008FD1F92001A911C141230022DB000121A2
:10A640001000039400950494FEF77EFC002892D13C
:10A65000642001A911C10022FF231A331100100048
:10A66000039400950494FEF76FFC002895D1002216
:10A670001C23110010000294039401960095049489
:10A68000FEF762FC002888D12A2001A911C100220E
:10A69000FF230C3311001000039400950494FEF77F
:10A6A00053FC00288BD1F62001A911C10022FF2301
:10A6B000D93311001000039400950494FEF744FC74
:10A6C00000288AD1952001A911C1002289239B006D
:10A6D00011001000039400950494FEF735FC002847
:10A6E0008AD16E46029403940022A0C6FF2304334D
:10A6F000110010000494FEF727FC07B0F0BC08BC62
:10A7000000281847A027F02900D1FEE30ADC02291F
:10A7100000D1FBE3BF297ED0C52900D1DDE3E829C4
:10A7200008D1CCE0F1290AD0FF390B3974D00229C5
:10A7300000D1ECE3222007B0F0BC08BC184706A803
:10A74000F9F7DCFAB92001A911C1FF230022E73390
:10A7500001211000039400950494FEF7F5FB0028F6
:10A76000E9D1F32001A911C1430000220121100009
:10A77000039400950494FEF7E7FB0028DBD1CF2774
:10A78000FF230294039405E0090200000702000081
:10A79000160200000022E733012110000197009506
:10A7A0000494FEF7D1FB0028C5D1BD2001A911C139
:10A7B000FF230022DF33012110000394009504944D
:10A7C000FEF7C2FB0028B6D1FF230022DF330121B0
:10A7D000100002940394019700950494FEF7B4FBD3
:10A7E0000028A8D1F72001A911C1FF230022DF33DF
:10A7F00001211000039400950494FEF7A5FB0028A6
:10A8000099D1BA2001A911C1FF23D7330022012118
:10A810001000039401E088E064E000950494FEF7E2
:10A8200093FB002887D1CA2001A911C1FF23002270
:10A83000D73301211000039400950494FEF784FBA4
:10A8400000288DD1F42001A911C1FF230022D733A4
:10A8500001211000039400950494FEF775FB002875
:10A860008CD1BE2001A911C1FF230022EF330121A9
:10A870001000039400950494FEF766FB002893D122
:10A88000694602940394A0C1FF27EF3700223B00E2
:10A89000012110000494FEF757FB002884D13B00EF
:10A8A0006F460294039460C70022012110000494B3
:10A8B000FEF74AFB07B0F0BC08BC0028184706A802
:10A8C000F9F71CFA6E46029403940022A0C6DC231A
:10A8D000110010000494FEF737FB002807B0F0BC0D
:10A8E00008BC184706A8F9F709FAF22001A911C116
:10A8F000FF230022E6330121100003940095049405
:10A90000FEF722FB0028E9D16E4602940394002250
:10A91000A0C6FF23E133110010000494FEF714FBDE
:10A92000002807B0F0BC08BC184706A8F9F7E6F9FC
:10A93000562001A911C10022272311001000039401
:10A9400000950494FEF700FB0028EAD11C2001A921
:10A9500011C10022282311001000039400950494D3
:10A96000FEF7F2FA0028DCD1C02001A911C10022B3
:10A97000292311001000039400950494FEF7E4FAD3
:10A980000028CED11D2001A911C1002228231100C9
:10A990001000039400950494FEF7D6FA0028C0D165
:10A9A00000222923110010000194029403940095C1
:10A9B0000494FEF7C9FA0028B3D11E2001A911C1E1
:10A9C0000022282311001000039400950494FEF740
:10A9D000BBFA0028A5D1092001A911C10022292311
:10A9E00011001000039400950494FEF7ADFA0028BE
:10A9F00097D11F2001A911C10022282311001000A6
:10AA0000039400950494FEF79FFA002889D1002250
:10AA100029231100100001940294039400950494DA
:10AA2000FEF792FA002890D1202001A911C100223E
:10AA3000282311001000039400950494FEF784FA73
:10AA4000002890D19D2001A911C1002229231100C5
:10AA50001000039400950494FEF776FA002890D134
:10AA6000212001A911C10022282311001000039404
:10AA700000950494FEF768FA002890D1002229235B
:10AA80001100100001940294039400950494FEF7C1
:10AA90005BFA002890D1242001A911C100222823AB
:10AAA00011001000039400950494FEF74DFA00285D
:10AAB00090D10022292311001000019402940394E4
:10AAC00000950494FEF740FA002891D1252001A9B1
:10AAD00011C1002228231100100003940095049452
:10AAE000FEF732FA002891D100222923110010002C
:10AAF00002940394019600950494FEF725FA002829
:10AB000084D1262001A911C10022282311001000A0
:10AB1000039400950494FEF717FA002891D1402081
:10AB200001A911C1002229231100100003940095EE
:10AB30000494FEF709FA002891D1272001A911C138
:10AB40000022282311001000039400950494FEF7BE
:10AB5000FBF9002891D1F02001A911C1002229237D
:10AB600011001000039400950494FEF7EDF90028FD
:10AB700090D15B2001A911C10022272311001000F0
:10AB8000039400950494FEF7DFF9002890D1832008
:10AB900001A911C100222E23012110000394009568
:10ABA0000494FEF7D1F900288FD1982600222E2395
:10ABB0000121100002940394019600950494FEF77D
:10ABC000C3F900288FD100222E2301211000029406
:10ABD0000394019700950494FEF7B6F900288FD1ED
:10ABE000B42001A911C100222E23012110000394D9
:10ABF00000950494FEF7A8F900288FD1E82001A958
:10AC000011C100222E230121100003940095049409
:10AC1000FEF79AF900288FD100222F23012110007E
:10AC200002940394019600950494FEF78DF9002890
:10AC300090D1922001A911C10022342301211000DA
:10AC4000039400950494FEF77FF9002890D16E4696
:10AC500002940394A0C6002234230121100004941E
:10AC6000FEF772F9002891D1BC2001A911C1002280
:10AC7000342301211000039400950494FEF764F935
:10AC8000002891D1F62001A911C100222A23012117
:10AC90001000039400950494FEF756F9002891D112
:10ACA00024266F4602940394002260C726231100D5
:10ACB00010000494FEF748F9002890D1E22001A981
:10ACC00011C100222A23012110000394009504944D
:10ACD000FEF73AF9002890D1DB2001A911C100222A
:10ACE0002A2301211000039400950494FEF72CF907
:10ACF000002890D18D2001A911C100223423012107
:10AD00001000039400950494FEF71EF900288FD1DB
:10AD10000022A42725231100100002940394019718
:10AD200000950494FEF710F900288FD10022252306
:10AD30001100100002940394019600950494FEF70C
:10AD400003F900288FD1812001A911C100223423E9
:10AD500001211000039400950494FEF7F5F80028F3
:10AD60008FD1D42001A911C1002235230121100067
:10AD7000039400950494FEF7E7F800288FD1062687
:10AD800000224F23110010000294039401960096B4
:10AD90000494FEF7D9F800288FD1082001A911C129
:10ADA0000F2000220090FF4B110010000394049428
:10ADB000FEF7CAF800288ED1022001A911C1002295
:10ADC0004F2311001000039400960494FEF7BCF882
:10ADD00000288ED10022CD263323110010000294CA
:10ADE0000394019600950494FEF7AEF800288ED1E6
:10ADF00000222E2301211000029403940196009555
:10AE00000494FEF7A1F800288FD16846007E01283F
:10AE100044D1C02001A911C100222F23012110001B
:10AE2000039400950494FEF78FF800288AD1D0206F
:10AE300001A911C100222F230121100003940095C4
:10AE40000494FEF781F800288AD1ED2001A911C1F0
:10AE500000222F2301211000039400950494FEF793
:10AE600073F800288AD100222F23012110000294B8
:10AE70000394019500950494FEF766F800288BD1A1
:10AE8000842001A911C100222F2301211000039465
:10AE900000950494FEF758F800288CD16E46029471
:10AEA00003940022A0C62523110010000494FEF78D
:10AEB0004BF800288DD103207D2300220490DB0075
:10AEC000022110000194029403940094FEF73CF8D0
:10AED000002807B0F0BC08BC184706A8F8F70EFF1A
:10AEE000562001A911C1002238231100100003943B
:10AEF00000950494FEF728F80028EAD11C2001A947
:10AF000011C139230022039402E096E3C4E3B6E2C0
:10AF10001100100000950494FEF716F80028D8D10F
:10AF2000C02001A911C100223A231100100003948E
:10AF300000950494FEF708F80028CAD11D2001A945
:10AF400011C10022392311001000039400950494CC
:10AF5000FDF7FAFF0028BCD100223A2311001000AF
:10AF600001940294039400950494FDF7EDFF0028EA
:10AF7000AFD11E2001A911C10022392311001000F8
:10AF8000039400950494FDF7DFFF0028A1D1092068
:10AF900001A911C100223A23110010000394009569
:10AFA0000494FDF7D1FF002893D11F2001A911C1FE
:10AFB0000022392311001000039400950494FDF73A
:10AFC000C3FF002885D100223A231100100001940C
:10AFD0000294039400950494FDF7B6FF00288CD1E9
:10AFE000202001A911C1002239231100100003946F
:10AFF00000950494FDF7A8FF002890D19D2001A999
:10B0000011C100223A23110010000394009504940A
:10B01000FDF79AFF002890D1212001A911C100223B
:10B02000392311001000039400950494FDF78CFF60
:10B03000002890D100223A231100100001940294BC
:10B04000039400950494FDF77FFF002890D12420FD
:10B0500001A911C1002239231100100003940095A9
:10B060000494FDF771FF002890D100223A231100CB
:10B07000100001940294039400950494FDF764FF7A
:10B08000002891D1252001A911C1002239231100E6
:10B090001000039400950494FDF756FF002891D109
:10B0A00000223A23110010000294039401960095A7
:10B0B0000494FDF749FF002884D1262001A911C17D
:10B0C0000022392311001000039400950494FDF729
:10B0D0003BFF002891D1402001A911C100223A2351
:10B0E00011001000039400950494FDF72DFF002833
:10B0F00091D1272001A911C100223923110010008C
:10B10000039400950494FDF71FFF002891D1F020CF
:10B1100001A911C100223A231100100003940095E7
:10B120000494FDF711FF002890D15B2001A911C103
:10B130000022382311001000039400950494FDF7B9
:10B1400003FF002890D1832001A911C100223F23D1
:10B1500001211000039400950494FDF7F5FE0028EA
:10B160008FD1982600223F230121100002940394DE
:10B17000019600950494FDF7E7FE00288FD1002288
:10B180003F23012110000294039401970095049439
:10B19000FDF7DAFE00288FD1B42001A911C13F23A9
:10B1A000039401E0420300000022012110000095F9
:10B1B0000494FDF7C9FE00288CD1E82001A911C133
:10B1C00000223F2301211000039400950494FDF711
:10B1D000BBFE00288CD100224023012110000294E4
:10B1E0000394019600950494FDF7AEFE00288DD1DE
:10B1F000922001A911C100224523012110000394CE
:10B2000000950494FDF7A0FE00288DD16E460294AF
:10B210000394A0C600224523012110000494FDF7E9
:10B2200093FE00288ED1BC2001A911C10022452324
:10B2300001211000039400950494FDF785FE002879
:10B240008ED1F62001A911C100223B23012110005B
:10B25000039400950494FDF777FE00288ED12426F0
:10B260006F4602940394002260C737231100100038
:10B270000494FDF769FE00288DD1E22001A911C1D7
:10B2800000223B2301211000039400950494FDF754
:10B290005BFE002890D1DB2001A911C100223B23D5
:10B2A00001211000039400950494FDF74DFE002841
:10B2B00090D18D2001A911C1002245230121100048
:10B2C000039400950494FDF73FFE00288FD1A4203D
:10B2D00001A911C10022362311001000039400952A
:10B2E0000494FDF731FE00288FD16F460294039439
:10B2F000002260C73623110010000494FDF724FEDD
:10B3000000288FD1812001A911C1002245230121EC
:10B310001000039400950494FDF716FE00288FD1C9
:10B32000D42001A911C10022462301211000039459
:10B3300000950494FDF708FE00288FD10626002210
:10B340004F23110010000294039401960096049478
:10B35000FDF7FAFD00288FD1082001A911C10F20A7
:10B3600000220090E74B1100100003940494FDF7B5
:10B37000EBFD00288ED1022001A911C100224F232C
:10B3800011001000039400960494FDF7DDFD0028E1
:10B390008ED1CD266F4602940394002260C74423C9
:10B3A000110010000494FDF7CFFD00288ED16F46E8
:10B3B0000294039460C700223F23012110000494EB
:10B3C000FDF7C2FD00288FD16846007E012844D1D8
:10B3D000C02001A911C100224023012110000394C3
:10B3E00000950494FDF7B0FD00288AD1D02001A972
:10B3F00011C1002240230121100003940095049400
:10B40000FDF7A2FD00288AD1ED2001A911C100227B
:10B41000402301211000039400950494FDF794FD4E
:10B4200000288AD1002240230121100002940394B5
:10B43000019500950494FDF787FD00288BD18420A9
:10B4400001A911C10022402301211000039400959D
:10B450000494FDF779FD00288CD103207D23002280
:10B460000490DB00022110000194029403940094E4
:10B47000FDF76AFD002807B0F0BC08BC184706A815
:10B48000F8F73CFC152001A911C100220C23110082
:10B490001000039400950494FDF756FD0028EAD1AE
:10B4A000842001A911C1FF26ED36002233000121BD
:10B4B0001000039400950494FDF746FD0028DAD1AE
:10B4C0003B2001A911C100220C231100100003949C
:10B4D00000950494FDF738FD0028CCD1992001A9EE
:10B4E00011C100223300012110000394009504943F
:10B4F000FDF72AFD0028BED1A32001A911C1002219
:10B50000330001211000039400950494FDF71CFD05
:10B510000028B0D1AC2001A911C1761C0022330053
:10B5200001211000039400950494FDF70DFD0028FF
:10B53000A1D1D027002233000121100002940394EE
:10B54000019700950494FDF7FFFC002893D1C520D6
:10B5500001A911C1002233000121100003940095BC
:10B560000494FDF7F1FC002885D1EA2001A911C15E
:10B570000022330001211000039400950494FDF78C
:10B58000E3FC00288BD1C42001A911C10022731E45
:10B5900001211000039400950494FDF7D5FC0028C8
:10B5A0008DD1A72001A911C1761C002233000121F1
:10B5B0001000039400950494FDF7C6FC00288CD17C
:10B5C00033006E4602940394A0C6002201211000AD
:10B5D0000494FDF7B9FC00288DD1F42001A911C114
:10B5E000FF230022EE330121100003940095049400
:10B5F000FDF7AAFC00288CD1CE2001A911C10022A0
:10B60000FF23E93311001000039400950494FDF723
:10B610009BFC00288CD10320FF2300220490F533EB
:10B62000022110000194029403940094FDF78CFC15
:10B63000002807B0F0BC08BC184706A8F8F75EFB66
:10B640006E4602940394A0C60022DB230121100061
:10B650000494FDF779FC0028EBD1C62001A911C1A3
:10B660000022DA2311001000039400950494FDF7E2
:10B670006BFC0028DDD1032000220490C8230221A6
:10B6800010000194029403940094FDF75DFC07B050
:10B69000F0BC08BC0028184706A8F8F72FFBD820F4
:10B6A00001A911C100220723110010000394009585
:10B6B0000494FDF749FC07B0F0BC08BC002818470B
:10B6C00070B504000D0016000020F8F7D0FA172816
:10B6D00007D019280DD018280BD070BC08BC322018
:10B6E0001847320029002000FEF700FE70BC08BC9D
:10B6F0001847320029002000FDF7BCFC70BC08BCD4
:10B700001847000045030000F0B58BB000210A91F6
:10B7100000680990FF4D0026009601966846067263
:10B72000079609986946FBF7B4FD00240127082015
:10B730000090F94801906846077207960998694693
:10B74000FBF7A7FD002813D07D20C000FDF7FAF914
:10B75000641C032CEBD3002437200090019668462C
:10B76000077209986946FBF794FD00282FD10DE078
:10B7700003990800FF38AB3804D00A980BB0F0BC2E
:10B7800008BC1847012080070543E4E72920009002
:10B7900001956846077209986946FBF77AFD00280B
:10B7A00015D1039800280CDA0398400004D50BB09B
:10B7B000F0BC08BC052018470BB0F0BC08BC012049
:10B7C0001847D648FDF7BEF9641C142CC4D30A9858
:10B7D0000BB0F0BC08BC1847002910D00278130940
:10B7E0000B701207120F4A704078C2098A70420625
:10B7F000520FCA700007000F087101207047002027
:10B800007047F0B58DB004000D0000220292039243
:10B810003320049005920126684606760B92A265B5
:10B82000082000900322200002AB04A9FBF7CDF909
:10B830000700A665002F04D038000DB0F0BC08BC8E
:10B840001847290002A8FFF7C7FF38000DB0F0BC69
:10B8500008BC1847002909D0027892090A70027AB8
:10B860000A72807A000988720120704700207047B0
:10B8700070B58AB004000E00A948402101F064FBB5
:10B880000D20019000200290012569460D7308905B
:10B89000A06540200090A24B0322200001A9FBF7E5
:10B8A00094F90300A565002B04D00AB070BC180001
:10B8B00008BC18479A483100FFF7CCFF0AB070BCAB
:10B8C000180008BC184770B4002949D00278120249
:10B8D0000A8043781A430A8002230522C45C55007B
:10B8E00024026D186C805B1C1B061B0EC65C344367
:10B8F0006C805B1C1B061B0E521E12061216002AC1
:10B90000ECDA0E230522C55C541E24062E092416EB
:10B91000521896732A07120F0D19AA735B1C1B0687
:10B920001B0E641E22061216002AECDC427C0A75ED
:10B9300012230522C45C550024026D18EC825B1CA6
:10B940001B061B0EC65C3443EC825B1C1B061B0EE5
:10B95000521E12061216002AECDA70BC0120704743
:10B9600070BC00207047F0B593B005006D484021D1
:10B9700001F0EAFA06200A906B480B90012708A80C
:10B98000077400241194AC6540200090654B02229E
:10B9900028000AA9FBF719F90600AF65002E04D0AC
:10B9A000300013B0F0BC08BC18475E4801A9FFF78F
:10B9B0008AFF68468088002804D06846007E0128F7
:10B9C00005D008E013B0F0BC08BC01201847684659
:10B9D000408B022809D06846C0885449884258D113
:10B9E0006846807C012805D053E013B0F0BC08BC49
:10B9F000012018474B48402101F0A6FA0194029417
:10BA00000394049405940694079408940994484870
:10BA10000B90AC6540200090424B022228000AA9FE
:10BA2000FBF7D3F80600AF65002E04D0300013B04A
:10BA3000F0BC08BC18473B4801A9FFF744FF684623
:10BA40008088002803D06846807C012804D013B089
:10BA5000F0BC08BC012018476846007E012803D1CD
:10BA60006846408B022819D02868324A8100324843
:10BA70004058416803239B039943114341607D2053
:10BA8000C000FDF75FF85F20475501212800FBF754
:10BA900090FA300013B0F0BC08BC184713B0F0BCEB
:10BAA00008BC0120184710B584B0040000210091A3
:10BAB00001910291039120006946FFF7D9FE002809
:10BAC00003D16946097A6034217004B010BC08BC07
:10BAD000184730B589B0040001206946087200207B
:10BAE0000790372000906089000401902000FBF748
:10BAF000D0FB00280BD106200090022001902000EE
:10BB00006946FBF7C6FB0500002D19D0280009B0D7
:10BB100030BC13E00080FF00AA01000050C3000009
:10BB20001066022A5066022A01FFFF00038000000F
:10BB300001FFFF8000800000F065022A08BC184762
:10BB400020680121FDF7D1F9280009B030BC08BCFC
:10BB500018470120704730B5002829D0002927D088
:10BB60000268120ECA8702680C001202120C4034DE
:10BB700022800268A270436804228D184035AB70A1
:10BB80001B0A521E002AF8DC0022E2718268120EA3
:10BB900062728268C36812021B0E1A43CA64C068CC
:10BBA0000003000DFFF7D5FF30BC08BC012018478B
:10BBB00030BC08BC00201847F7B5C8B0844696468C
:10BBC0000025704600287EDD4998A9010B18002049
:10BBD0008100CE18B778F47872783F023C435F5CFE
:10BBE000160408AA3F063E4334435450401C102814
:10BBF000EEDB10211400881E80002058112306005F
:10BC0000DE4113270300FB415E40800A46400800E6
:10BC10000F388000235807201F00C7411800122248
:10BC2000D0414740D8084740C81FF3198000265824
:10BC30000800103880002058301818188A00A050CA
:10BC4000491C4029D7DB00206A4681006346CB1897
:10BC500080339B685350401C0828F6DB0020049971
:10BC60000623D941049B0B24E3415940049B19242A
:10BC7000E341594004AB18CB049E2340069CB443D7
:10BC80006340CC18FF4B81005B58079EF318E31804
:10BC900008AC61585918009B0224E341009C0D2612
:10BCA000F4416340009C1626F44163406C4650CC3E
:10BCB000029F3440009E3E407440019E3E407440CE
:10BCC0001B19069C00E022E00794059C0694049C46
:10BCD0000594039C64180494029C0394019C0294B0
:10BCE000009C0194C9180091401C4028B7DB00203B
:10BCF0008300614659188031D3588C68E3188B60F3
:10BD0000401C0828F4DB6D1C754500DA5CE74BB07D
:10BD1000F0BC08BC1847F0B583B004000D006068A3
:10BD200001218206920E372A00D80021491C019178
:10BD300021680918CE0001998F01210008313A1AB3
:10BD400040180291110001F0FFF86268029980200A
:10BD50005054E019C671310A8171310C4171310EB4
:10BD60000171019A02992000FFF726FF002290003E
:10BD7000031980339E684119CE709E68360A8E7012
:10BD80009E68360C4E709968090E2954521C082A78
:10BD9000EDDB03B0F0BC08BC1847F7B50400150094
:10BDA00082B061684020401A2E00854200D3060010
:10BDB00020000830019008180399320001F01AF8A9
:10BDC00060684019402804D2606005B0F0BC08BC2F
:10BDD0001847AF1BBD09039886190199012220005D
:10BDE000FFF7EAFE2A0031002000FFF7E5FEBF065C
:10BDF000BF0EA801811901983A0000F0FBFF6760AF
:10BE000020686D1CA9014018206005B0F0BC08BC7A
:10BE1000184710B400219C4B8A009C58121880329D
:10BE20009460491C0829F7DB00214160016010BCC7
:10BE3000704770B5AAB004000D0016006846FFF701
:10BE4000E8FF2A0021006846FFF7A7FF3100684697
:10BE5000FFF761FF2AB070BC08BC1847F7B5FFB008
:10BE6000D5B000208646D69800287EDD7046C101F8
:10BE7000D5980C180021CA0010198379C6790025BD
:10BE80001F0E1B021E4343792D023D43B44600277B
:10BE90001E0C3F04374366462F43BC4607791B04FC
:10BEA0001E4300233D0A1B062B4365461D43C378F2
:10BEB0003F063E431D43837840781B021D43000428
:10BEC0000543A05C0006054314A88218166055605F
:10BED000491C1029CFDB10218C466046801EC20011
:10BEE00014A8811803C914ACA4584B03C50C1D43F6
:10BEF000CB0C6403234314AC1219460FCC0034431B
:10BF00005268C600520F324355408A0680091043DA
:10BF1000454060460F3863408909C2004B4014A871
:10BF2000811803C914AFBA58CE0744083443CD92E0
:10BF30004E08D2071643CC960A06060A1643CD9A37
:10BF4000D3941206CB923200CB9E0C0A3443CA948F
:10BF5000D39CCA9F54404A06CC9EC0097E401043E1
:10BF6000C90944404E40281900E017E17341614679
:10BF7000C91FCA0014A989186246103AD50014AA2C
:10BF800052190C6860CA49686419714104194B411F
:10BF90006046C10014A84018046043606046401C1D
:10BFA00084466046502898DB0020D49AC1008A1845
:10BFB000FF320132946804ABD26859180C604A60B1
:10BFC000401C0828F1DB002084460CA803C8850B20
:10BFD0008A0415430C9A8B0B920413438C03820C36
:10BFE00022430C9C8E0CA70355400D9A3E43734090
:10BFF000560A440ACA052243C40553400F9A2643F1
:10C0000075400E9EC992170002003240C896CC437C
:10C010000E00C792119A3E40C696CE94109EC592CD
:10C020002240C743C3923740C79AC4967A40AF189C
:10C03000C69EC39C139A129D6640D092734162467D
:10C04000124CD200C292A218CF97C0CAD09AAD1992
:10C050007A41CF9F14AC7D195341C29AA41814CCD5
:10C06000AD18634102950393059A049E1401170FBE
:10C07000C192049A330F12011743059A234395087E
:10C08000C09605E0B0F4002A10F4002AB0F5002AAA
:10C09000C19AB40892072243B40725435740059A32
:10C0A0006B40D509C09EC19ABF93F30952061A434B
:10C0B00073061D435740BF9BC19A6B40D19206AA9D
:10C0C000D2930CCABCAC0CC4D19C16401C40BAAA7A
:10C0D00050C208AC30CCC19AC09E2A402640130002
:10C0E000B8AAB79630C2BAAC50CCB79A5C405640AA
:10C0F000B5AA50C2BC9EB89CBD9B26402B40B5AC97
:10C1000030CC5C40D29B75405E1967416A46C0C224
:10C11000C4AB48CB12AA48C2C8AEC0CE10AAC0C297
:10C120000EAA03C2029D0A99039B0B984919584114
:10C130000C910D90B8AC30CC0AA830C0BCAA0CCA87
:10C1400008A80CC0C0AA44CA06A844C06E46C0CE07
:10C15000029D039BA8197B4104A909C16046401CAC
:10C1600084466046502800DA2FE7002004AED499B8
:10C17000C3005918FF310131F4188D6818CCCA6812
:10C18000EB1862418B60CA60401C0828EFDB7046E8
:10C19000401C8646D6998E4500DA67E67FB058B0D7
:10C1A000F0BC08BC1847F0B583B004000D0060680F
:10C1B00001214206520E6F2A00D80021491C01912C
:10C1C00021680918CE000199CF01210008313A1ADF
:10C1D00040180291110000F0B7FE626802998020B9
:10C1E0005054E019C671310A8171310C4171310E20
:10C1F0000171019A02992000FFF730FE0020C10072
:10C200000A19FF32013296684B19DE71D7689668B9
:10C210003F06360A3E439E71D76896683F04360C47
:10C220003E435E71D76896683F02360E3E431E71EC
:10C23000D668DE70D668360A9E70D668360C5E7098
:10C24000D268120E6A54401C0828D8DB03B0F0BC38
:10C2500008BC1847F7B50400150082B0616880205B
:10C26000401A2E00854200D30600200008300190BD
:10C2700008180399320000F0BDFD6068401980285D
:10C2800004D2606005B0F0BC08BC1847AF1BFD09C4
:10C2900003988619019901222000FFF7DFFD2A008B
:10C2A00031002000FFF7DAFD7F067F0EE8018119DB
:10C2B00001983A0000F09EFD676020686D1CE9015E
:10C2C0004018206005B0F0BC08BC184730B400210D
:10C2D000C24CCA00A31812181D68FF325B680132F5
:10C2E0009560D360491C0829F3DB0021416001609F
:10C2F00030BC704770B5D2B004000D00160068461F
:10C30000FFF7E4FF2A0021006846FFF7A3FF310092
:10C310006846FFF748FF52B070BC08BC1847F0B53C
:10C3200083B004000D00606801214206520E6F2A9E
:10C3300000D80021491C019121680918CE000199FB
:10C34000CF01210008313A1A40180291110000F083
:10C35000FBFD6268029980205054E019C671310AD1
:10C360008171310C4171310E0171019A02992000E5
:10C37000FFF774FD0020C1000A19FF3201329668F0
:10C380004B19DE71D76896683F06360A3E439E71A8
:10C39000D76896683F04360C3E435E71D76896684E
:10C3A0003F02360E3E431E71D668DE70D668360AEE
:10C3B0009E70D668360C5E70D268120E6A54401CAD
:10C3C0000628D8DB03B0F0BC08BC1847F7B504005A
:10C3D000150082B061688020401A2E00854200D38B
:10C3E000060020000830019008180399320000F080
:10C3F00001FD60684019802804D2606005B0F0BC7F
:10C4000008BC1847AF1BFD09039886190199012242
:10C410002000FFF723FD2A0031002000FFF71EFD5A
:10C420007F067F0EE801811901983A0000F0E2FCD6
:10C43000676020686D1CE9014018206005B0F0BC01
:10C4400008BC184730B40021654CCA00A318121864
:10C450001D68FF325B6801329560D360491C082972
:10C46000F3DB00214160016030BC704770B5D2B091
:10C4700004000D0016006846FFF7E4FF2A002100C3
:10C480006846FFF7A3FF31006846FFF748FF52B048
:10C4900070BC08BC1847F0B583B004000D0060689C
:10C4A00001218206920E372A00D80021491C0191F1
:10C4B00021680918CE0001998F01210008313A1A2C
:10C4C00040180291110000F03FFD6268029980203F
:10C4D0005054E019C671310A8171310C4171310E2D
:10C4E0000171019A02992000FFF766FB002290007B
:10C4F000031980339E684119CE709E68360A8E708B
:10C500009E68360C4E709968090E2954521C072AF1
:10C51000EDDB03B0F0BC08BC1847F7B5040015000C
:10C5200082B061684020401A2E00854200D3060088
:10C5300020000830019008180399320000F05AFCDE
:10C5400060684019402804D2606005B0F0BC08BCA7
:10C550001847AF1BBD0903988619019901222000D5
:10C56000FFF72AFB2A0031002000FFF725FBBF065A
:10C57000BF0EA801811901983A0000F03BFC6760EA
:10C5800020686D1CA9014018206005B0F0BC08BCF3
:10C59000184710B40021134B8A009C58121880329F
:10C5A0009460491C0829F7DB00214160016010BC40
:10C5B000704770B5AAB004000D0016006846FFF77A
:10C5C000E8FF2A0021006846FFF7A7FF3100684610
:10C5D000FFF761FF2AB070BC08BC184770F4002A4E
:10C5E00030F4002AF0F3002A10B4002920D08A8900
:10C5F0008B88012B01D19B021A434B89012B01D15E
:10C6000040231A430B89012B01D180231A434B8805
:10C61000012B01D1DB021A430B88012B01D11B0333
:10C620001A430B695E4980000C58A3600858C26029
:10C6300010BC70470A8812018B78002B01D00823A8
:10C640001A430B79012B01D102231A43CB78002B1B
:10C6500001D004231A434979002901D001210A435A
:10C660004F4980000858C26270474D498000085801
:10C67000C06B7047052916D20A007A4412799218C5
:10C680009744020406080A00464906E0464904E0C9
:10C69000082102E0454900E04549820040488058B1
:10C6A000C26B0A43C263704705291AD20A007A4452
:10C6B000127992189744020406080A00394906E0E4
:10C6C000394904E0082102E0384900E03849344A99
:10C6D00080001058C26B0A4001208A4200D000201E
:10C6E00070470020704710B4052918D20B007B4416
:10C6F0001B79DB189F44020406080A00294906E05A
:10C70000294904E0082102E0284900E02849244C96
:10C710008300E058C06B88431060E158C86310BCC8
:10C7200070471F4A80001058C06B086070471C4A51
:10C7300080001058C163704770B50D00140083006D
:10C740001C48C15880311648C25801233432DB03DB
:10C75000280000F061FF2168401B081A206070BCAF
:10C7600008BC184730B50D00140085B08200114890
:10C77000805880300A498958343100910E4901911E
:10C78000216802911A21039129006A4600F048FFAE
:10C790002168401B081A206005B030BC08BC18474F
:10C7A000F065022A00000002000080000000800204
:10C7B000000100000066022A00400000032000057E
:10C7C0000168A64A114001229203114301600168E9
:10C7D000A34A1140016070477047704710B40320AE
:10C7E000000503689F4C89072340090F0B43036032
:10C7F00001689D4B92071940920E1143016010BCD5
:10C8000070470320000501290AD0032908D0042914
:10C8100005D10168914A114080221143016070479F
:10C820000168924A1140016070470839072908D809
:10C830000322120510688E4B49071840490D084322
:10C840001060704710B4FF238A48403306294CD249
:10C850000C007C4424792419A7444702101E2C3A6A
:10C86000002A05D0016A02241940214301623CE0FC
:10C87000016AFF243E342140016236E0002A05D0DF
:10C88000016A04241940214301622EE0016AFF2459
:10C890003C342140016228E0002A05D0016A0824C6
:10C8A00019402143016220E0016AFF24383421400D
:10C8B00001621AE0002A05D0016A102419402143C0
:10C8C000016212E0016AFF243034214001620CE071
:10C8D000002A05D0016A202419402143016204E0A6
:10C8E000016AFF24203421400162002A04D0016A39
:10C8F000012219401143016210BC7047032000055A
:10C90000062A0ED213007B441B79DB189F44020ACF
:10C91000121A222A8268584B49071A40490F0A43C3
:10C92000826070478268554B49071A40890E0A4356
:10C93000826070478268524B49071A40C90D0A430A
:10C940008260704782684F4B49071A40090D0A43BD
:10C950008260704782684C4B49071A40490C0A4371
:10C9600082607047826849075204520C890B0A435F
:10C9700082607047092907D803208900000508183C
:10C98000016AD106C90E01627047042A0DD200293E
:10C990000BDD491E88008018132806D88100354811
:10C9A0000818416A5904490C41627047002B0FD0A6
:10C9B000042A0DD200290BDD491E88008018132897
:10C9C00006D82C4980004018406A4004400C18608A
:10C9D000704703221205D0680843D168D0607047C1
:10C9E00003221205D0688843D168D06070470320C5
:10C9F000000500698006800EC20706D0002902D01B
:10CA00008006C00E0860012070470020704710B4F7
:10CA10000320124B0005002906D0016801241940AB
:10CA2000A4032143016003E00168184C2140016028
:10CA3000002A05D00168164A1140016010BC7047F9
:10CA4000016801221940D2031143016010BC7047F4
:10CA5000002901D00F48086070470000BFF70F00A1
:10CA6000BFD70F00B3F70F008FF70F003FF70F008E
:10CA7000BFF00F0080003000F8FF0300C7FF030085
:10CA80003FFE0300FFF10300FF8F0300BFB70F005D
:10CA9000BF770F00B0EB002A704770477047032044
:10CAA000000500680006C00F002801D00420704770
:10CAB000032070470320000500684005400F083040
:10CAC0007047F8B50D0064240521090548685D4FDD
:10CAD00038405D4E0AE03168002903D0012000F0A3
:10CAE000EAFD641E05200005406838400101890FF9
:10CAF00001D1002CEFDC002C03DCF8BC08BC0120C9
:10CB00001847010103D4F8BC08BC01201847002DC8
:10CB100000D02870F8BC08BC00201847F8B50E00FB
:10CB200017001D000024C0680090002D0DD013D9FF
:10CB3000305D395D000208434449086000980021D7
:10CB4000FFF7BFFF002807D103E02000F8BC08BCB6
:10CB50001847641CAC42EBD32000F8BC08BC184753
:10CB6000F8B50E0017001D000024C0680090002DCD
:10CB70000ED014D9305D0102012000060918334897
:10CB8000016000983919FFF79CFF002807D103E0E6
:10CB90002000F8BC08BC1847641CAC42EAD3200053
:10CBA000F8BC08BC1847F8B50E0017001D0000249B
:10CBB000C0680090002D0FD015D96000305A395D43
:10CBC0004004400A08432149086000980021FFF70B
:10CBD00078FF002807D103E02000F8BC08BC184704
:10CBE000641CAC42E9D32000F8BC08BC1847F8B577
:10CBF0000E0017001D000024C0680090002D10D00A
:10CC000016D96000305A4004410A01200006091874
:10CC10000E48016000983919FFF753FF002807D12B
:10CC200003E02000F8BC08BC1847641CAC42E8D301
:10CC30002000F8BC08BC1847002901D0044808604F
:10CC400070470000FFFF7F0FBCF3002A0000500078
:10CC500020EC002A0FB41CB50C0007AA009001D0EC
:10CC60000019401E084B7B4469460190069800F06D
:10CC700030FB002C03D06946002000F03DFB1CBCBB
:10CC800008BC04B01847000099060000F8B504007D
:10CC90000E00002030E0E168200000F00CFD0028CC
:10CCA0002CD0252802D06268A16821E0E168002725
:10CCB000200000F000FD050020D028004138192890
:10CCC00002D80127FF02203532002900200027600A
:10CCD000F3F7D0F9002808D0012804D0F61DF60893
:10CCE000F6000836D7E7361DD5E76268A168280048
:10CCF00000F0E2FC206A401C2062CCE7206AF8BC0D
:10CD000008BC184701C08FE21CFF2FE1F7B50026D1
:10CD100075291068009915A511D0C046C046002895
:10CD200002DA404212A508E0009909688A0701D595
:10CD300010A502E0490704D50FA5012601E0C04671
:10CD4000C046009F0024243704E000F0E3FA3031AD
:10CD50003955641C0028F8D1009833002A002100BE
:10CD600000F056FAFEBC08BC1847000000000000A6
:10CD70002D0000002B0000002000000003000B43EA
:10CD800010B49B071DD1042A1BD308C810C9121F59
:10CD9000A342F8D018062106000E090E401A0ED143
:10CDA00018042104000C090C401A08D118022102B1
:10CDB000000A090A401A02D1180E210E401A10BCAE
:10CDC0007047002A03D0D30703D0521C07E000208D
:10CDD000F5E703780C78401C491C1B1B07D103782E
:10CDE0000C78401C491C1B1B01D1921EF1D118006C
:10CDF000E5E700007847C046030052E32A00009AA6
:10CE000003C010E20800000A0130D1E402005CE334
:10CE10000C2082E001C0D1940130C0E40130D13453
:10CE200001C0C094042042E20130C034033011E25A
:10CE30002600000A042052E21B00003A03C031E73A
:10CE4000020053E30800000A0F00008A2C34A0E11E
:10CE500004C0B1E5042052E20C3C83E1043080E4DC
:10CE6000F9FFFF2A011081E20F0000EA2C38A0E14F
:10CE700004C0B1E5042052E20C3883E1043080E4C0
:10CE8000F9FFFF2A021081E2070000EA2C3CA0E132
:10CE900004C0B1E5042052E20C3483E1043080E4A4
:10CEA000F9FFFF2A031081E20000A0E1822FB0E128
:10CEB0000130D12401C0D1240120D1440130C0244B
:10CEC00001C0C0240120C0441EFF2FE17847C046A6
:10CED00010402DE9202052E20500003A1850B1E838
:10CEE000202052E21850A0E81850B1E81850A0E8ED
:10CEF000F9FFFF2A02CEB0E11850B1281850A0283F
:10CF00001800B1481800A0481040BDE802CFB0E1B9
:10CF100004309124043080241EFF2F01822FB0E1C1
:10CF2000B230D1200120D144B230C0200120C04411
:10CF30001EFF2FE17847C046FF3002E2032483E161
:10CF4000022882E1010000EA7847C0460020A0E301
:10CF5000040051E30700003A03C010E20C00000A8D
:10CF600004C06CE202005CE30120C0140C1041E03C
:10CF7000B220C0A0060000EA81CFB0E10120C024A9
:10CF80000120C0240120C0441EFF2FE17847C04685
:10CF90000020A0E300402DE90230A0E102C0A0E1A2
:10CFA00002E0A0E1201051E20C50A0280C50A02873
:10CFB00020105122FBFFFF2A011EB0E10C50A028D7
:10CFC0000C00A0480040BDE80111B0E1042080241D
:10CFD0001EFF2F01B220C040010111E30120C01447
:10CFE0001EFF2FE1013090E14C00004AA03071E0BB
:10CFF0004400003A0020B0E3203271E03400003AEF
:10D00000203471E02600003A203671E01700003A23
:10D01000203871E00900003A0114A0E1203871E0E5
:10D02000FF2482E3FF2882230114A021203671E02F
:10D030000E00003A003071E26F00002A2114A02196
:10D04000A03771E0810740200220B2E0203771E074
:10D05000010740200220B2E0A03671E081064020A6
:10D060000220B2E0203671E0010640200220B2E04A
:10D07000A03571E0810540200220B2E0203571E04A
:10D08000010540200220B2E0A03471E0810440207C
:10D090000220B2E0203471E0010440200220B2E01E
:10D0A000E5FFFF2AA03371E0810340200220B2E0B7
:10D0B000203371E0010340200220B2E0A03271E091
:10D0C000810240200220B2E0203271E001024020C3
:10D0D0000220B2E0A03171E0810140200220B2E0E4
:10D0E000203171E0010140200220B2E0A03071E067
:10D0F000810040200220B2E0011050E00010A03179
:10D100000200A2E01EFF2FE1011050E00100A02369
:10D110001EFF2F210010A0E10000B0E31EFF2FE151
:10D12000022111E20010614240C032E000006022A2
:10D13000203271E01D00003A203471E00F00003A07
:10D140000113A0E1203471E03F2382E30B00003A99
:10D150000113A0E1203471E03F2682E30700003A8A
:10D160000113A0E1203471E03F2982E30113A021E3
:10D170003F2C8223003071E21D00002A2113A021E0
:10D18000A03371E0810340200220B2E0203371E03F
:10D19000010340200220B2E0A03271E08102402071
:10D1A0000220B2E0203271E0010240200220B2E011
:10D1B000A03171E0810140200220B2E0203171E015
:10D1C000010140200220B2E0EBFFFF2AA03071E015
:10D1D000810040200220B2E0011050E00010A03198
:10D1E0000200A2E0CCCFB0E100006042001061225A
:10D1F0001EFF2FE1CCCFB0E10000604201402DE9DD
:10D200000000B0E30000A0E10240BDE81EFF2FE1F6
:10D21000FFB5040081B024300D000090216888061D
:10D2200004D51022E0699143216000E0012000272D
:10D23000A84200DD471B0498A1697A191018081A42
:10D24000A0612068C00602D42000C046C046002667
:10D2500009E00398A1686268805D00F02DFA206AF9
:10D26000401C761C206204988642F2DB2068C006CF
:10D270000BD52000C046C04607E06268A168302098
:10D2800000F01AFA206A401C206238007F1E002835
:10D29000F3DC08E00098A1686268405D00F00CFAD9
:10D2A000206A401C206228006D1E0028F2DC20004D
:10D2B000C046C04621680220090600D4012005B0FE
:10D2C000F0BC08BC1847000001694A1C02610878DC
:10D2D000704700B58FB00291002105910549019377
:10D2E00079440391110004906846FFF7CFFC0FB01A
:10D2F00008BC1847E5FFFFFF0A681070521C0A605F
:10D3000070474B680A689A4202D2531C0B60107037
:10D31000704700007847C0460A1040E2200140E014
:10D32000200280E0200480E0200880E0A001A0E14D
:10D33000002180E0821051E0010080520A108142F9
:10D340001EFF2FE17847C0460020B0E3203171E096
:10D3500065FFFF3AA03271E05AFFFF3A203471E0D6
:10D360004FFFFF3A203671E040FFFF3A203871E06E
:10D3700032FFFF3A27FFFFEA000000000000000034
:10D380000B10A0E3910000E0A002A0E1010050E238
:10D39000FDFFFFCA1EFF2FE1D3F021E328D09FE558
:10D3A00028009FE5100F01EE100F11EE010A80E337
:10D3B000100F01EE18209FE50000A0E3000082E5B9
:10D3C00010D09FE510009FE510FF2FE10000042A18
:10D3D00078000500B8F2002A3038012A2503002A17
:10D3E00034109FE52A04A0E3000081E530109FE59A
:10D3F00030009FE5000081E52C009FE5000081E5FD
:10D4000028009FE5000081E524009FE5000081E5FC
:10D4100020009FE5000081E5FEFFFFEA0400010215
:10D420000000002A04800802090100000101000038
:10D43000210100002000000080000000C0D09FE516
:10D44000C0009FE5C0E09FE510FF2FE1BC109FE505
:10D450000000A0E3000081E5B4109FE50000A0E318
:10D46000000081E5AC109FE50000A0E3000081E52D
:10D47000A4109FE50000A0E3000081E5691AA0E385
:10D480000000A0E3000081E590109FE50000A0E30C
:10D49000000081E588009FE588E09FE510FF2FE10F
:10D4A00084109FE5810CA0E3000081E578109FE5E2
:10D4B00078009FE5000081E5090000EB68109FE51A
:10D4C000160CA0E3000081E5050000EB58109FE575
:10D4D000020CA0E3000081E5010000EB1F0000EA60
:10D4E0000097FF0F3D0AA0E3900080E300A0A0E1B9
:10D4F00001A04AE200005AE3FCFFFF1A0EF0A0E18F
:10D5000090D003003038012AF739002A4CD4002A81
:10D5100000404001005040010440400104504001DF
:10D5200004900600793F002AA0D4002A14100102BA
:10D53000E0D4002A0000000000000000000000000D
:10D54000A8009FE5A8109FE50140A0E30020A0E30C
:10D55000010050E104208034FCFFFF3AB6FFFFEAEF
:10D5600090109FE590009FE5002090E58C309FE5AE
:10D57000030051E10400000A000091E5000082E58B
:10D58000041081E2042082E2F8FFFFEA70009FE5C8
:10D59000001090E56C209FE50830A0E3000092E5C4
:10D5A000000081E5041081E2042082E2013053E2B0
:10D5B000F9FFFF1A40109FE5000091E510FF2FE1F1
:10D5C000FEFFFFEAFDFFFFEA4CF09FE54CF09FE510
:10D5D0004CF09FE54CF09FE54CF09FE54CF09FE54B
:10D5E0004CF09FE54CF09FE500E002000000002AAF
:10D5F00030F8002A9066022AE0D3002AE8D5002AF3
:10D600003CD4002AECD5002AC8D5002A000000002E
:10D610007847C04659FFFFEA7847C046080000EA4D
:10D620007847C0460E0000EAF00F2DE9F00FB1E890
:10D63000F00FA0E8F00FBDE81EFF2FE1042091E4F9
:10D64000042080E4F00F2DE9F00F91E8F00FA0E83E
:10D65000005092E5055013E0FAFFFF1AF00FBDE805
:10D660001EFF2FE1F05F2DE908C092E5043092E53E
:10D6700000E092E5F00FB1E8F00F80E820C04CE246
:10D6800020005CE3060000BA00509EE50C6092E5C5
:10D69000066015E00200001A035015E0F9FFFF0ACA
:10D6A000F3FFFFEA08C082E5F05FBDE80100A0E1FA
:10D6B0001EFF2FE100470847104728473847000062
:10D6C0007847C04614309FE5931082E01830A0E3FD
:10D6D000013B43E22213A0E1930120E01EFF2FE172
:10D6E000D34D62107847C046030031E110402DE968
:10D6F000023123422001004A024050E003C0D1E041
:10D700000300002A042092E00C30A3E0040050E063
:10D710000C10C1E01CE19FE5214AA0E123CA44E0CE
:10D7200083001EE1840A3E113700000A0E30C3E177
:10D7300020E07CE2041AC1E1013683E31400003AE0
:10D74000320C90E0331CA1E0130E90E00010B1E227
:10D75000010651E31800002A041A81E0122EB0E1FC
:10D760001040BDE81EFF2F51010090E28220B03131
:10D770001EFF2F11000050E30100C0130010A10292
:10D780008130A0E1020673E31EFF2F31061241E251
:10D79000F10000EA010052E30320A3E020C04CE2C4
:10D7A0001FE07CE200E0A033330C9020041AA1E0DB
:10D7B000210A54E1E8FFFF0A041A41E0011681E260
:10D7C000A110B0E16000B0E1041A81E00800003A65
:10D7D0000000B0E212EEB0310500001A1040BDE8C2
:10D7E000E3FFFFEA010090E28220B031E3FFFF1A7D
:10D7F000DFFFFFEA1040BDE88130A0E1020673E3DD
:10D800001EFF2F31061241E2D30000EA840A3EE1F6
:10D810000400000AAE0011E11040BDE80000A003C2
:10D82000021101021EFF2FE11040BDE870402DE9FA
:10D83000990000EB64FBBE3E0000E0FF7847C04665
:10D84000213AA0E1013B43E21E3073E220C073A203
:10D85000040000BA0221A0E3812582E1A02A92E11E
:10D860003203B0E11EFF2FE1010011E10700004A81
:10D87000100053E30000A0C31EFF2FC13ECE83E281
:10D8800001007CE30300000A0000E0E31EFF2FE13B
:10D890000000A0E31EFF2FE170402DE97E0000EBA9
:10D8A000922449800000A0E31EFF2FE1F5FFFFEA6C
:10D8B000023110E2001060120010A001013183E378
:10D8C0002108B0E1013483120118B0011EFF2F01BD
:10D8D000FF0411E3023583120114A0010F0211E3CA
:10D8E000013583120112A001030111E302368312F4
:10D8F0000111B001013683428110A051810AA0E1DB
:10D90000C11583E01EFF2FE17847C0460131A0E337
:10D910000010A0E1E9FFFFEA7847C0466CC19FE52F
:10D9200070402DE921E21CE023521C100C003E1136
:10D930000C0035113D00000A034021E08C32C3E1A8
:10D94000A4EF8EE18C12C1E1011681E3013683E37D
:10D9500005E08EE091428CE0906385E0FFE74EE2C7
:10D96000046096E00C50B5E091438CE00030ACE2EE
:10D9700090128CE00C6096E00450B5E00030B3E209
:10D98000010011E101608613020C13E30600001A86
:10D990000316A0E10506A0E10646B0E1251A81E1E3
:10D9A000260A80E10320E0E3050000EA8315A0E1F8
:10D9B0008505A0E18645B0E1A51A81E1A60A80E1CE
:10D9C0000220E0E34E2882E0025A81E08E1F25E02B
:10D9D0000400000A84C0B0E10241C4130000B0E2B8
:10D9E0000010A1E2A40FC0E1A4C09FE50C0052E129
:10D9F0000100002A7040BDE81EFF2FE1050050E144
:10DA00000141A0130341A003000056E30040A0031E
:10DA100001035EE37040BDE8061241A24E0000AA79
:10DA20000000A0E3061281E2021101E21EFF2FE1D5
:10DA30000C003EE123520CE00C0035110400000AFA
:10DA40000000A0E303E021E002110EE27040BDE817
:10DA50001EFF2FE1100000EB8900013E030000EAE9
:10DA6000040000EA83C0A0E1ACCAB0E10400000AEF
:10DA7000031021E0380000EA81C0A0E1ACCAB0E1A7
:10DA8000FAFFFF1A0000A0E308109FE51EFF2FE138
:10DA90000000FF07FE0700000000F87F04609EE41E
:10DAA000060016E10300004A010052E30350A3E020
:10DAB000020675E30A00008A010050E301C0A1E0FC
:10DAC00002067CE30600008A0700001AA1CFA0E14D
:10DAD000020675E38CC08CE002C08CE2A3CFAC00E0
:10DAE000020000EA08C0A0E3000000EAA3CFA0E122
:10DAF0008C508CE03665A0E1076006E204C056E277
:10DB00000200002A06C18EE07040BDE81CFF2FE134
:10DB10000CF18FE00000A0E1060000EA070000EA37
:10DB2000FFFFFFEA7040BDE80000A0E30211A0E3A0
:10DB3000021741E21EFF2FE10310A0E10200A0E165
:10DB4000010050E30140B1E0024674127040BDE8AC
:10DB50000000A083021101821EFF2FE12100B0E12D
:10DB6000021640E26110A0E11EFF2FE1030031E147
:10DB700010402DE902312342DEFEFF4A024050E010
:10DB800003C0D1E00400002A042092E002C12CE28C
:10DB90000C30A3E0040050E00C10C1E008E29FE567
:10DBA000214AA0E123CA44E083001EE1840A3E1119
:10DBB0006F00000A002072E2CE30C3E1CE30E3E015
:10DBC00020E07CE2041AC1E10F00003A320C90E040
:10DBD000531CA1E0130E90E00010B1E21400004AC3
:10DBE000122EB0E1041A81E01040BDE81EFF2F5153
:10DBF000010090E2020152131EFF2F11000050E3BA
:10DC0000011081020100C0131EFF2FE102E092E02B
:10DC10000320A3E001E0A01320C04CE282208EE1AB
:10DC20001EE07CE24000009A530C90E00010D1E22C
:10DC3000EAFFFF5A01E08EE212EEB0E10000B0E030
:10DC40000110A1E084CA81E0ACCAB0E10800009AEA
:10DC5000AE0F90E002015E33041A81E01040BDE88F
:10DC60001EFF2F11000050E3011081020100C013BC
:10DC70001EFF2FE12F00002A021691E20000500340
:10DC80001040BD081EFF2F01A4C5A0E1024BC4E354
:10DC9000010011E1024044E20600001A0010A0E178
:10DCA000010850E3104044E22118A0210008A021FF
:10DCB0000000A0331040443200E0A0E3200051E314
:10DCC0000118A03110E08E32020A51E30114A03194
:10DCD00008E08E32020851E30112A03104E08E32D6
:10DCE000020751E30111A03102E08E32010651E337
:10DCF00001E08E3220206EE28110A031301281E1ED
:10DD0000100EA0E10E4044E08C1F81E0000054E3BF
:10DD1000041A81E01040BDE81EFF2FA10000A0E31F
:10DD2000061281E2021101E21EFF2FE1041A81E0D6
:10DD30001040BDE81EFF2FE1C110B0E1041A81E0E0
:10DD40001040BDE86000A0E1010000EA0010A0E37F
:10DD50001EFF2FE18120B0E100001001FAFFFF0A51
:10DD6000020652E31EFF2F210000A0E3021101E290
:10DD70001EFF2FE1840A3EE10400000AAE0011E11B
:10DD80001040BDE80010A0030000A0031EFF2FE11B
:10DD90001040BDE870402DE93FFFFFEB40DFF63E4D
:10DDA000021123E20200A0E11EFF2FE10000E0FFCC
:10DDB00000000000C7B9302049CA51208E736100AD
:10DDC000552D93209294A3001CE7C200DB5EF22045
:10DDD0006DE31621AA5A260124294701E3907721F1
:10DDE00038CE8501FF77B5217104D421B6BDE40199
:10DDF0001D7F1D22DAC62D0254B54C02930C7C22E5
:10DE000048528E028FEBBE220198DF22C621EF021C
:10DE1000709C0B03B7253B2339565A23FEEF6A0348
:10DE200025B19823E208A8036C7BC903ABC2F92390
:10DE3000FD470A243AFE3A04B48D5B0473346B2424
:10DE4000A86A99046FD3A924E1A0C8242619F8046C
:10DE500090A41C05571D2C25D96E4D251ED77D0578
:10DE6000C5898F250230BF058C43DE054BFAEE25B0
:10DE7000E038170627812726A9F246266E4B76063C
:10DE8000B515842672ACB406FCDFD5063B66E526E4
:10DE90008DDB01274A623107C411500703A86027B0
:10DEA000D8F692071F4FA227913CC3275685F30748
:10DEB0003D362428FA8F140874FC7508B3454528AC
:10DEC000681BB708AFA2872821D1E628E668D608E4
:10DED00050D53209976C0229191F6329DEA6530910
:10DEE00005F8A129C24191094C32F0098B8BC02958
:10DEF0002049390AE7F0092A6983682AAE3A580AA4
:10DF00007564AA2AB2DD9A0A3CAEFB0AFB17CB2A3B
:10DF10004DAA2F2B8A131F0B04607E0BC3D94E2BE7
:10DF20001887BC0BDF3E8C2B514DED2B96F4DD0B8F
:10DF3000C0712E0C07C81E2C89BB7F2C4E024F0CC3
:10DF4000955CBD2C52E58D0CDC96EC0C1B2FDC2C6B
:10DF5000AD92382D6A2B080DE458690D23E1592D37
:10DF6000F8BFAB0D3F069B2DB175FA2D76CCCA0DCF
:10DF7000DD0E332E1AB7030E94C4620E537D522E5B
:10DF80008823A00E4F9A902EC1E9F12E0650C10EA3
:10DF9000B0ED250F7754152FF927742F3E9E440FAF
:10DFA000E5C0B62F2279860FAC0AE70F6BB3D72FE7
:10DFB000BDD578307A6C4810F41F291033A619307B
:10DFC000E8F8EB102F41DB30A132BA30668B8A10B3
:10DFD000D0366E11178F5E3199FC3F315E450F11BF
:10DFE000851BFD3142A2CD11CCD1AC110B689C3107
:10DFF000A0AA651267135532E96034322ED9041293
:10E00000F587F632323EC612BC4DA7127BF497322A
:10E01000CD4973330AF0431384832213433A1233F6
:10E020009864E0135FDDD033D1AEB133161781139E
:10E0300040927214872B423409582334CEE11314D2
:10E0400015BFE134D206D1145C75B0149BCC80347A
:10E050002D716435EAC8541564BB3515A302053526
:10E06000785CF715BFE5C7353196A635F62F9615BE
:10E070005DED6F369A545F1614273E16D39E0E360A
:10E0800008C0FC16CF79CC36410AAD3686B39D1652
:10E09000300E7917F7B7493779C42837BE7D18177E
:10E0A0006523EA37A29ADA172CE9BB17EB508B37B6
:10E0B00080E35C18475A6C38C9290D380E903D181A
:10E0C000D5CECF381277FF189C049E185BBDAE38B2
:10E0D000ED004A392AB97A19A4CA1B1963732B397E
:10E0E000B82DD9197F94E939F1E78839365EB81926
:10E0F0009D9C413A5A25711AD456101A13EF203AB2
:10E10000C8B1D21A0F08E23A817B833A46C2B31AE9
:10E11000F07F571B37C6673BB9B5063B7E0C361BF5
:10E12000A552C43B62EBF41BEC98951B2B21A53B3D
:10E130007DA4563CBA1D661C346E071CF3D7373CD1
:10E140002889C51CEF30F53C6143943CA6FAA41C19
:10E150001047401DD7FE703D598D113D9E34211D45
:10E16000456AD33D82D3E31D0CA0821DCB19B23D7D
:10E1700060DB4B1EA7627B3E29111A3EEEA82A1EC9
:10E1800035F6D83EF24FE81E7C3C891EBB85B93E71
:10E190000D385D3FCA816D1F44F20C1F834B3C3F1D
:10E1A0005815CE1F9FACFE3F11DF9F3FD666AF1FB5
:10E1B00000002110422063308440A550C660E77003
:10E1C000088129914AA16BB18CC1ADD1CEE1EFF1AB
:10E1D0003112100273325222B5529442F772D66253
:10E1E000399318837BB35AA3BDD39CC3FFF3DEE3FB
:10E1F0006224433420040114E664C774A4448554A3
:10E200006AA54BB528850995EEE5CFF5ACC58DD54A
:10E210005336722611163006D776F6669556B446F2
:10E220005BB77AA719973887DFF7FEE79DD7BCC79A
:10E23000C448E5588668A778400861180228233842
:10E24000CCC9EDD98EE9AFF9488969990AA92BB9EA
:10E25000F55AD44AB77A966A711A500A333A122A92
:10E26000FDDBDCCBBFFB9EEB799B588B3BBB1AAB3A
:10E27000A66C877CE44CC55C222C033C600C411CE2
:10E28000AEED8FFDECCDCDDD2AAD0BBD688D499D8A
:10E29000977EB66ED55EF44E133E322E511E700E32
:10E2A0009FFFBEEFDDDFFCCF1BBF3AAF599F788FDA
:10E2B0008891A981CAB1EBA10CD12DC14EF16FE1BA
:10E2C0008010A100C230E3200450254046706760F2
:10E2D000B9839893FBA3DAB33DC31CD37FE35EF30A
:10E2E000B1029012F322D232354214527762567242
:10E2F000EAB5CBA5A89589856EF54FE52CD50DC55A
:10E30000E234C324A0148104667447642454054491
:10E31000DBA7FAB79987B8975FE77EF71DC73CD7A9
:10E32000D326F2369106B0165766767615463456E1
:10E330004CD96DC90EF92FE9C899E9898AB9ABA9F9
:10E340004458654806782768C018E1088238A32831
:10E350007DCB5CDB3FEB1EFBF98BD89BBBAB9ABB49
:10E36000754A545A376A167AF10AD01AB32A923A81
:10E370002EFD0FED6CDD4DCDAABD8BADE89DC98D99
:10E38000267C076C645C454CA23C832CE01CC10CD1
:10E390001FEF3EFF5DCF7CDF9BAFBABFD98FF89FE9
:10E3A000176E367E554E745E932EB23ED10EF01E21
:10E3B0000000891112239B322446AD573665BF7485
:10E3C000488CC19D5AAFD3BE6CCAE5DB7EE9F7F835
:10E3D0008110080193331A22A5562C47B7753E6465
:10E3E000C99C408DDBBF52AEEDDA64CBFFF976E815
:10E3F00002218B30100299132667AF763444BD5545
:10E400004AADC3BC588ED19F6EEBE7FA7CC8F5D9F4
:10E4100083310A2091121803A7772E66B5543C4524
:10E42000CBBD42ACD99E508FEFFB66EAFDD874C9D4
:10E4300004428D5316619F702004A9153227BB3604
:10E440004CCEC5DF5EEDD7FC6888E1997AABF3BAB4
:10E4500085520C4397711E60A1142805B3373A26E4
:10E46000CDDE44CFDFFD56ECE9986089FBBB72AA94
:10E4700006638F7214409D512225AB343006B917C4
:10E480004EEFC7FE5CCCD5DD6AA9E3B8788AF19B74
:10E4900087730E6295501C41A3352A24B1163807A4
:10E4A000CFFF46EEDDDC54CDEBB962A8F99A708B54
:10E4B000088481951AA793B62CC2A5D33EE1B7F084
:10E4C0004008C919522BDB3A644EED5F766DFF7C34
:10E4D000899400859BB712A6ADD224C3BFF136E064
:10E4E000C1184809D33B5A2AE55E6C4FF77D7E6C14
:10E4F0000AA583B4188691972EE3A7F23CC0B5D144
:10E500004229CB38500AD91B666FEF7E744CFD5DF3
:10E510008BB502A499961087AFF326E2BDD034C123
:10E52000C3394A28D11A580BE77F6E6EF55C7C4DD3
:10E530000CC685D71EE597F42880A1913AA3B3B203
:10E54000444ACD5B5669DF78600CE91D722FFB3EB3
:10E550008DD604C79FF516E4A9902081BBB332A2E3
:10E56000C55A4C4BD7795E68E11C680DF33F7A2E93
:10E570000EE787F61CC495D52AA1A3B03882B193C3
:10E58000466BCF7A5448DD59622DEB3C700EF91F73
:10E590008FF706E69DD414C5ABB122A0B9923083A3
:10E5A000C77B4E6AD5585C49E33D6A2CF11E780F53
:10E5B00000000000B71DC1046E3B8209D926430D3F
:10E5C000DC7604136B6BC517B24D861A0550471ED7
:10E5D000B8ED08260FF0C922D6D68A2F61CB4B2B77
:10E5E000649B0C35D386CD310AA08E3CBDBD4F381F
:10E5F00070DB114CC7C6D0481EE09345A9FD5241BF
:10E60000ACAD155F1BB0D45BC2969756758B565256
:10E61000C836196A7F2BD86EA60D9B6311105A67F6
:10E6200014401D79A35DDC7D7A7B9F70CD665E749E
:10E63000E0B6239857ABE29C8E8DA19139906095FE
:10E640003CC0278B8BDDE68F52FBA582E5E6648616
:10E65000585B2BBEEF46EABA3660A9B7817D68B336
:10E66000842D2FAD3330EEA9EA16ADA45D0B6CA05E
:10E67000906D32D42770F3D0FE56B0DD494B71D97E
:10E680004C1B36C7FB06F7C32220B4CE953D75CA96
:10E6900028803AF29F9DFBF646BBB8FBF1A679FFB6
:10E6A000F4F63EE143EBFFE59ACDBCE82DD07DECDE
:10E6B00077708634C06D4730194B043DAE56C5396E
:10E6C000AB0682271C1B4323C53D002E7220C12AA6
:10E6D000CF9D8E1278804F16A1A60C1B16BBCD1FA6
:10E6E00013EB8A01A4F64B057DD00808CACDC90CEE
:10E6F00007AB9778B0B6567C69901571DE8DD475EE
:10E70000DBDD936B6CC0526FB5E6116202FBD06625
:10E71000BF469F5E085B5E5AD17D1D576660DC5325
:10E7200063309B4DD42D5A490D0B1944BA16D8406D
:10E7300097C6A5AC20DB64A8F9FD27A54EE0E6A1AD
:10E740004BB0A1BFFCAD60BB258B23B69296E2B265
:10E750002F2BAD8A98366C8E41102F83F60DEE87E5
:10E76000F35DA9994440689D9D662B902A7BEA94AD
:10E77000E71DB4E0500075E4892636E93E3BF7ED2D
:10E780003B6BB0F38C7671F7555032FAE24DF3FEE5
:10E790005FF0BCC6E8ED7DC231CB3ECF86D6FFCB65
:10E7A0008386B8D5349B79D1EDBD3ADC5AA0FBD82D
:10E7B000EEE00C6959FDCD6D80DB8E6037C64F648D
:10E7C0003296087A858BC97E5CAD8A73EBB04B7745
:10E7D000560D044FE110C54B383686468F2B474205
:10E7E0008A7B005C3D66C158E4408255535D4351CD
:10E7F0009E3B1D252926DC21F0009F2C471D5E280D
:10E80000424D1936F550D8322C769B3F9B6B5A3BC4
:10E8100026D6150391CBD40748ED970AFFF0560E84
:10E82000FAA011104DBDD014949B93192386521D4C
:10E830000E562FF1B94BEEF5606DADF8D7706CFC4C
:10E84000D2202BE2653DEAE6BC1BA9EB0B0668EF84
:10E85000B6BB27D701A6E6D3D880A5DE6F9D64DAC4
:10E860006ACD23C4DDD0E2C004F6A1CDB3EB60C90C
:10E870007E8D3EBDC990FFB910B6BCB4A7AB7DB0CC
:10E88000A2FB3AAE15E6FBAACCC0B8A77BDD79A304
:10E89000C660369B717DF79FA85BB4921F46759644
:10E8A0001A163288AD0BF38C742DB081C33071858C
:10E8B00099908A5D2E8D4B59F7AB085440B6C950DC
:10E8C00045E68E4EF2FB4F4A2BDD0C479CC0CD43F4
:10E8D000217D827B9660437F4F460072F85BC17654
:10E8E000FD0B86684A16476C93300461242DC5657C
:10E8F000E94B9B115E565A1587701918306DD81C5C
:10E90000353D9F0282205E065B061D0BEC1BDC0F73
:10E9100051A69337E6BB52333F9D113E8880D03AD3
:10E920008DD097243ACD5620E3EB152D54F6D429FB
:10E930007926A9C5CE3B68C1171D2BCCA000EAC81B
:10E94000A550ADD6124D6CD2CB6B2FDF7C76EEDBB3
:10E95000C1CBA1E376D660E7AFF023EA18EDE2EE93
:10E960001DBDA5F0AAA064F4738627F9C49BE6FD3B
:10E9700009FDB889BEE0798D67C63A80D0DBFB849B
:10E98000D58BBC9A62967D9EBBB03E930CADFF9733
:10E99000B110B0AF060D71ABDF2B32A66836F3A213
:10E9A0006D66B4BCDA7B75B8035D36B5B440F7B1BB
:10E9B00030313233343536373839414243444546B5
:10E9C0000051434F4D206661737420646F776E6C05
:10E9D0006F61642070726F746F636F6C20686F7307
:10E9E000740051434F4D206661737420646F776EDD
:10E9F0006C6F61642070726F746F636F6C207461F0
:10EA00007267000036000000040309043E03510051
:10EA1000750061006C0063006F006D006D002000E8
:10EA2000430044004D004100200054006500630095
:10EA300068006E006F006C006F0067006900650081
:10EA4000730020004D0053004D002403500072005D
:10EA50006F00640075006300740020006E006100A8
:10EA60006D006500200068006500720065002203EB
:10EA700031003200330034003500360037003800F2
:10EA80003900300041004200430044004500460088
:10EA900000020000000200000A0000000B0000005D
:10EAA0000000000001010100020201000202010059
:10EAB0000201000000000001010101020202020344
:10EAC00003030000900000000000000001000000AF
:10EAD000CF000100D000000001000000803E0000D7
:10EAE0000000000001000000FE010000FF00000027
:10EAF000000000006842000000000000010000006B
:10EB0000FE010000FF00000000000000004B0000BC
:10EB10000000000000000000FE010000FF000000F7
:10EB200000000000A86100000000000000000000DC
:10EB3000FE010000FF0000000000000050C30000C4
:10EB40000000000000000000FE010000FF000000C7
:10EB50000000000005000000000000000E000000A2
:10EB6000010000000F000000020000000D00000086
:10EB70000300000007000000040000000600000081
:10EB80000500000000000000000000000A00000076
:10EB900004000000A5EF002A0000000000000000B3
:10EBA00054EB002A010000008CEB002A0100000059
:10EBB000BDC7002ABDC7002AD9C7002ADBC7002A63
:10EBC000DDC7002A000000000000000003C8002A82
:10EBD0002BC8002A00000000000000009FCA002A85
:10EBE000B5CA002A45C8002AFDC8002A1DCB002A44
:10EBF00061CB002AA7CB002AEFCB002A000000003F
:10EC00000000000075C9002A8BC9002AADC9002A7E
:10EC1000D3C9002AE1C9002AEFC9002A0FCA002A75
:10EC200099CA002A99CA002A9BCA002A9DCA002AAA
:10EC300000000000000000000000000000000000D4
:10EC40000000000000000000000000009FCA002A31
:10EC5000B5CA002A00000000000000001DCB002AF9
:10EC600061CB002AA7CB002AEFCB002A00000000CE
:10EC70000000000000000000000000000000000094
:10EC80000000000000000000000000000000000084
:10EC900041524D5052472073697A65206D73672049
:10ECA0006F76657272756E00546F74616C20627954
:10ECB00074657320726563642062792041524D50FF
:10ECC000524720307800534443435F4552525F44DB
:10ECD0004D4100534443435F4552525F5344494FB3
:10ECE0005F5245414400534443435F4552525F5392
:10ECF00050535F4D4F44455F555345440053444383
:10ED0000435F4552525F434152445F554E44455420
:10ED1000454354454400534443435F4552525F4684
:10ED20004541545552455F554E535550504F5254DE
:10ED3000454400534443435F4552525F434152446C
:10ED40005F52454D4F56454400534443435F45523F
:10ED5000525F524541445F5345435F434D445F4ECC
:10ED60004F545F414C4C4F57454400534443435F1D
:10ED70004552525F41424F52545F524541445F53A6
:10ED800045435F434D4400534443435F4552525F04
:10ED900050524F475F444F4E4500534443435F45F5
:10EDA00052525F455241534500534443435F4552DD
:10EDB000525F494E56414C49445F54585F53544149
:10EDC000544500534443435F4552525F5344494FB7
:10EDD0005F575249544500534443435F4552525F85
:10EDE00053574954434800534443435F4552525F8D
:10EDF000444154415F4352435F4641494C005344B0
:10EE000043435F4552525F434D445F4352435F4625
:10EE100041494C00534443435F4552525F494E566B
:10EE2000414C49445F504152414D00534443435F7C
:10EE30004552525F57505F56494F4C4154494F4ECF
:10EE400000534443435F4552525F554E4B4E4F571C
:10EE50004E00534443435F4552525F524541445F25
:10EE60004649464F00534443435F4552525F575211
:10EE70004954455F4649464F00534443435F45521A
:10EE8000525F5344494F00534443435F4552525FDE
:10EE90005344494F5F52355F5245535000534443EA
:10EEA000435F4E4F5F4552524F5200534443435FBE
:10EEB0004552525F5350535F57524954494E475F32
:10EEC00044455343524950544F5200534443435FC7
:10EED0004552525F5345435552455F434F4D4D4157
:10EEE0004E445F494E5F50524F4752455353005373
:10EEF0004443435F4552525F434152445F494E4948
:10EF00005400534443435F4552525F444D4C5F4964
:10EF10004E495400534443435F4552525F434D446E
:10EF20005F53454E5400534443435F4552525F5331
:10EF300050535F4745545F4556454E540053444334
:10EF4000435F4552525F5057525F4F4E5F57524991
:10EF500054455F50524F5400534443435F4552520F
:10EF60005F434D445F54494D454F5554005344430E
:10EF7000435F4552525F54494D454F5554005344E9
:10EF800043435F4552525F434152445F52454144BF
:10EF90005900534443435F4552525F5345545F42C7
:10EFA0004C4B535A0048414C5F5342495F535342C4
:10EFB000495F56325F504D49435F41524249544583
:10EFC00052000000ED02002AED02002AED02002AA4
:10EFD000ED02002A00000000000000001C035100A8
:10EFE000480053005500530042005F0041005200AA
:10EFF0004D005000520047000F04002AED03002A84
:10F00000CD03002AB103002AC103002A0001000039
:10F0100000000000000000000100000000000000EF
:10F02000A8EC002A90EC002A00000000000000007C
:10F0300000000000000000000000000000000000D0
:10F040007709002A6509002A930A002A6509002A1F
:10F05000710C002A6509002A830C002A6509002A20
:10F060001B10002A6509002A290C002A6509002ABC
:10F070006509002A6509002A6509002A6509002A30
:10F080004D10002A6509002A6B10002A6509002A24
:10F09000CF10002A6509002A2111002A6509002ADB
:10F0A0005911002A6509002AF511002A6509002A6C
:10F0B0000B0D002A6509002A9912002A6509002A09
:10F0C0006509002A6509002AA50A002A6509002A9F
:10F0D0006509002A6509002A0B18002A6509002A1B
:10F0E0007516002A6509002AFF16002A6509002AFC
:10F0F0006509002A6509002A6509002A6509002AB0
:10F100005118002A6509002A5519002A6509002AA4
:10F110008D18002A6509002A000000000000000088
:10F12000000000000000000012010002000000408A
:10F13000C60508900000010200010902200001013B
:10F140000080010904000002FFFFFF0007058102A3
:10F1500040000007050102400000000070F1002A95
:10F160000000000084F1002A000000000000000000
:10F17000000000000000000084F1002A00000000F0
:10F180000000000000000000000000009CF1002AC8
:10F190005CF1002A000000000000000000000000F8
:10F1A00000000000ACF1002A000000000000000098
:10F1B0009CF1002A48F2002A00000000D51C002A19
:10F1C000000000000000000000000000000000003F
:10F1D000000000000000000000000000000000002F
:10F1E000000000000000000000000000000000001F
:10F1F000000000000000000000000000000000000F
:10F2000000000000000000000000000000000000FE
:10F2100000000000000000000000000000000000EE
:10F2200000000000000000000000000000000000DE
:10F2300000000000000000000000000000000000CE
:10F24000000000000000000054F2002A08EA002A32
:10F250000000000060F2002A0CEA002A0904010004
:10F260006CF2002A4AEA002A0904020000000000A9
:10F270006EEA002A09040300F40100001126002AA6
:10F280003B26002A2B25002A000000000000000079
:10F29000000000000000000000000000000000006E
:10F2A0000000000001000000030000000300000057
:10F2B0000000000000010203010000000000000047
:10F2C000000000000000000000000000000000003E
:10F2D000000000000000000000000000000000002E
:10F2E000000000009DEE002A41EE002A58EF002A9F
:10F2F0006DEF002AFEED002AE7ED002A14EF002A48
:10F3000087ED002A7EEF002AA9ED002A92EF002A5D
:10F3100087EE002AC6EC002A52EE002A65EE002A8B
:10F320009AED002A79EE002AD3EC002AC3ED002AD8
:10F33000D7ED002A14EE002AFDEC002A16ED002A73
:10F34000CBEE002A49ED002A6BED002AEFEE002AF1
:10F3500033ED002A3DEF002A2BEE002AE6EC002ACE
:10F3600002EF002A26EF002AABEE002A0000000080
:10F37000000050120000000000000000000000002B
:10F38000000000000000000000000000000000007D
:10F39000000000004A52443A3132333435363738AF
:10F3A00039303A544553540000000000000000007A
:10F3B00000000000140000000A000000000000002F
:10F3C000000000000000000000000000000000003D
:10F3D00000000000200000002100000000000000EC
:10F3E000020000000000000000000000000000001B
:10F3F000D89E05C107D57C3617DD703039590EF718
:10F40000310BC0FF11155868A78FF964A44FFABEDD
:10F4100067E6096A85AE67BB72F36E3C3AF54FA5A5
:10F420007F520E518C68059BABD9831F19CDE05BD1
:10F43000D89E05C15D9DBBCB07D57C362A299A6233
:10F4400017DD70305A01599139590EF7D8EC2F1544
:10F45000310BC0FF6726336711155868874AB48E91
:10F46000A78FF9640D2E0CDBA44FFABE1D48B547DB
:10F4700008C9BCF367E6096A3BA7CA8485AE67BBC7
:10F480002BF894FE72F36E3CF1361D5F3AF54FA5F2
:10F49000D182E6AD7F520E511F6C3E2B8C68059BCE
:10F4A0006BBD41FBABD9831F79217E1319CDE05B86
:10F4B000982F8A4291443771CFFBC0B5A5DBB5E9DF
:10F4C0005BC25639F111F159A4823F92D55E1CAB53
:10F4D00098AA07D8015B8312BE853124C37D0C55E1
:10F4E000745DBE72FEB1DE80A706DC9B74F19BC129
:10F4F000C1699BE48647BEEFC69DC10FCCA10C2419
:10F500006F2CE92DAA84744ADCA9B05CDA88F976FC
:10F5100052513E986DC631A8C82703B0C77F59BF66
:10F52000F30BE0C64791A7D55163CA066729291492
:10F53000850AB72738211B2EFC6D2C4D130D38532F
:10F5400054730A65BB0A6A762EC9C281852C7292F1
:10F55000A1E8BFA24B661AA8708B4BC2A3516CC71F
:10F5600019E892D1240699D685350EF470A06A1058
:10F5700016C1A419086C371E4C774827B5BCB034A7
:10F58000B30C1C394AAAD84E4FCA9C5BF36F2E6845
:10F59000EE828F746F63A5781478C8840802C78CD4
:10F5A000FAFFBE90EB6C50A4F7A3F9BEF27871C6D7
:10F5B00022AE28D7982F8A42CD65EF239144377128
:10F5C0002F3B4DECCFFBC0B5BCDB8981A5DBB5E99A
:10F5D00038B548F35BC2563919D005B6F111F15967
:10F5E0009B4F19AFA4823F9218816DDAD55E1CAB98
:10F5F000420203A398AA07D8BE6F7045015B83122D
:10F600008CB2E44EBE853124E2B4FFD5C37D0C55E7
:10F610006F897BF2745DBE72B196163BFEB1DE80DF
:10F620003512C725A706DC9B942669CF74F19BC1D0
:10F63000D24AF19EC1699BE4E3254F388647BEEF6D
:10F64000B5D58C8BC69DC10F659CAC77CCA10C2425
:10F6500075022B596F2CE92D83E4A66EAA84744A97
:10F66000D4FB41BDDCA9B05CB5531183DA88F976CF
:10F67000ABDF66EE52513E981032B42D6DC631A804
:10F680003F21FB98C82703B0E40EEFBEC77F59BFE8
:10F69000C28FA83DF30BE0C625A70A934791A7D5D3
:10F6A0006F8203E05163CA06706E0E0A672929143F
:10F6B000FC2FD246850AB72726C9265C38211B2E87
:10F6C000ED2AC45AFC6D2C4DDFB3959D130D3853B4
:10F6D000DE63AF8B54730A65A8B2773CBB0A6A76C7
:10F6E000E6AEED472EC9C2813B358214852C72925D
:10F6F0006403F14CA1E8BFA2013042BC4B661AA8DA
:10F700009197F8D0708B4BC230BE5406A3516CC792
:10F710001852EFD619E892D110A96555240699D64A
:10F720002A20715785350EF4B8D1BB3270A06A100B
:10F73000C8D0D2B816C1A41953AB4151086C371EBA
:10F7400099EB8EDF4C774827A8489BE1B5BCB034D5
:10F75000635AC9C5B30C1C39CB8A41E34AAAD84EB7
:10F7600073E363774FCA9C5BA3B8B2D6F36F2E687E
:10F77000FCB2EF5DEE828F74602F17436F63A57844
:10F7800072ABF0A11478C884EC39641A0802C78CF3
:10F79000281E6323FAFFBE90E9BD82DEEB6C50A405
:10F7A0001579C6B2F7A3F9BE2B5372E3F27871C68E
:10F7B0009C6126EACE3E27CA07C2C021C7B886D1BF
:10F7C0001EEBE0CDD67DDAEA78D16EEE7F4F7DF587
:10F7D000BA6F1772AA67F006A698C8A2C57D630A19
:10F7E000AE0DF9BE04983F111B471C13350B711B5E
:10F7F000847D0423F577DB289324C7407BABCA3292
:10F80000BCBEC9150ABE9E3C4C0D109CC4671D436E
:10F81000B6423ECBBED4C54C2A7E65FC9C297F599E
:10F82000ECFAD63AAB6FCB5F1758474A8C19446C49
:10F8300030F5BDDC4DECE7FEC7F8999937965DE2EF
:10F84000135049E8565EF63EC448502AD08B2CA18E
:10F8500051C481506D11311DC3EF1C0F4E15F1BE07
:10F860000BAD806BA0DDA60DC184362A29E45C7344
:10F87000C4F4E21A557E9A54BBC8E37D71B7C841FF
:10F8800074471F16B8757726F31A7604755CBAA00C
:10F890007F55972CE1AA26B2020EFCE914B03D7503
:10F8A000F309B2687C07296BF85B48AFE5877156AE
:10F8B000337D0347BB190F4DE9C97A06E34229FCA2
:10F8C000C9737CAAE9F15E16E5BA11B614D17422A7
:10F8D00058F42BC95F3805F81B33B23BDD29FD0B0B
:10F8E000209FB1AE8CFDA1F9CE2044EA2F322EF339
:10F8F00049F0A76508C5C94CC04E511B6902345276
:10F90000FD7CB930194AB6B228E115A7FECE68468B
:10F9100080BAE73F5061C9D3389052526A6D8692DF
:10F9200002880AB5423FD8F4EE6D1BD9C0C11F7ED4
:10F93000308204C1308203A9A00302010202030045
:10F940009766300D06092A864886F70D01010505E0
:10F9500000307D310B300906035504061302555360
:10F96000310B3009060355040813024341311130AD
:10F970000F0603550407130853414E444945474FAA
:10F98000310C300A060355040A13034F454D312349
:10F990003021060355040B131A47656E6572616CBE
:10F9A000204F454D206174746573746174696F6E86
:10F9B000204341311B3019060355040313124F45F0
:10F9C0004D206174746573746174696F6E20434176
:10F9D000301E170D31333036323530323439303055
:10F9E0005A170D3333303632303032343930305AE2
:10F9F0003082014D310B30090603550406130255C0
:10FA000053312F302D060355040313265175616CB5
:10FA1000636F6D6D20446576656C6F706D656E7497
:10FA2000205369676E696E6720546F6F6C20557341
:10FA30006572311230100603550407130953616EC5
:10FA400020446965676F310D300B060355040A13B6
:10FA50000441534943311330110603550408130A76
:10FA600043616C69666F726E696131173015060308
:10FA700055040B140E30342030303432204F454DB5
:10FA80005F4944311C301A060355040B14133035FA
:10FA90002030303030463833302053575F53495A86
:10FAA0004531193017060355040B14103036203039
:10FAB000303037204D4F44454C5F494431173015A5
:10FAC000060355040B130E303720303030312053ED
:10FAD000484132353631223020060355040B1419C3
:10FAE0003031203030303030303030303030303025
:10FAF0003030332053575F494431223020060355BC
:10FB0000040B141930322030303732433045313055
:10FB1000303432303030372048575F49443122305A
:10FB200020060355040B13193033203030303030A9
:10FB3000303030303030303030304620444542555F
:10FB40004730820120300D06092A864886F70D01CC
:10FB5000010105000382010D0030820108028201CB
:10FB60000100C220B80903EC6E9894B0E4B1455B83
:10FB700030349DF219DA93188CA452327ED03EF0C4
:10FB8000CE4F62A837FD5CB97A2AE88ED5D49D9A0B
:10FB900004C55017A4212A909DD63A683CD026E788
:10FBA000037D7D709733D5A32832E8A246A3A0F940
:10FBB00032705E5C5AFF17DC4424A35051FC52C8DB
:10FBC000CE116A9342AA19E3CBA319807F65F08610
:10FBD000EACD72AA23EF40189FB026E97A49573937
:10FBE0004E6455AEC3DA080EF40655C559B746CA79
:10FBF0003214431CEF4619044A25CB17A643673934
:10FC0000AEAD65AEF39E0C980504B2AA5064DB0F4E
:10FC100044CD1ECB9A105AAA2C34397874EE7365F1
:10FC2000E0582DE0DC4BA0E3D592D747312F1515D6
:10FC3000296B190AF010388BB12DDD3A80264494D7
:10FC400035BB66677E981EE0E47ACF4FAAFC826ED1
:10FC500032AB15936770C38122CCDF2EAA97C8B749
:10FC60000A8B020103A37A3078303A0603551D1F30
:10FC700004333031302FA02DA02B86296874747086
:10FC80003A2F2F63726C2E716473742E636F6D2F15
:10FC900063726C732F7163746465766174746573D9
:10FCA000742E63726C301F0603551D230418301622
:10FCB000801487E3401C348CA7E03E42B80A329A95
:10FCC0008D9A4805EBE8300C0603551D13040530EA
:10FCD00003020100300B0603551D0F040403020448
:10FCE000F0300D06092A864886F70D01010505004A
:10FCF000038201010002F2EE2E2895EAB3640DFBA7
:10FD000094C47ABC4EB9095979B282D14D6D241E82
:10FD10007E2388C39FD691ADF4BDB0AF7A1542EA79
:10FD2000121CDE4D9CEE615CFF70AD6731FB5CEA3E
:10FD30002C0B651F74DA6CF0741A80637D3BD964F8
:10FD4000BB74ABA78D08529B71F0DE222053CAC74B
:10FD50007DAB5209768C85BB8E43942B870E60C792
:10FD6000D4482181FCBCDC2894F98CD140FA65AAE6
:10FD7000DB7789242962A01179B8F2C9D61FC07D2A
:10FD80006B6BFF2C7E5E6D4441231EF623A0060C98
:10FD9000C240C6A141E96F092E8E4BBE99FCF7EA1D
:10FDA0005BCE1FA9B9D21EADCF689FBC133195CBD6
:10FDB0006296456E5C94C0C34123A077D885ECE77A
:10FDC000D70B6D2B403E9F4782485E8B26591D51B5
:10FDD000001E62962BDB735C13B1FFEE5A2998610B
:10FDE000605F7020DA342C34FAD3241496926BB30B
:10FDF0002CF33F86FE308203C4308202ACA00302A3
:10FE00000102020105300D06092A864886F70D0118
:10FE100001050500306E310B300906035504061349
:10FE2000025553310B3009060355040813024341B0
:10FE30003111300F0603550407130853414E44494E
:10FE400045474F310C300A060355040A13034F454A
:10FE50004D311B3019060355040B131247656E65AF
:10FE600072616C204F454D20726F6F746361311465
:10FE700030120603550403130B4F454D20524F4FCC
:10FE800054204341301E170D313330313038303774
:10FE9000313831325A170D33333031303330373156
:10FEA0003831325A307D310B3009060355040613C0
:10FEB000025553310B300906035504081302434120
:10FEC0003111300F0603550407130853414E4449BE
:10FED00045474F310C300A060355040A13034F45BA
:10FEE0004D31233021060355040B131A47656E6507
:10FEF00072616C204F454D20617474657374617438
:10FF0000696F6E204341311B3019060355040313FA
:10FF1000124F454D206174746573746174696F6E1E
:10FF200020434130820120300D06092A864886F799
:10FF30000D01010105000382010D0030820108025C
:10FF400082010100AE0CFCF74BD9ADCDD7F34B7558
:10FF5000C87C404FD3BDB1FDB961BC61A31DC75E74
:10FF6000242552A3E242AA095742697357E55AC2AF
:10FF70007F042C8B098B3E7B4AC067D4F3492A1C33
:10FF80009C6DD768F9E663BE42A4BE6921F6AC3029
:10FF9000DBB22245226574D7E56109EFC3BB24CBF0
:10FFA000F4370B429A71C6A57E9AE67036A34F17B6
:10FFB000E2C9BDDC8268D671909D7CEC8E0A3CE182
:10FFC00012BF7EED4161AA7C4E8FAC4349B383736F
:10FFD000B0876B31754ECDD77BAFAAA072B3F963F2
:10FFE000E6D1460BF730426E60C125F0C30ADD5FF3
:10FFF000C225D3A046E38F9DE77DFAEF60938D463F
:020000042A01CF
:100000002F598E2A154936840967F85CB6DE51648B
:10001000A8DCCA8CE478E635200A04A2AAB63D0B17
:100020003E54CAF01C7AB779566DCE02495536FD5A
:100030003E6E50FCC54A099B2ECF568C77474A2509
:1000400066F8662B020103A360305E301F0603557D
:100050001D23041830168014C987BFD0C31B9B5CB6
:1000600066A8FECC94B8733E1A9CC692301D060357
:10007000551D0E0416041487E3401C348CA7E03E83
:1000800042B80A329A8D9A4805EBE8300F060355BC
:100090001D13040830060101FF020100300B0603A6
:1000A000551D0F040403020106300D06092A864877
:1000B00086F70D010105050003820101005EA347DB
:1000C0004A7E0A427F8B1466D20575E6B2DCABD35A
:1000D00068418D1DE3ABA0F5982F4715E0A7DF2AF7
:1000E0001BD41327BF91FFFC76BDB32E55368EDE91
:1000F00045439EC8E77F1E8EE7D26CFDC6682A6D19
:100100004C9952494C2E37784388C7803A4EB67B7B
:1001100038F84474A7690EACD219D8BFF6AA851472
:10012000D38176001600F31D5C5BC63DB4E12798D1
:10013000CCD8574F5F748876E343B085A7CF6F6FF5
:10014000AE9D691DED97AA913371F4D12FC4CFA94B
:100150008F18FBA067E6B46F5EDDAD6CD2256F240F
:10016000CD5BAB3CD872E22C8C0DA3C2BD9D36C0DA
:10017000C8090A8ABA0149BEA270E897DA64214028
:10018000C4E61B6019708A5BE51A7A1CF5FCF28ED6
:1001900032C50BAF29D36774E4E54AD234F20CDFE1
:1001A0005A8C89D587F544BADC636CE2FF51BC39BF
:1001B000D1A44D305938C7EC7B2DD4A558308203DB
:1001C0009130820279A003020102020101300D0682
:1001D000092A864886F70D0101050500306E310BAE
:1001E0003009060355040613025553310B30090636
:1001F00003550408130243413111300F060355041F
:1002000007130853414E444945474F310C300A0605
:100210000355040A13034F454D311B30190603558E
:10022000040B131247656E6572616C204F454D20BB
:10023000726F6F7463613114301206035504031337
:100240000B4F454D20524F4F54204341301E170D48
:100250003133303130383037313030305A170D3398
:1002600033303130333037313030305A306E310B3B
:100270003009060355040613025553310B300906A5
:1002800003550408130243413111300F060355048E
:1002900007130853414E444945474F310C300A0675
:1002A0000355040A13034F454D311B3019060355FE
:1002B000040B131247656E6572616C204F454D202B
:1002C000726F6F74636131143012060355040313A7
:1002D0000B4F454D20524F4F542043413082012057
:1002E000300D06092A864886F70D01010105000335
:1002F00082010D00308201080282010100C4264CF7
:10030000F82F725637C8EDBEC403903DA8BC788D57
:10031000D005B46C5130ECC6AB7162FC27E693ABF0
:10032000B2367C8D86A2DA9DCBC1F37A48100CBE22
:1003300084582F202949CC91049AA014FFF3873EBA
:100340002D3675AB58B18068F74388208B491EE382
:1003500023F8B41807A7124BD93F189EEE32D1DB11
:100360007EBB87B4FD5FD2F0BF378BD8F0A9C4E75E
:1003700080E25F5F4575BD7D29D22F010B019D0194
:10038000883EFE25B5721ED6288B92023B3434B5CA
:100390008978E4271DE89BC43D40A48A8FA16E4262
:1003A0001177C73DC239E33FD8B66DF86956C99495
:1003B000B9B802745F1E32BDBCB05F070D39396336
:1003C000B08716BC4DEB9E6E8314E180A196A1DA36
:1003D0007A7774F6CCC2A29E4ACCCBDF956548589A
:1003E00046E1817171210EB627A9C70E01931D0246
:1003F00066DB9475C89B9E7CEF2AC4EA3102010338
:10040000A33C303A301D0603551D0E04160414C9D2
:1004100087BFD0C31B9B5C66A8FECC94B8733E1A02
:100420009CC692300C0603551D13040530030101D0
:10043000FF300B0603551D0F040403020106300DA7
:1004400006092A864886F70D010105050003820189
:1004500001004E7AAEA1B194D3B307E737A35C870E
:10046000EA217459380C3750B6B2EB69DF6CC6001C
:100470006426820951A4342BC6C59ED03CF4C9E23F
:10048000017AF34FAF7CA96969C72DA589F1A67DD3
:10049000492E6BD808D41DBB9FD6F89B83F7939643
:1004A0001BB61C087E82D884DCD5F2957A4A2403D8
:1004B000F2E5F942C05A8962422E778AFF08CB4B97
:1004C00001E54EAC67F46D008B0EBDA3D2DA0223BA
:1004D000F1999A2653099AAAB5D89498DDC5D553AF
:1004E000218874EFB6C1D0C0ACF4B3A616A473AF24
:1004F000947CE0CCE430B95B6FC3481165AA9EECF4
:1005000071EE2381ED096BE8CBBEF61AFDEDDE94AA
:100510004068173C2B9B3C7046E866F78B2450D80C
:10052000383313F011E08EEDC0B525038A8D5518D0
:1005300091E8645C610A268A81F110B0684E7CB94A
:10054000EBEFABD7BFA0B196B7630506ECA27AC8B4
:1005500080D8FFFFFFFFFFFFFFFFFFFFFFFFFFFF51
:10056000FFFFFFFFFFFFFFFFFFFFFFFFFFFFFFFF9B
:10057000FFFFFFFFFFFFFFFFFFFFFFFFFFFFFFFF8B
:10058000FFFFFFFFFFFFFFFFFFFFFFFFFFFFFFFF7B
:10059000FFFFFFFFFFFFFFFFFFFFFFFFFFFFFFFF6B
:00000001FF
